:100000000C9486060C94A5060C94A5060C94A506E3
:100010000C94A5060C94A5060C941F090C945E097B
:100020000C94A5060C94A5060C94A5060C94A506A4
:100030000C94A5060C94A5060C94A5060C94D40C5F
:100040000C94A5060C94A5060C94A5060C94A50684
:100050000C94A1410C94C3380C94A5060C94A506ED
:100060000C94A5060C9498390C94A5060C948C3924
:100070000C94A5060C94A5060C94A5060C94A50654
:100080000C944D4E0C94A5060C94A5060C94A50654
:100090000C94D6390C94A5060C94CA390C94A50678
:1000A0000C94A5060C94A5060C94A5060C94A50624
:1000B0000C94A5060C94A5060C94A5060C94A50614
:1000C0000C94A5060C94A5060C94A5060C94A50604
:1000D0000C94A5060C94A5060C94A5060C94A506F4
:1000E0000C94A5060C945A410C9464410C94504114
:1000F0000C940A410C9495410C9486410C947A41DD
:100100000C946E410C94A5060C94A5060C94A506BF
:100110000C94A5060C94A5060C94A5060C94A506B3
:100120000A0025303278002025362E3266204F6EA8
:100130002D426F61726400202573002530327800F3
:100140002025362E3266200020257300756E6B6EDA
:100150006F776E20636D640A00256300682020209D
:10016000202020202020202020202020202020208F
:1001700020202020202020202D2068656C700A0D72
:100180000076202020202020202020202020202039
:10019000202020202020202020202020202D2076FC
:1001A000657273696F6E0A0D007520202020202073
:1001B000202020202020202020202020202020203F
:1001C00020202020202D20757074696D650A0D0097
:1001D000616573205B6F6E7C6F66665D20202020FA
:1001E0002020202020202020202020202D20696E6B
:1001F000746567726574790A0D006164632020205C
:1002000020202020202020202020202020202020EE
:100210002020202020202D2073686F7720765F69B2
:100220006E2C2061312C20613220766F6C746167F6
:1002300065730A0D0063616C69205B5B765F696EB4
:100240007C61317C61325D20766F6C746167655DC5
:10025000202D2063616C6962726174650A0D00640F
:1002600065205B6D61736B5D2020202020202020A5
:1002700020202020202020202020202D20646562A6
:1002800075670A0D0068756D202020202020202031
:10029000202020202020202020202020202020205E
:1002A000202D2068756D69646974792073656E739B
:1002B0006F720A0D0068756D70205B6F6E7C6F66E3
:1002C000665D2020202020202020202020202020AB
:1002D000202D2068756D6964697479207065726D70
:1002E0002073656E736F72207077720A0D006964F7
:1002F000205B72657365745D202020202020202003
:10030000202020202020202020202D20696420680B
:10031000616E646C696E670A0D006D637520202044
:1003200020202020202020202020202020202020CD
:100330002020202020202D206D637520696E666F9F
:100340000A0D006E65205B666C7573685D20202069
:100350002020202020202020202020202020202D90
:10036000206E65696768626F72207461626C650AED
:100370000D006C6F67205B6175746F7C6F6E7C6FB6
:1003800066665D20202020202020202020202D2097
:100390006D6F7465732064617461206F6E205553B6
:1003A000420A0D006F7720202020202020202020CE
:1003B000202020202020202020202020202020203D
:1003C0002D206F6E652D776972652073656E736F72
:1003D00072730A0D007265205B6D61736B5D202086
:1003E000202020202020202020202020202020200D
:1003F000202D206D6F7465207265706F727420738C
:10040000657474696E670A0D007269205B696E74A9
:100410005D2020202020202020202020202020209F
:1004200020202020202D207265706F727420696E4C
:1004300074657276616C0A0D007273202020202092
:1004400020202020202020202020202020202020AC
:1004500020202020202D20726164696F2073746138
:1004600074730A0D00737320202020202020202088
:10047000202020202020202020202020202020207C
:10048000202D207374617475732073756D6D6172A6
:10049000790A0D0070777231205B6F6E7C6F666633
:1004A0005D2020202020202020202020202020200F
:1004B0002D2070696E31207077720A0D007265739D
:1004C0007420656570726F6D202020202020202010
:1004D0002020202020202020202D20726573746F82
:1004E000726520656570726F6D0A0D00626F6F74C2
:1004F00020202020202020202020202020202020FC
:1005000020202020202020202D207265626F6F7413
:100510000A0D0075706772202020202020202020E6
:100520002020202020202020202020202020202DBE
:10053000207265626F6F742076696120626F6F74DC
:100540006C6F616465720A0D00557074696D652089
:10055000256420646179732C20253032643A25307B
:1005600032643A253032640A00204E657665722D79
:100570007573656420737461636B203E202564206D
:1005800062797465730A0025352E3266200025379E
:100590002E33662025372E3366002530327800252D
:1005A000730A004E65772064656275673D30782573
:1005B000580A0043757272656E74206465627567CF
:1005C0003D307825580A00445F4F5045523D307801
:1005D00025780A00445F52583D307825780A004457
:1005E0005F54583D307825780A00445F504B543DA5
:1005F0006E307825780A00445F4F573D3078257873
:100600000A00445F4C45443D307825780A00445F39
:10061000504F5745523D307825780A00445F455683
:10062000454E543D307825780A00445F50305F4C89
:1006300045443D307825780A00445F50315F4C4591
:10064000443D307825780A00445F4145533D307879
:1006500025780A00445F5057525F313D3078257845
:100660000A002563002563002563004F4B0A00251F
:1006700063007478206C656E202020202072682032
:100680006D697373202020207268207374616C651B
:100690002020207268206D6973630A00252D313097
:1006A0006C7520252D31306C7520252D31306C7501
:1006B00020252D31306C75200A002563004D4355EF
:1006C0003D2530366C780020467573653A206565A7
:1006D0003D253032782068663D25303278206C66C2
:1006E0003D25303278206C623D2530327800204F35
:1006F000534343414C3D256420002563002563009E
:100700002563002563004E6577207265706F7274F3
:100710003D307825580A005573696E672072657000
:100720006F72743D307825580A00525F49443D0984
:1007300009307825780A00525F543D090930782540
:10074000780A00525F54313D0909307825780A0053
:10075000525F545F4D43553D09307825780A005269
:100760005F565F4D43553D09307825780A00525F4A
:1007700050303D0909307825780A00525F50305FCB
:10078000543D0909307825780A00525F50313D09FF
:1007900009307825780A00525F50315F543D0909CD
:1007A000307825780A00525F555054494D453D092F
:1007B000307825780A00525F52483D090930782583
:1007C000780A00525F565F494E3D09093078257816
:1007D0000A00525F41313D0909307825780A0052FC
:1007E0005F41323D0909307825780A002563004EC3
:1007F0006577207265706F727420696E74657276A9
:10080000616C3D252D64207365630A004375727227
:10081000656E74207265706F727420696E74657293
:1008200076616C3D252D64207365630A00256300A5
:100830002563005374617475732053756D6D617217
:10084000790A49443D004E65696768626F72207499
:1008500061626C652073697A653D25640A005249BE
:100860004D4520616464723D252D642E252D640A5A
:1008700000526164696F205265706F727420496E16
:1008800074657276616C3D252D640A00526164695D
:100890006F205265706F7274204D61736B3D3078BC
:1008A000252D780A00565F494E3D252D352E32669E
:1008B0000A00565F4D43553D252D352E32660A0000
:1008C0005553425F5057523D25730A00546F74616F
:1008D0006C20696E74723A2050303D252D6C642076
:1008E00050313D252D6C640A004C6F67206D6F649C
:1008F0006520697320006175746F0A0025730A0012
:1009000048554D5F5057525F414C574159533D2513
:10091000730A0044656275673D3078252D780A00BA
:10092000507772312069732025730A0025630025F2
:10093000630052483D252D342E31662000545F520D
:10094000483D252D342E3166200025630058544142
:100950004C5F5452494D3D2564004572726F7220C0
:100960003020566F6C74004572726F7220302056C2
:100970006F6C74004572726F72203020566F6C7409
:100980000025352E3266200025372E336620253788
:100990002E33660025730A0025730A0025730A00AA
:1009A00025730A00256300256300532025642E2546
:1009B0006420636C6F636B20256C75207478202530
:1009C0006C7520727820256C752072747820256CE7
:1009D000752072727820256C75207265786D697447
:1009E00020256C752061636B747820256C75206EF2
:1009F0006F61636B747820256C752061636B72780E
:100A000020256C752074696D65646F757420256C84
:100A1000752062616461636B727820256C75207447
:100A20006F6F6C6F6E6720256C7520746F6F7368C5
:100A30006F727420256C752062616473796E6368CF
:100A400020256C752062616463726320256C7520BB
:100A5000636F6E74656E74696F6E64726F7020255B
:100A60006C752073656E64696E6764726F702025A3
:100A70006C75206C6C747820256C75206C6C7278A9
:100A800020256C750A00452025642E256420636CA2
:100A90006F636B20256C752063707520256C752045
:100AA0006C706D20256C752069727120256C752025
:100AB000676C656420256C7520796C656420256CF5
:100AC0007520726C656420256C7520747820256C07
:100AD00075206C697374656E20256C752073656E66
:100AE000736F727320256C752073657269616C2059
:100AF000256C750A000A2A2A2A2A2A2A2A426F6F96
:100B000074696E672025732A2A2A2A2A2A2A0A004B
:100B100052616E646F6D20455549363420616464BE
:100B2000726573732067656E6572617465640A002F
:100B30004D41432061646472657373200025783AE7
:100B4000000A0025732025732C206368616E6E6592
:100B50006C20257520706F776572202575002C201C
:100B6000636865636B207261746520257520487A1F
:100B7000000A004F6E6C696E650A00257325730AC2
:100B8000006C6F63616C686F73740041544D45472E
:100B9000413132387266613100020000FFFE000010
:100BA00001454550524F4D20697320636F72727535
:100BB00070742C20726577726974696E672077692A
:100BC00074682064656661756C74732E0A006E61CA
:100BD0006E00696E660000407A10F35A00A0724EF3
:100BE00018090010A5D4E80000E87648170000E4D2
:100BF0000B54020000CA9A3B000000E1F50500001A
:100C000080969800000040420F000000A08601007E
:100C10000000102700000000E8030000000064004E
:100C2000000000000A0000000000010000000000B9
:100C30002C76D888DC674F0823DFC1DFAE59E1B1DD
:100C4000B796E5E3E453C63AE651997696E8E6C2EC
:100C50008426EB898C9B62ED407C6FFCEFBC9C9FF3
:100C600040F2BAA56FA5F490055A2AF75C936B6C15
:100C7000F9676DC11BFCE0E40D47FEF520E6B50009
:100C8000D0ED902E0300943577050080841E080077
:100C900000204E0A000000C80C333333330F986E27
:100CA00012831141EF8D2114893BE65516CFFEE6E4
:100CB000DB18D1844B381BF77C1D901DA4BBE424AA
:100CC000203284725E228100C9F124ECA1E53D2727
:100CD000494E46494E4954594E414E00002041006C
:100CE00000C84200401C4620BCBE4CCA1B0E5AAE77
:100CF000C59D74CDCCCC3D0AD7233C17B7D13877EE
:100D0000CC2B329595E6241FB14F0A0011241FBE4B
:100D1000CFEFD1E4DEBFCDBF16E0A0E0B2E0EEEB56
:100D2000F0ED00E00BBF02C007900D92A831B107B3
:100D3000D9F718E2A8E1B6E001C01D92A63CB107C0
:100D4000E1F70E94755B0C945D680C940000E091E3
:100D5000E212F0E0EF71F070E15DFC4E8083809173
:100D6000E2128F5F8093E21280910020886080936E
:100D7000002046E554E0CA0161E10E94982B80E022
:100D800090E008956F927F928F929F92AF92BF9260
:100D9000CF92DF92EF92FF920F931F93CF93DF9347
:100DA0004B01809122069091230681FD74980E9448
:100DB000F0305C018CE296E00E94942C0AC0CE01D7
:100DC0000296B4010E946F290097E9F4CE010E94B7
:100DD0003A2DEC01009799F7CCC0CE010296B401F0
:100DE0000E946629D5018C918150888780E091E02E
:100DF000A0E0B0E089879A87AB87BC878CE296E059
:100E0000BE010E94032D84E00E9414329D838C83D6
:100E100083E00E9414323C019F838E83F501C080E1
:100E20008885C81ADD24EE24FF24A6E0CC0CDD1C46
:100E3000EE1CFF1CAA95D1F769857A858B859C8568
:100E400020EC30E040E050E00E945D61DC01CB012D
:100E5000892F9A2FAB2FBB27C80ED91EEA1EFB1E67
:100E6000C986DA86EB86FC86D5018C9188878091CD
:100E700022069091230681FD08C080918C0480FD9C
:100E800004C081FF6EC01D9B6CC0EDB7FEB77297AA
:100E90000FB6F894FEBF0FBEEDBF0DB71EB70F5FC4
:100EA0001F4F80E092E092838183C5010196D801B3
:100EB00013969C938E931297F401808114968C93D1
:100EC000149715961C921597818116968C931697F8
:100ED00017961C92D5018C91F801808711868C8120
:100EE0009D819387828775866486BB27AF2D9E2D53
:100EF0008D2D97878687C701B60124E630E040E054
:100F000050E00E945D61672F782F892F99270E94FA
:100F1000A361DC01CB01F801918B808B0E943365CA
:100F20002091A8048DB79EB742960FB6F8949EBF45
:100F30000FBE8DBF2223A9F000D000D0EDB7FEB7C1
:100F4000319687EA99E0ADB7BEB712969C938E931F
:100F50001197228313820E9445650F900F900F9086
:100F60000F90809122069091230681FF0BC0749A06
:100F700009C08DEB94E00E94212CEC01009709F050
:100F80002CCFEFCFDF91CF911F910F91FF90EF907A
:100F9000DF90CF90BF90AF909F908F907F906F9099
:100FA000089587EE93E08115910511F00197F1F70F
:100FB00008950F931F93CF93DF93C4EBDFE10CE30E
:100FC00012E088819981009739F12DB73EB72850FA
:100FD00030400FB6F8943EBF0FBE2DBFEDB7FEB741
:100FE0003196ADB7BEB712961C930E9311974A81F6
:100FF0005B816C817D814283538364837583978396
:1010000086830E9433652DB73EB7285F3F4F0FB6EA
:10101000F8943EBF0FBE2DBF26963FE1C03FD307D9
:1010200081F6DF91CF911F910F910895E4EBFFE1DD
:101030001182108236968FE1E03FF807C9F70895D4
:10104000CF93DF93C4EBDFE1E881F981309761F161
:10105000409118065091190660911A0670911B066E
:101060008091260690912706A0912806B091290626
:10107000841B950BA60BB70B4A815B816C817D812C
:10108000840F951FA61FB71F8A839B83AC83BD83E4
:10109000181619061A061B063CF0099519821882C3
:1010A0001A821B821C821D8226968FE1C03FD807C0
:1010B00059F68091180690911906A0911A06B091E0
:1010C0001B068093260690932706A0932806B093CC
:1010D0002906DF91CF910895CF93DF93EC018881AA
:1010E0009981009729F027E08A389207A9F40BC06C
:1010F00084E396E060E870E00E942C2E8AE897E096
:10110000998388830DC084E396E00E94572E009750
:1011100039F00E942008ECCF1982188283E001C0C8
:1011200081E0DF91CF910895DC01E4EBFFE180E005
:1011300090E0208131812115310591F4FC01EE0F01
:10114000FF1FE80FF91FEE0FFF1FEC54F04E428314
:10115000538364837583B183A08381E090E0089515
:10116000019636968A30910521F780E090E0089547
:1011700088EB98E040EA50E060E070E00E9494085C
:1011800088EB98E040EA50E060E070E00E9494084C
:101190000097B9F1809122069091230687FF31C014
:1011A000409118065091190660911A0670911B061D
:1011B0008DB79EB70A970FB6F8949EBF0FBE8DBF2E
:1011C000EDB7FEB731968EE592E0ADB7BEB7129699
:1011D0009C938E931197428353836483758380EA33
:1011E00090E0A0E0B0E086839783A087B1870E945B
:1011F00033658DB79EB70A960FB6F8949EBF0FBEA3
:101200008DBF0895882369F06D987598ED9A809147
:101210006A00886080936A00809168008160809392
:1012200068006E987698EE9A80916A00806280934A
:101230006A008091680081608093680008951F9221
:101240000F920FB60F9211248F939F93AF93BF937A
:101250008091680080FF29C08091B01F9091B11FDC
:1012600001969093B11F8093B01F8091A81B90911D
:10127000A91BA091AA1BB091AB1B0196A11DB11D8A
:101280008093A81B9093A91BA093AA1BB093AB1BA0
:10129000809122069091230690FF07C0749882E007
:1012A00090E09093B6048093B504BF91AF919F9165
:1012B0008F910F900FBE0F901F9018951F920F9255
:1012C0000FB60F9211248F939F93AF93BF9380918A
:1012D000680080FF29C08091B21F9091B31F0196D2
:1012E0009093B31F8093B21F8091AC1B9091AD1B64
:1012F000A091AE1BB091AF1B0196A11DB11D8093B3
:10130000AC1B9093AD1BA093AE1BB093AF1B809111
:1013100022069091230691FF07C0739882E090E027
:101320009093B6048093B504BF91AF919F918F9134
:101330000F900FBE0F901F90189580937C008091A6
:101340007B00877F80937B0080917C00806C809302
:101350007C0085E080937A0080917A008068809399
:101360007A0080917B0087FFFCCF80917B0085FF16
:10137000FCCF80917A00806480937A0080917A001B
:1013800086FDFCCF109279001092780084E090E006
:1013900060E070E020917A00206420937A00209130
:1013A0007A0026FDFCCF2091780030917900620F01
:1013B000731F019779F710927C0080917A008F77E4
:1013C00080937A00769567957695679580E090E0B2
:1013D0000E944860462F572F682F792FCB01BA0102
:1013E000089580E00E949D092091B1043091B204DB
:1013F0004091B3045091B4040E94FA6021EE3AE7A0
:1014000044E95EE30E94785F462F572F682F792FBB
:10141000CB01BA01089580E180935101809351017D
:101420009091510195FF03C08F5F8F31B9F76BE445
:10143000869FB0011124882777FD8095982F0E9400
:101440004A6020E030E64FE954E40E94785F462F7E
:10145000572F682F792FCB01BA0120E030E04AE7FF
:1014600054E40E94E05F462F572F682F792FCB015D
:10147000BA0108958091900483FF4DC080917B0054
:10148000886080937B0089EC80937C0085E080936A
:101490007A0080917A00806880937A0080917B0046
:1014A00087FFFCCF80917B0085FFFCCF80917A0085
:1014B000806480937A0080917A0086FDFCCF8091D1
:1014C0007A00806480937A0080917A0086FDFCCF58
:1014D000609178007091790080E090E00E9448600F
:1014E00027ED33EA40E95FE30E94FA6026E636E63C
:1014F00048E853E40E94775FDC01CB018093D61269
:101500009093D712A093D812B093D91280917A00F9
:101510008F7780937A000895CF92DF92EF92FF92B7
:101520001F93CF93DF93CDB7DEB729970FB6F8940B
:10153000DEBF0FBECDBF6C0110921C068FEF8983FA
:101540005BEEE52E52E1F52E10E03FC0183009F4B5
:1015500040C0CE010196BE016E5F7F4F0E94D7331F
:1015600089818F3F11F08E3F19F480931C0631C0A2
:10157000CE010296C114D10479F40E94F033809315
:10158000FD1FDE011296E5EFFFE188E09D9191934A
:101590008150E1F711E01DC00E94F033F701808314
:1015A000DE01129620E030E0C70108974D91FC0162
:1015B000E20FF31F40832F5F3F4F28303105B1F713
:1015C0001F5F89E090E0E80EF91E8981882309F009
:1015D000BDCF812F29960FB6F894DEBF0FBECDBFC9
:1015E000DF91CF911F91FF90EF90DF90CF90089502
:1015F00000D080E291E0EDB7FEB7928381830E9434
:1016000045650F900F9008952F923F924F925F92F1
:101610006F927F928F929F92AF92BF92CF92DF9202
:10162000EF92FF920F931F93CF93DF9300D000D0E0
:10163000CDB7DEB78C01009741F489E290E06BE210
:1016400070E04AE250E027E00AC08130910549F499
:1016500089E290E06BE270E04AE250E026E00E940E
:10166000AC32C8010E948C0A3DE1832E36E0932EF5
:10167000800E911ED4018C930115110599F01BEE7B
:10168000A12E12E1B12E00E010E08BE3682E81E084
:10169000782E90E4492E91E0592E28E4222E21E064
:1016A000322E10C185EF9FE10E941335FC01BF016E
:1016B000882777FD8095982F0E944A60F82EE92EA2
:1016C00005EF1FE1AA24BB24B2E2CB2EB1E0DB2E52
:1016D000D8018D918D0100D000D0EDB7FEB73196C5
:1016E000ADB7BEB71296DC92CE9211978283138269
:1016F0006B837C830E9445650894A11CB11C0F90EC
:101700000F900F900F906B817C81B8E0AB16B10405
:10171000F9F600D000D000D00DB71EB70F5F1F4FF5
:1017200087E291E0EDB7FEB7928381839701862F20
:10173000972FA32FBE2DBC01CD0120E030E048EC57
:1017400052E40E94E05FDC01CB01F80182839383C5
:10175000A483B5830E9445652DB73EB72A5F3F4FEE
:101760000FB6F8943EBF0FBE2DBF8091FD1F88239A
:1017700019F081E892E002C08AE892E000D000D03F
:1017800027E331E0ADB7BEB712963C932E93119785
:1017900014969C938E9313970E9445650F900F901B
:1017A0000F900F900E94F80A94C0C80163E0880F60
:1017B000991F6A95E1F7800F911F8D519D4E0E94F0
:1017C0001335FC01BF01882777FD8095982F0E9473
:1017D0004A606C0120E030E0A8EFEA2EAFEFFA2E6D
:1017E000EA0CFB1C00D000D0ADB7BEB71196EDB728
:1017F000FEB772826182F701E20FF31F80811296B9
:101800008C93129713961C9229833A836B837C8363
:101810000E94456529813A812F5F3F4F0F900F90BD
:101820000F900F906B817C8128303105D9F600D064
:1018300000D000D0EDB6FEB60894E11CF11CADB7A7
:10184000BEB712965C924E921197862F972FAC2DB1
:10185000BD2DBC01CD0120E030E048EC52E40E94F7
:10186000E05FDC01CB01F70182839383A483B5831E
:101870000E9445652DB73EB72A5F3F4F0FB6F894DB
:101880003EBF0FBE2DBFD5018C91882319F081E892
:1018900092E002C08AE892E000D000D0EDB7FEB737
:1018A00032822182948383830E9445650F900F903A
:1018B0000F900F900E94F80A0F5F1F4F29E030E051
:1018C000A20EB31ED4018C9190E0081719070CF4F6
:1018D0006CCF0F900F900F900F90DF91CF911F91D1
:1018E0000F91FF90EF90DF90CF90BF90AF909F90BF
:1018F0008F907F906F905F904F903F902F900895C2
:10190000CF93DF9300D0CDB7DEB78091F61F8983E8
:101910008091FC1F8A83CE0101960E9481290F903D
:101920000F90DF91CF910895CF93DF93EC018091D9
:10193000F51F8F3FB1F58091F61F8F3F91F5809194
:10194000F71F8F3F71F58091F81F8F3F51F5809100
:10195000F91F8F3F31F58091FA1F8F3F11F580916C
:10196000FB1F8F3FF1F48091FC1F8F3FD1F489E280
:1019700090E06BE270E04AE250E027E00E94AC3277
:1019800080E090E00E948C0AC35ED94F888385EF87
:101990009FE160E070E049E050E00E948B660E94A9
:1019A000800CDF91CF9108951F920F920FB60F9286
:1019B0000BB60F9211242F933F934F935F936F9326
:1019C0007F938F939F93AF93BF93EF93FF938091F8
:1019D00000208260809300208091B5049091B6042D
:1019E0001816190614F4749A739A8091220690912D
:1019F000230685FF02C07498739880911806909111
:101A00001906A0911A06B0911B060196A11DB11DE1
:101A10008093180690931906A0931A06B0931B069C
:101A20008091B7049091B80401979093B804809383
:101A3000B704009709F064C080912A0690912B06A4
:101A40009C012F5F3F4F30932B0620932A06409135
:101A5000531B5091541B6091551B7091561B4F5F47
:101A60005F4F6F4F7F4F4093531B5093541B6093B6
:101A7000551B7093561B20E130E03093B80420933F
:101A8000B70420918C0420FD02C01D9B05C010925C
:101A9000200610921F0606C021E030E03093200699
:101AA00020931F0620918E0430918F04211531055B
:101AB000A1F00296B9010E947C61009771F47798B9
:101AC000809122069091230693FF07C0749884E0CA
:101AD00090E09093B6048093B5042115310581F010
:101AE00080912A0690912B06B9010E947C61009793
:101AF00039F48EE394E062E140E050E00E94982BDC
:101B0000FF91EF91BF91AF919F918F917F916F91D5
:101B10005F914F913F912F910F900BBE0F900FBE91
:101B20000F901F9018958091E2129091671B891B6E
:101B300008950E94930D882379F0E091671BF0E0EF
:101B4000EF71F070E15DFC4E808190E02091671BA9
:101B50002F5F2093671B08958FEF9FEF0895CF931A
:101B6000DF93EC011092250610922406888199815A
:101B7000009731F022E08C3D920709F0B7C009C010
:101B80000E94930D882341F48CED92E09983888321
:101B9000B1C0613109F0AEC0F89478940E94990DFB
:101BA00090E090933D0680933C068D3009F47CC014
:101BB0008F3F31F38231910569F18F37910521F023
:101BC0008830910509F053C080913E0690913F0600
:101BD000181619060CF060C06091C0287091C128D9
:101BE00088E090E00E9407656091C0287091C1284C
:101BF00080E290E00E9407656091C0287091C12842
:101C000088E090E00E94076580913E0690913F0633
:101C100001973EC06091C0287091C1288DE090E08E
:101C20000E940765109241061092400614C0885920
:101C3000944EFC0180816091C0287091C12890E091
:101C40000E9407658091400690914106019690930D
:101C50004106809340068091400690914106209174
:101C60003E0630913F06821793070CF315C0609132
:101C7000C0287091C1280E94076580913E0690910E
:101C80003F0620913C06FC01E859F44E2083019662
:101C900090933F0680933E0680913E0690913F06CA
:101CA0008F33910509F06CCF1092671B1092E212EE
:101CB00080913E0690913F06FC01E859F44E108257
:101CC000909325068093240610923F0610923E06BC
:101CD0008091FE1F9091FF1F009709F451CF6091F2
:101CE000320640E050E00E94982B4ACF19821882B9
:101CF00083E001C081E0DF91CF91089578948091D5
:101D00001F0690912006009719F483B7817F03C0C6
:101D100083B7817F866083BFF89483B7816083BF78
:101D20007894889583B78E7F83BF78940895CF93F6
:101D3000DF93EC0188819981009721F027E08739B2
:101D4000920789F40E947E0E8091D0099091D1096A
:101D500065E840E050E00E94982B87E997E099837E
:101D6000888381E003C01982188283E0DF91CF91DC
:101D70000895FF920F931F93CF93DF93729A8091F0
:101D80008C0483FD06C0C0E5D0E00E94D1072197F6
:101D9000E1F78EE40E949135882309F08BC0C0E5FD
:101DA000D0E00E94D1072197E1F78FE40E9491359E
:101DB0000E94F935C82F829586958695837081306B
:101DC000A9F440915B1B50915C1B60915D1B70916D
:101DD0005E1B4F5F5F4F6F4F7F4F40935B1B509376
:101DE0005C1B60935D1B70935E1B16C08230A0F07D
:101DF00040915F1B5091601B6091611B7091621B51
:101E00004F5F5F4F6F4F7F4F40935F1B5093601B3F
:101E10006093611B7093621B0E94F9351C2F1F7326
:101E200000E0080F111D0E94F935F82E0E940336BC
:101E3000DF2D90E0C92FC80FD11DD695C795D69537
:101E4000C7950E94E03580918C0483FF7298B80199
:101E500080E090E00E94486020E134E048EC5BE3E1
:101E60000E94FA60DC01CB0180934F1390935013D2
:101E7000A0935113B0935213BE0180E090E00E94F2
:101E8000486024EA3CEF44E25CE30E94FA6020E010
:101E900030E040E252E40E94775FDC01CB018093A6
:101EA000012090930220A0930320B093042080E0AF
:101EB00090E015C08091571B9091581BA091591B21
:101EC000B0915A1B0196A11DB11D8093571B909391
:101ED000581BA093591BB0935A1B81E090E0DF91EF
:101EE000CF911F910F91FF9008950E943A0A80911F
:101EF00090049091910492FF02C00E94B90E8091CB
:101F000090049091910493FF0CC00E94F109DC01B0
:101F1000CB018093F01F9093F11FA093F21FB09319
:101F2000F31F08957298729A8EE40E94913580EAA8
:101F30000E94E83580E00E94E83580E00E94E835A4
:101F40008FE40E9491350E94F93582958695869599
:101F500083708130A9F440915B1B50915C1B6091B0
:101F60005D1B70915E1B4F5F5F4F6F4F7F4F4093C4
:101F70005B1B50935C1B60935D1B70935E1B16C0D4
:101F80008230A0F040915F1B5091601B6091611BFB
:101F90007091621B4F5F5F4F6F4F7F4F40935F1B8E
:101FA0005093601B6093611B7093621B00D000D044
:101FB000EDB7FEB731962BE832E0ADB7BEB712965B
:101FC0003C932E931197828313820E9433650F9066
:101FD0000F900F900F908EE40E94913580E80E9440
:101FE000E83580E00E94E83580E00E94E8350E94F4
:101FF000E03580E090E0089500D08CE491E0ADB74A
:10200000BEB712969C938E9311970E9445652091BE
:10201000A8040F900F902223A9F000D000D0EDB7B4
:10202000FEB7319689E591E0ADB7BEB712969C93A5
:102030008E931197228313820E9445650F900F9013
:102040000F900F90089500D08CE591E0EDB7FEB7AA
:10205000928381830E94456581E891E0EDB7FEB7E8
:10206000928381830E94456589EA91E0EDB7FEB7CE
:10207000928381830E94456580ED91E0EDB7FEB7C4
:10208000928381830E9445658AEF91E0EDB7FEB7A8
:10209000928381830E94456585E392E0EDB7FEB7A8
:1020A000928381830E9445658FE592E0EDB7FEB78C
:1020B000928381830E94456585E892E0EDB7FEB783
:1020C000928381830E94456585EB92E0EDB7FEB770
:1020D000928381830E9445658EEE92E0EDB7FEB754
:1020E000928381830E9445658AE193E0EDB7FEB754
:1020F000928381830E94456583E493E0EDB7FEB748
:10210000928381830E94456582E793E0EDB7FEB735
:10211000928381830E94456584EA93E0EDB7FEB720
:10212000928381830E94456585ED93E0EDB7FEB70C
:10213000928381830E94456589E094E0EDB7FEB704
:10214000928381830E94456589E394E0EDB7FEB7F1
:10215000928381830E94456585E694E0EDB7FEB7E2
:10216000928381830E94456584E994E0EDB7FEB7D0
:10217000928381830E9445658DEB94E0EDB7FEB7B5
:10218000928381830E9445658CEE94E0EDB7FEB7A3
:10219000928381830E94456583E195E0EDB7FEB7A8
:1021A000928381830E9445650F900F9008958BE97B
:1021B00092E00E946C6508954F925F926F927F92B9
:1021C0008F929F92AF92BF92CF92DF92EF92FF9247
:1021D0000F931F93CF93DF9300D000D0CDB7DEB71E
:1021E0006091531B7091541B8091551B9091561B0D
:1021F0008090531B9090541BA090551BB090561B81
:102200004090531B5090541B6090551B7090561B70
:102210002091531B3091541B4091551B5091561BDC
:1022200029833A834B835C834DB75EB74A50504055
:102230000FB6F8945EBF0FBE4DBF0DB71EB70F5F50
:102240001F4F29E435E0EDB7FEB732832183A0E8C4
:10225000CA2EA1E5DA2EA1E0EA2EF12CA701960103
:102260000E94A361F80133832283C501B401A70151
:1022700096010E94A361B0E1CB2EBEE0DB2EE12CE3
:10228000F12CA70196010E94A361332727FD309509
:10229000F80135832483C301B201A70196010E948E
:1022A000A3612CE3C22ED12CE12CF12CA7019601C5
:1022B0000E94A361332727FD3095F80137832683D9
:1022C00069817A818B819C81A70196010E94A3611B
:1022D000772767FD7095F801718760870E944565D3
:1022E0002DB73EB7265F3F4F0FB6F8943EBF0FBEE7
:1022F0002DBF0F900F900F900F90DF91CF911F91F6
:102300000F91FF90EF90DF90CF90BF90AF909F9094
:102310008F907F906F905F904F900895E6ECF8E279
:102320008081918122E482349207B9F000D000D0FC
:1023300089E695E0ADB7BEB712969C938E93119740
:10234000E65CF8421496FC93EE9313970E94456561
:102350000F900F900F900F9008953A96B1E4E53FDB
:10236000FB07F0F20895EF92FF920F931F93CF9324
:10237000DF930E94F109DC01CB0100D000D000D036
:1023800027E835E0EDB7FEB732832183838394835A
:10239000A583B6830E9445658DB79EB706960FB696
:1023A000F8949EBF0FBE8DBF81E00E949D092091D1
:1023B000AD043091AE044091AF045091B0040E943E
:1023C000FA608B01D82FC92F82E00E949D09AB01D2
:1023D000BC01EDB7FEB73A970FB6F894FEBF0FBE3B
:1023E000EDBFEDB6FEB60894E11CF11C2EE835E019
:1023F000328321839E01802F912FA32FB22FF701CB
:1024000082839383A483B583CB01BA012091A9046D
:102410003091AA044091AB045091AC040E94FA6040
:10242000DC01CB01F70186839783A087B1870E94E7
:1024300045658DB79EB70A960FB6F8949EBF0FBE3E
:102440008DBF0E94F80ADF91CF911F910F91FF90ED
:10245000EF900895EF92FF920F931F93CF93DF9326
:10246000882389F085EF9FE16FEF70E049E050E04D
:102470000E94BD6485EF9FE160E070E049E050E0BC
:102480000E948B6622C005EF1FE1C0E0D0E03AE970
:10249000E32E35E0F32ED8018D918D0100D000D0D0
:1024A000EDB7FEB73196ADB7BEB71296FC92EE927D
:1024B0001197828313820E94456521960F900F9099
:1024C0000F900F90C830D10531F70E94F80ADF91C4
:1024D000CF911F910F91FF90EF900895CF92DF92CF
:1024E000EF92FF926091A6047091A70480E090E0C3
:1024F0000E94AF646CEB72E00E94C464009709F024
:1025000077C083E19AE0909391048093900480E9EE
:1025100094E06DE070E042E050E00E948B668CE356
:1025200090E090938F0480938E048EE894E06BE0AB
:1025300070E042E050E00E948B6682E090E0909371
:102540008D0480938C048CE894E069E070E042E0B4
:1025500050E00E948B66109223061092220682E2BF
:1025600096E06BE170E042E050E00E948B660F2E37
:10257000F2E2CF2EFFEFDF2EFCECEF2EFBE3FF2E7F
:10258000F02DC092AD04D092AE04E092AF04F09270
:10259000B0048DEA94E063E170E044E050E00E9412
:1025A0008B66C092A904D092AA04E092AB04F09288
:1025B000AC0489EA94E06FE070E044E050E00E94EF
:1025C0008B668DEE97E4AAE8BCE38093B104909308
:1025D000B204A093B304B093B40481EB94E067E138
:1025E00070E044E050E00E948B6681E00E942A1275
:1025F000FF90EF90DF90CF9008952F923F924F92EF
:102600005F926F927F928F929F92AF92BF92CF9282
:10261000DF92EF92FF920F931F93CF93DF9300D03F
:10262000CDB7DEB79A838983DC018D919C91119798
:10263000009711F00C945B216091A6047091A7049F
:1026400088E69BE10E94AF6488E69BE160E470E06D
:102650000E94CD64009759F46091C0287091C12800
:102660008AE090E00E94076581E00C94612181304E
:10267000910549F42090681B332444245524662492
:1026800077244301BEC18230910599F43091681BD3
:102690002091691B932F80E0820F911D1C01892FCF
:1026A000880F880B482E582E682E782E882E982E4C
:1026B000A8C18330910509F09CC02091681B8090CF
:1026C000691BB0906A1B30E040E050E060E070E0D1
:1026D00080E090E000E10E94B85A922EA32E142FC1
:1026E000F52EE62EC72E282ED92E282D30E040E0DC
:1026F00050E060E070E080E090E008E00E94B85AAE
:10270000290DB1E0291508F0B0E03A0DE1E03A15E5
:1027100008F0E0E0B30FF1E0B31708F0F0E0EF2BC2
:10272000410F31E0411708F030E0E40FF1E0E41729
:1027300008F0F0E03F2B5F0D41E05F1508F040E04E
:10274000A32FA50F31E0A51708F030E0432B6E0D45
:1027500031E06E1508F030E0F42FF60F41E0F61787
:1027600008F040E0342B7C0D41E07C1508F040E09F
:10277000532F570F31E0571708F030E0432B820DED
:1027800031E0821508F030E0480F61E0481708F0AA
:1027900060E0362BD90ED30EB20E81E0B21608F0EF
:1027A00080E0182F1B0F71E01B1708F070E07E0F00
:1027B00061E07E1708F060E06A0F31E06A1708F008
:1027C00030E03F0F21E03F1708F020E0250F91E0B7
:1027D000251708F090E0940F81E0941708F080E04E
:1027E0002B2C312E472E562E632E722E892E982E8C
:1027F000FDC08430910509F0FBC02091681B8090DA
:10280000691BA0906A1BB0906B1B30E040E050E069
:1028100060E070E080E090E008E10E94B85A722E1B
:10282000932E142FF52EE62EC72E282ED92E282DC6
:1028300030E040E050E060E070E080E090E000E1F7
:102840000E94B85A270DF1E0271508F0F0E0390D85
:10285000E1E0391508F0E0E0F30FA1E0F31708F02C
:10286000A0E0EA2B410F31E0411708F030E0E40F1F
:10287000A1E0E41708F0A0E03A2B5F0D41E05F15FE
:1028800008F040E0B32FB50F31E0B51708F030E0A5
:10289000432B6E0D31E06E1508F030E0A42FA60F2B
:1028A00041E0A61708F040E0342B7C0D41E07C1598
:1028B00008F040E0532F570F31E0571708F030E091
:1028C000432B820D31E0821508F030E0480F61E0C3
:1028D000481708F060E0362BD90ED30E222E2B0CB1
:1028E00081E0221608F080E0B82EBF0E81E0BF160E
:1028F00008F080E0982E9E0E81E09E1608F080E0A1
:10290000C82ECB0E11E0CB1608F010E01A0F81E0B4
:102910001A1708F080E0F82EF50E81E0F51608F0A1
:1029200080E0E82EE40E81E0E41608F080E0D80EA6
:102930002A2D30E040E050E060E070E080E090E080
:1029400008E00E94B85A220DE1E0221508F0E0E00C
:102950003B0DF1E03B1508F0F0E0E30FA1E0E317D9
:1029600008F0A0E0FA2B490D31E0491508F030E0FD
:10297000F40FA1E0F41708F0A0E03A2B5C0D41E061
:102980005C1508F040E0A32FA50F31E0A51708F073
:1029900030E0432B610F31E0611708F030E0542F35
:1029A000560F41E0561708F040E0342B7F0D41E010
:1029B0007F1508F040E0632F670F31E0671708F0DC
:1029C00030E0432B8E0D31E08E1508F030E0480FDB
:1029D00071E0481708F070E0372BD90E222E3E2EFA
:1029E0004F2E5A2E652E762E842E932E9D0C09C0C6
:1029F0008AE0282E3324442455246624772488240E
:102A000099240E94F80AB2E62B1689F4E5E63E16F0
:102A100071F4F4E64F1659F4552049F4662039F460
:102A2000772029F4882019F4992009F40DC5910123
:102A3000A201B301C401B2E6AB2E15E6B12E04E645
:102A4000C02EDD24EE24FF2400E010E00E94325B63
:102A5000823008F099C187E7281681F49FE639167D
:102A600069F4442059F4552049F4662039F477205C
:102A700029F4882019F4992009F4D3C79101A201FF
:102A8000B301C401F7E7AF2EAFE6BA2ECC24DD24A4
:102A9000EE24FF2400E010E00E94325B823008F058
:102AA000B6C0A4E62A1689F4B1E63B1671F44420B8
:102AB00061F4552051F4662041F4772031F48820E8
:102AC00021F4992011F40C94C0209101A201B301CA
:102AD000C40104E6A02EE1E6BE2ECC24DD24EE24C3
:102AE000FF2400E010E00E94325B823008F046C014
:102AF000E5E72E1679F4332069F4442059F4552083
:102B000049F4662039F4772029F4882019F49920B3
:102B100009F4BAC5F6E72F1679F4332069F4442096
:102B200059F4552049F4662039F4772029F4882097
:102B300019F4992009F4B7C588E6281611F00C9409
:102B40005921332011F00C945921442011F00C9498
:102B50005921552011F00C945921662011F00C9444
:102B60005921772011F00C945921882011F00C94F0
:102B70005921992011F00C94592163C594E6291626
:102B800081F4A9E63A1669F4442059F4552049F431
:102B9000662039F4772029F4882019F4992009F463
:102BA00053C5B5E62B1681F4EEE63E1669F44420D3
:102BB00059F4552049F4662039F4772029F4882007
:102BC00019F4992009F487C7F5E62F1611F00C9433
:102BD000592184E6381611F00C945921442011F043
:102BE0000C945921552011F00C945921662011F0B4
:102BF0000C945921772011F00C945921882011F060
:102C00000C945921992011F00C9459211DC493E77B
:102C1000291689F4A2E73A1671F4442061F455208C
:102C200051F4662041F4772031F4882021F4992072
:102C300011F40C944C1F9101A201B301C401B3E73C
:102C4000AB2E12E7B12ECC24DD24EE24FF2400E0CD
:102C500010E00E94325B823008F04AC0B5E62B16C5
:102C600079F43B1469F4442059F4552049F4662062
:102C700039F4772029F4882019F4992009F494C7AD
:102C8000E9E62E1689F4F2E73F1671F4442061F468
:102C9000552051F4662041F4772031F4882021F446
:102CA000992011F40C94F31E83E3281611F00C9470
:102CB000592191E7391611F00C945921442011F053
:102CC0000C945921552011F00C945921662011F0D3
:102CD0000C945921772011F00C945921882011F07F
:102CE0000C945921992011F00C9459210C94C02076
:102CF000A3E62A1691F4B4E63B1679F4E1E64E1603
:102D000061F4552051F4662041F4772031F4882095
:102D100021F4992011F40C94C020F3E72F1689F4C4
:102D200085E6381671F491E6491659F4552049F4B0
:102D3000662039F4772029F4882019F4992009F4C1
:102D4000C1C4A3E72A1611F00C9459213A1611F0C8
:102D50000C945921442011F00C945921552011F064
:102D60000C945921662011F00C945921772011F010
:102D70000C945921882011F00C945921992011F0BC
:102D80000C9459210C945B1FB4E72B1689F4EFE6E1
:102D90003E1671F44E1661F4F2E65F1649F46620B1
:102DA00039F4772029F4882019F4992009F4C6C44D
:102DB0009101A201B301C40104E7A02EEFE6BE2EEB
:102DC000FFE6CF2EA2E6DA2EEE24FF2400E010E08C
:102DD0000E94325B823008F0A8C085E7281689F48B
:102DE00093E6391671F4ADE64A1659F4552049F4C4
:102DF000662039F4772029F4882019F4992009F401
:102E000091C59101A201B301C401A5E7AA2EB3E6C1
:102E1000BB2E1DE6C12EDD24EE24FF2400E010E0D1
:102E20000E94325B8230B0F52C1489F43A1479F4A4
:102E3000B8E64B1661F4552051F4662041F4772032
:102E400031F4882021F4992011F40C94CF20E7E686
:102E50002E1689F4FFE63F1671F48CE6481659F4F5
:102E6000552049F4662039F4772029F4882019F494
:102E7000992009F497C492E7291611F00C9459216E
:102E8000391611F00C945921A5E64A1611F00C944C
:102E9000592136C0B1E32B1681F43B1671F4E1E7FA
:102EA0004E1659F4552049F4662039F4772029F458
:102EB000882019F4992009F435C5F0E72F1689F414
:102EC00085E6381671F492E7491659F4552049F40D
:102ED000662039F4772029F4882019F4992009F420
:102EE00063C6A0E32A1611F00C945921B1E33B16F6
:102EF00011F00C945921E1E74E1611F00C94592170
:102F0000552011F00C945921662011F00C94592190
:102F1000772011F00C945921882011F00C9459213C
:102F2000992011F00C9459219AC4F0E72F1691F4CE
:102F30008DE6381679F495E7491661F4A8E65A1635
:102F400049F4662039F4772029F4882019F499206F
:102F500009F48DC59101A201B301C40110E7A12EAE
:102F60000DE6B02EE5E7CE2EF8E6DF2EEE24FF24A8
:102F700000E010E00E94325B823008F04DC02A145D
:102F800089F4BCE63B1671F4E5E64E1659F45D147F
:102F900049F4662039F4772029F4882019F499201F
:102FA00009F44FC3F1E62F1691F48DE6381679F443
:102FB00095E7491661F4A8E65A1649F4662039F4F3
:102FC000772029F4882019F4992009F43FC5B9E63F
:102FD0002B1611F00C945921ECE63E1611F00C94CE
:102FE0005921F1E64F1611F00C94592183E6581639
:102FF00011F00C945921662011F00C94592177207E
:1030000011F00C945921882011F00C945921992029
:1030100011F00C945921B0C094E7291691F4A3E75C
:103020003A1679F4B5E64B1661F4E2E75E1649F418
:10303000662039F4772029F4882019F4992009F4BE
:10304000B0C59101A201B301C401E4E7AE2EF3E7DC
:10305000BF2EA5E6CA2EB2E7DB2EEE24FF2400E049
:1030600010E00E94325B823020F5F1E32F1611F060
:103070000C9459213D1411F00C94592187E74816FE
:1030800011F00C94592190E7591611F00C94592124
:10309000662011F00C945921772011F00C945921DD
:1030A000882011F00C945921992011F00C94592189
:1030B0003BC0A2E72A1691F4B7E63B1679F4E0E7A5
:1030C0004E1661F4F5E75F1649F4662039F477206F
:1030D00029F4882019F4992009F433C38CE62816C2
:1030E00011F00C94592191E6391611F00C945921E4
:1030F000A4E74A1611F00C945921B8E75B1611F0B9
:103100000C945921662011F00C945921772011F06C
:103110000C945921882011F00C945921992011F018
:103120000C9459210C941F216091A6047091A7045E
:1031300080E090E00E94AF648C0163EC72E00E943A
:10314000C464009719F477980C945B21C80166EC6D
:1031500072E00E94C464009719F4779A0C945B2182
:10316000779903C083EC92E002C086EC92E000D035
:1031700000D02FE935E0AAC46091A6047091A7049D
:1031800080E090E00E94AF648C016DEC72E00E94E0
:10319000C464009709F043C06091A6047091A7042D
:1031A00080E090E00E94AF648C01009711F40C94D1
:1031B0005B2160ED72E00E94C464009729F482E212
:1031C0009FEFACECBBE318C0C8010E94A2636B0187
:1031D0007C0120E030E040E050E00E94DC5F88238A
:1031E000D1F081E00E949D099B01AC01C701B601AD
:1031F0000E94E05FDC01CB018093AD049093AE04AC
:10320000A093AF04B093B0048DEA94E063E170E062
:1032100044E050E075C200D08AE599E09DC0C80145
:1032200066ED72E00E94C464009709F045C06091A9
:10323000A6047091A70480E090E00E94AF648C0126
:10324000009711F40C945B2160ED72E00E94C4645D
:10325000009729F482E29FEFACECBBE318C0C801F1
:103260000E94A2636B017C0120E030E040E050E06E
:103270000E94DC5F8823C1F082E00E949D099B01CF
:10328000AC01C701B6010E94E05FDC01CB01809375
:10329000A9049093AA04A093AB04B093AC0489EA68
:1032A00094E06FE070E0B4CF00D087E699E0EDB72E
:1032B000FEB79283818356C0C80169ED72E00E9417
:1032C000C464009709F053C06091A6047091A704EC
:1032D00080E090E00E94AF648C01009711F40C94A0
:1032E0005B2160ED72E00E94C464009729F48DEECA
:1032F00097E4AAE8BCE320C0C8010E94A2636B0166
:103300007C0120E030E040E050E00E94DC5F882358
:1033100001F180E00E949D094B015C01C701B601EB
:1033200021EE3AE744E95EE30E94775FA50194014C
:103330000E94E05FDC01CB018093B1049093B20462
:10334000A093B304B093B40481EB94E067E170E020
:103350005FCF00D084E799E0ADB7BEB712969C93DB
:103360008E9311970E9445650F900F90A4C70E94FD
:10337000F109AB01BC0100D000D000D081E899E098
:10338000EDB7FEB79283818343835483658376834D
:103390000E944565EDB7FEB736960FB6F894FEBFAE
:1033A0000FBEEDBF81E00E949D092091AD043091D8
:1033B000AE044091AF045091B0040E94FA606B01DA
:1033C000182F092F82E00E949D09AB01BC018DB727
:1033D0009EB70A970FB6F8949EBF0FBE8DBFEDB68D
:1033E000FEB60894E11CF11C88E899E0ADB7BEB7C1
:1033F00012969C938E93119798018C2D9D2DA32F3F
:10340000B22FF70182839383A483B583CB01BA01E2
:103410002091A9043091AA044091AB045091AC04CE
:103420000E94FA60DC01CB01F70186839783A087B5
:10343000B1870E9445658DB79EB70A960FB6F8947E
:103440009EBF0FBE8DBF32C76091A6047091A704C6
:1034500080E090E00E94AF64009771F160E070E05E
:1034600040E150E00E946162AB01BC018091220604
:10347000909123068417950799F150932306409362
:10348000220682E296E06BE170E042E050E00E94AA
:103490008B66809122069091230600D000D023EA0B
:1034A00035E0ADB7BEB712963C932E9311971496A4
:1034B0009C938E9313970EC08091220690912306C1
:1034C00000D000D023EB35E0EDB7FEB73283218387
:1034D000948383830E9445650F900F900F900F9007
:1034E0000E94F80A00D000D087EC95E0ADB7BEB7D7
:1034F00012969C938E93119781E090E014969C9382
:103500008E9313970E94456584ED95E0EDB7FEB765
:103510009283818382E090E0948383830E94456557
:103520008FED95E0ADB7BEB712969C938E93119731
:1035300084E090E014969C938E9313970E944565C7
:103540008AEE95E0EDB7FEB79283818388E090E044
:10355000948383830E94456587EF95E0ADB7BEB73E
:1035600012969C938E93119780E190E014969C9311
:103570008E9313970E94456582E096E0EDB7FEB703
:103580009283818380E290E0948383830E944565E7
:103590008EE096E0ADB7BEB712969C938E931197CE
:1035A00080E490E014969C938E9313970E94456557
:1035B0008CE196E0EDB7FEB79283818380E890E0DE
:1035C000948383830E9445658AE296E0ADB7BEB7D7
:1035D00012969C938E93119780E091E014969C93A1
:1035E0008E9313970E94456589E396E0EDB7FEB789
:1035F0009283818380E092E0948383830E94456577
:1036000088E496E0ADB7BEB712969C938E9311975F
:1036100080E094E014969C938E9313970E944565E6
:1036200084E596E0EDB7FEB79283818380E098E071
:10363000948383830E9445650F900F900F900F90A5
:103640003AC60E94231037C66091A6047091A70461
:1036500080E090E00E94AF6460ED72E00E94C4647C
:10366000009711F481E001C080E00E942A122091AD
:10367000A804222309F41FC600D000D0EDB7FEB77E
:10368000319682E696E0D2C50E94DC102091A80413
:10369000222309F410C600D000D0EDB7FEB7319652
:1036A00085E696E0C3C50E94D7102091A804222386
:1036B00009F401C600D000D0EDB7FEB7319688E618
:1036C00096E0B4C56091A6047091A70480E090E0F4
:1036D0000E94AF648C0163EC72E00E94C4640097A6
:1036E00091F480918C0490918D04846090938D046A
:1036F00080938C048CE894E069E070E042E050E054
:103700000E948B66D8C5C80166EC72E00E94C46452
:103710009C0180918C0490918D042115310511F448
:103720008B7FE4CF82FF03C083EC92E002C086EC83
:1037300092E000D000D024E939E0C8C10C94000028
:10374000BAC500D08BE696E0ADB7BEB712969C9393
:103750008E9311970E9445652091A8040F900F90B9
:103760002223A9F000D000D0EDB7FEB731968FE646
:1037700096E0ADB7BEB712969C938E9311972283B5
:1037800013820E9445650F900F900F900F9088E173
:103790000FB6F89480936000109260000FBE0C94F6
:1037A000007C89C56091A6047091A70480E090E038
:1037B0000E94AF647C0163EC72E00E94C4640097D5
:1037C00049F40E94D33B80918C0490918D048160D8
:1037D0008D7F8CCFC70166EC72E00E94C4640097B5
:1037E00041F40E94C43C80918C0490918D048C7FA4
:1037F0007DCF0EED12E0C701B8010E94C4640097AE
:1038000049F40E94C43C80918C0490918D048E7F79
:1038100082606CCF80918C0481FF0BC000D000D0FF
:1038200088E999E0EDB7FEB792838183148303831F
:1038300001CF80FF03C083EC92E002C086EC92E0EF
:1038400000D000D02CE939E0ADB7BEB712963C935A
:103850002E93119714969C938E931397EBCE00D0D2
:1038600082E796E0EDB7FEB7928381830E944565BB
:103870008DB79EB740970FB6F8949EBF0FBE8DBF11
:10388000EDB7FEB731968CE996E0ADB7BEB71296AC
:103890009C938E9311978091631B9091641BA091D0
:1038A000651BB091661B82839383A483B58380914B
:1038B000571B9091581BA091591BB0915A1B86839E
:1038C0009783A087B18780915B1B90915C1BA0912F
:1038D0005D1BB0915E1B82879387A487B58780911B
:1038E0005F1B9091601BA091611BB091621B86874A
:1038F0009787A08BB18B0E9445652091A804EDB7F6
:10390000FEB772960FB6F894FEBF0FBEEDBF22232E
:1039100009F4D1C400D000D0EDB7FEB731968AEBE0
:1039200096E084C4F89409E081E090E0FC01009303
:103930005700C895F02C20E030E0F90100935700C3
:10394000C895E02C7894F89423E030E0F9010093D6
:103950005700C895102D82E090E0FC0100935700BD
:10396000C895002D789400D000D000D02DEB36E023
:10397000EDB7FEB73283218380912B1390912C13E6
:10398000A0912D13B0912E1383839483A583B683C6
:103990000E94456500D000D0EDB7FEB7319687ECA8
:1039A00096E0ADB7BEB712969C938E9311970283A3
:1039B000138214831582E6821782F08611860E9494
:1039C0004565EDB7FEB73A960FB6F894FEBF0FBE49
:1039D000EDBF0E948E112091660000D000D0EDB79F
:1039E000FEB731968EEE96E0ADB7BEB712969C93B9
:1039F0008E931197228313820E9445650F900F903A
:103A00000F900F900E94F80A2091A804222309F435
:103A100052C400D000D0EDB7FEB731968AEF96E0E1
:103A200005C480E090E00E94040B81E090E00E94D9
:103A3000040B2091A804222309F43DC400D000D037
:103A4000EDB7FEB731968DEF96E0F0C30E94920F6E
:103A50000E94F80A2091A804222309F42CC400D063
:103A600000D0EDB7FEB7319680E097E0DFC36091FC
:103A7000A6047091A70480E090E00E94AF648C01DE
:103A800063EC72E00E94C464009731F480918C046E
:103A900090918D0488602ACEC80166EC72E00E9485
:103AA000C4649C0180918C0490918D042115310592
:103AB00011F4877F1BCE83FF03C083EC92E002C02A
:103AC00086EC92E000D000D020EA39E0EDB7FEB7F6
:103AD00032832183ADCD6091A6047091A70480E06C
:103AE00090E00E94AF6463EE72E00E94C4640097AD
:103AF00029F410922D0610922C0646C08CE296E016
:103B00000E94942C7C0109EE12E03BC08DB79EB759
:103B10000C970FB6F8949EBF0FBE8DBFEDB7FEB7E2
:103B20003196ADB7BEB712961C930E931197D7017D
:103B300012968C9112978283138213968C9113970D
:103B40008483158218968C91189786831782149611
:103B50008D919C9115979187808716968D919C9158
:103B60001797938782870E943365EDB7FEB73C961F
:103B70000FB6F894FEBF0FBEEDBFC7010E943A2DED
:103B80007C01E114F10411F62091A804222309F428
:103B900092C300D000D0EDB7FEB7319683E097E036
:103BA00045C30E946E1287C36091A6047091A7045A
:103BB00080E090E00E94AF64009731F160E070E037
:103BC00040E150E00E946162DC01CB0190939104DE
:103BD0008093900400D000D04DB75EB74F5F5F4F29
:103BE00026E037E0EDB7FEB732832183FA019383F5
:103BF00082830E9445650F900F900F900F9080E98F
:103C000094E06DE070E07ACD00D000D087E197E0DD
:103C1000ADB7BEB712969C938E9311978091900486
:103C20009091910414969C938E9313970E944565EE
:103C30000F900F900F900F900E94F80A00D000D0C4
:103C40008AE297E0EDB7FEB79283818381E090E04E
:103C5000948383830E94456587E397E0ADB7BEB741
:103C600012969C938E93119782E090E014969C9309
:103C70008E9313970E94456583E497E0EDB7FEB7F6
:103C80009283818384E090E0948383830E944565DE
:103C900080E597E0ADB7BEB712969C938E931197CF
:103CA00088E090E014969C938E9313970E9445654C
:103CB0008FE597E0EDB7FEB79283818380E190E0D6
:103CC000948383830E9445658EE697E0ADB7BEB7C7
:103CD00012969C938E93119780E290E014969C9399
:103CE0008E9313970E9445658BE797E0EDB7FEB77B
:103CF0009283818300E410E0148303830E9445656E
:103D00008AE897E0ADB7BEB712969C938E93119751
:103D100080E890E014969C938E9313970E944565DB
:103D200087E997E0EDB7FEB792838183148303831D
:103D30000E94456586EA97E0ADB7BEB712969C93A0
:103D40008E93119780E092E014969C938E93139734
:103D50000E94456586EB97E0EDB7FEB792838183BD
:103D600080E094E0948383830E94456583EC97E030
:103D7000ADB7BEB712969C938E93119780E098E0F2
:103D800014969C938E9313970E94456582ED97E05D
:103D9000EDB7FEB79283818380E090E194838383C3
:103DA0000E9445658FED97E0ADB7BEB712969C9324
:103DB0008E93119780E090E214969C938E931397C4
:103DC0000E9445652091A8040F900F900F900F90CE
:103DD000222309F470C200D000D0EDB7FEB73196AF
:103DE0008CEE97E023C26091A6047091A70480E056
:103DF00090E00E94AF64009751F160E070E04AE00B
:103E000050E00E946162DC01CB0190938F048093AB
:103E10008E0400D000D04DB75EB74F5F5F4F2FEEDE
:103E200037E0EDB7FEB732832183FA0193838283B3
:103E30000E9445650F900F900F900F908EE894E0D0
:103E40006BE070E042E050E00E948B6618C000D04A
:103E500000D08CE098E0ADB7BEB712969C938E93DD
:103E6000119780918E0490918F0414969C938E9359
:103E700013970E9445650F900F900F900F9020911F
:103E8000A804222309F417C200D000D0EDB7FEB772
:103E900031968DE298E0CAC10E94B12E2091A8040B
:103EA000222309F408C200D000D0EDB7FEB7319646
:103EB00080E398E0BBC100D083E398E0EDB7FEB7A4
:103EC000928381830E9445650F900F9080E00E944D
:103ED0002A120E94DC1000D000D086E498E0ADB732
:103EE000BEB712969C938E93119780E490E014963F
:103EF0009C938E9313970E94456500D0EDB7FEB753
:103F000031968EE598E0ADB7BEB712969C938E932E
:103F100011978091052082831382809106208483EB
:103F200015820E9445650F900F9081E798E0EDB7EC
:103F3000FEB79283818380918E0490918F04948345
:103F400083830E9445658CE898E0ADB7BEB71296B2
:103F50009C938E9311978091900490919104149664
:103F60009C938E9313970E9445650F900F900F902E
:103F70000F900E94F109AB01BC0100D000D000D02D
:103F800085EA98E0EDB7FEB792838183438354833B
:103F9000658376830E944565EDB7FEB736960FB60A
:103FA000F894FEBF0FBEEDBF0E943A0A0E940B0AB2
:103FB000AB01BC0100D000D000D082EB98E0ADB7DF
:103FC000BEB712969C938E931197EDB7FEB74383BD
:103FD0005483658376830E9445658DB79EB70696A8
:103FE0000FB6F8949EBF0FBE8DBF1D9B03C08AEC19
:103FF00092E002C086EC92E000D000D020EC38E0E5
:10400000ADB7BEB712963C932E93119714969C931E
:104010008E9313970E9445658091A81B9091A91BD0
:10402000A091AA1BB091AB1B4091AC1B5091AD1B52
:104030006091AE1B7091AF1B00D000D000D00DB7C7
:104040001EB70F5F1F4F2CEC38E0EDB7FEB7328381
:104050002183F80182839383A483B58346835783A6
:10406000608771870E944565EDB7FEB738960FB639
:10407000F894FEBF0FBEEDBF89EE98E09283818376
:104080000E94456580918C040F900F9081FF0EC0B7
:1040900000D086EF98E0ADB7BEB712969C938E9392
:1040A00011970E9445650F900F9017C080FF03C0C5
:1040B00083EC92E002C086EC92E000D000D02CEFBE
:1040C00038E0EDB7FEB732832183948383830E9467
:1040D00045650F900F900F900F9080918C0483FF97
:1040E00003C083EC92E002C086EC92E000D000D0E6
:1040F00020E039E0ADB7BEB712963C932E931197EE
:1041000014969C938E9313970E9445658091220686
:104110009091230623E139E0EDB7FEB73283218386
:10412000948383830E9445650F900F900F900F90AA
:10413000779903C083EC92E002C086EC92E000D055
:1041400000D020E239E0ADB7BEB712963C932E9373
:10415000119714969C938E9313970E944565209116
:10416000A8040F900F900F900F90222309F4A3C082
:1041700000D000D0EDB7FEB731968CE299E056C082
:104180000E94B3112091A804222309F494C000D006
:1041900000D0EDB7FEB731968FE299E047C00E949C
:1041A000B90E00D000D000D082E399E0EDB7FEB7A1
:1041B0009283818380914F1390915013A09151135A
:1041C000B091521383839483A583B6830E9445657F
:1041D0008DE399E0ADB7BEB712969C938E9311977D
:1041E0008091012090910220A0910320B0910420A1
:1041F000EDB7FEB783839483A583B6830E9445659C
:104200008DB79EB706960FB6F8949EBF0FBE8DBFB2
:104210000E94F80A2091A804222309F44CC000D07F
:1042200000D0EDB7FEB731968AE499E0ADB7BEB7DE
:1042300012969C938E93119722831382FBC96091EF
:10424000A6047091A70480E090E00E94AF6460E152
:1042500073E00E94C4640097A1F46091A604709179
:10426000A70480E090E00E94AF64009721F10E94D3
:10427000A663803100F590915201982B90935201E2
:104280001AC08091520100D000D02DE439E0EDB782
:10429000FEB73283218390E08F7090709483838384
:1042A0000E9445650F900F900F900F900E94F80AA2
:1042B00002C00E94FC0FA981BA8111961C921E9225
:1042C00083E00F900F90DF91CF911F910F91FF909E
:1042D000EF90DF90CF90BF90AF909F908F907F90A6
:1042E0006F905F904F903F902F900895F89491E2D7
:1042F000E0E0F0E0909357008491E2E0F0E09093EA
:1043000057004491E4E0F0E090935700E49190E08E
:10431000A0E0B0E0DC019927882750E060E070E081
:10432000762F652F542F4427840F951FA61FB71F84
:104330008E0F911DA11DB11D80932B1390932C13F3
:10434000A0932D13B0932E1378940895CF93DF93F9
:1043500000D000D000D0CDB7DEB7CE0101966DE021
:1043600070E042E050E00E946D6689819A812FEFF3
:104370008F3F920749F480E994E06DE070E042E0FD
:1043800050E00E948B6604C0909391048093900447
:10439000CE0101966BE070E042E050E00E946D6655
:1043A00089819A812FEF8F3F920779F48CE390E017
:1043B00090938F0480938E048EE894E06BE070E01D
:1043C00042E050E00E948B6604C090938F0480937B
:1043D0008E04CE01019669E070E042E050E00E9458
:1043E0006D6689819A812FEF8F3F920779F482E081
:1043F00090E090938D0480938C048CE894E069E0C5
:1044000070E042E050E00E948B6604C090938D04FF
:1044100080938C04CE0101966BE170E042E050E0A5
:104420000E946D6689819A812FEF8F3F920769F410
:10443000109223061092220682E296E06BE170E071
:1044400042E050E00E948B6604C090932306809364
:10445000220685EF9FE160E070E049E050E00E94B5
:104460006D660E94800CCE01039663E170E044E02B
:1044700050E00E946D668B819C81AD81BE818F3F33
:104480002FEF92072FEFA2072FEFB20749F48DEA23
:1044900094E063E170E044E050E00E948B6608C065
:1044A0008DEA94E063E170E044E050E00E946D66C4
:1044B000CE0103966FE070E044E050E00E946D662C
:1044C0008B819C81AD81BE818F3F2FEF92072FEFB3
:1044D000A2072FEFB20749F489EA94E06FE070E099
:1044E00044E050E00E948B6608C089EA94E06FE0E7
:1044F00070E044E050E00E946D66CE01039667E1F3
:1045000070E044E050E00E946D668B819C81AD813B
:10451000BE818F3F2FEF92072FEFA2072FEFB20739
:1045200049F481EB94E067E170E044E050E00E94E0
:104530008B6608C081EB94E067E170E044E050E0F6
:104540000E946D6626960FB6F894DEBF0FBECDBFF3
:10455000DF91CF9108956C9A6B9A6A9A6F9A729ACA
:10456000749A739A779A809880B3897F80BB87E02A
:1045700080937E00549A0E9476210E94A62181E0B9
:104580000E94020980E090E00E94940C0E948B350A
:104590000895CF93DF93EC0188819981009731F0E2
:1045A00027E08B37920709F077C06DC00E94AB22DD
:1045B00080918C0480FD02C00E94C43C80917000F8
:1045C0008C7F809370008091B60080628093B600EB
:1045D0001092B20082E08093B1008091B60090E02A
:1045E000877090700097C9F7809170008160809308
:1045F00070000E9416080E94B80880E090E067EA08
:1046000076E00E94963A0E94D71080E00E942A121B
:104610000E942D3F80932E060E94863D80932F0698
:1046200000D000D000D0EDB7FEB7319625E133E0E1
:10463000ADB7BEB712963C932E9311978283138227
:1046400080912E06848315820E9433651092310674
:10465000109230068DB79EB706960FB6F8949EBF9F
:104660000FBE8DBF82E894E09093FF1F8093FE1FE2
:1046700083E290E090933306809332068BE797E0D5
:10468000998388830DC0633259F480E396E060E03B
:1046900070E00E94FD12E6CF1982188283E001C00B
:1046A00081E0DF91CF9108958536910564F12091E5
:1046B00022063091230620FF10C000D000D027E250
:1046C00033E0EDB7FEB732832183948383830E9466
:1046D00033650F900F900F900F908091631B909116
:1046E000641BA091651BB091661B0196A11DB11DB5
:1046F0008093631B9093641BA093651BB093661B10
:1047000081E090E0089580E090E008954F925F92FC
:104710006F927F928F929F92AF92BF92CF92DF92D1
:10472000EF92FF920F931F93CF93DF93CDB7DEB736
:10473000CA57D0400FB6F894DEBF0FBECDBF2C01D4
:10474000633851F482E496E0EB966FAFEB970E94EA
:10475000D229EB966FADEB97D2018D919C91119779
:10476000009731F0B6E08A3A9B0709F08EC50EC07B
:1047700082E496E061E870E049EB54E00E94B729DA
:104780008AEA96E0F2019183808386C5623109F05E
:1047900083C50E94750F8091900480FF60C000D097
:1047A00000D000D0EDB7FEB7319672E0C72ED12C05
:1047B000CC0EDD1EADB7BEB71296DC92CE9211972D
:1047C00088E790E0938382838BE393E095838483EF
:1047D0000E949A658C0185EFA82E8FE1B82EEDB767
:1047E000FEB736960FB6F894FEBF0FBEEDBFEE24AF
:1047F000FF2498E7892E912C2FE3622E23E0722E5E
:10480000D5012D915D01EDB7FEB738970FB6F8943D
:10481000FEBF0FBEEDBF3196C601800F911FADB731
:10482000BEB712969C938E93119793828282758263
:104830006482268317820E949A65080F191F0894C4
:10484000E11CF11CEDB7FEB738960FB6F894FEBF29
:104850000FBEEDBFF8E0EF16F10491F602C000E0E4
:1048600010E08091900490919104009781F12DB710
:104870003EB7285030400FB6F8943EBF0FBE2DBF54
:10488000EDB7FEB73196CE010296800F911FADB7FE
:10489000BEB712969C938E93119788E790E093830E
:1048A000828384E493E09583848380911F069091B2
:1048B0002006978386830E949A65080F191FEDB71B
:1048C000FEB738960FB6F894FEBF0FBEEDBF8091CD
:1048D000900481FF51C089E290E06BE270E04AE20F
:1048E00050E027E00E94AC3285EF9FE10E94133533
:1048F0002DB73EB72A5030400FB6F8943EBF0FBEDA
:104900002DBFEDB6FEB60894E11CF11C9E012E5F92
:104910003F4F200F311FADB7BEB712963C932E9379
:10492000119728E730E0F701338322832BE433E04B
:10493000358324839C01B901882777FD8095982FC2
:104940000E944A6020E030E048EC52E40E94E05FC0
:10495000DC01CB01F70186839783A087B1870E9492
:104960009A65080F191F2DB73EB7265F3F4F0FB648
:10497000F8943EBF0FBE2DBF8091900482FF54C0BB
:1049800089E290E06BE270E04AE250E026E00E94AB
:10499000AC3281E090E00E948C0A80931E0683EE88
:1049A00092E10E941335ADB7BEB71A970FB6F894CF
:1049B000BEBF0FBEADBFEDB6FEB60894E11CF11C44
:1049C0009E012E5F3F4F200F311F12963C932E9376
:1049D000119728E730E0F7013383228325E533E0A0
:1049E000358324839C01B901882777FD8095982F12
:1049F0000E944A6020E030E048EC52E40E94E05F10
:104A0000DC01CB01F70186839783A087B1870E94E1
:104A10009A65080F191F2DB73EB7265F3F4F0FB697
:104A2000F8943EBF0FBE2DBF8091900483FF35C028
:104A30008DB79EB70A970FB6F8949EBF0FBE8DBF75
:104A4000EDB7FEB73196CE010296800F911FADB73C
:104A5000BEB712969C938E93119788E790E093834C
:104A6000828380E693E0958384838091D61290912F
:104A7000D712A091D812B091D91286839783A087BC
:104A8000B1870E949A65080F191FEDB7FEB73A96D5
:104A90000FB6F894FEBF0FBEEDBF8091900484FF67
:104AA00032C00E940B0AAB01BC012DB73EB72A50A1
:104AB00030400FB6F8943EBF0FBE2DBFEDB7FEB726
:104AC0003196CE010296800F911FADB7BEB71296F8
:104AD0009C938E93119788E790E0938382838EE670
:104AE00093E09583848346835783608771870E9410
:104AF0009A65080F191FEDB7FEB73A960FB6F894EE
:104B0000FEBF0FBEEDBF8091900485FF36C040917F
:104B1000A81B5091A91B6091AA1B7091AB1B2DB7CC
:104B20003EB72A5030400FB6F8943EBF0FBE2DBF9F
:104B3000EDB7FEB73196CE010296800F911FADB74B
:104B4000BEB712969C938E93119788E790E093835B
:104B500082838CE793E095838483468357836087C1
:104B600071870E949A65080F191FEDB7FEB73A9634
:104B70000FB6F894FEBF0FBEEDBF8091900486FF84
:104B80007EC080918E0490918F04009709F477C0C5
:104B9000F8948091A81B9091A91BA091AA1BB09199
:104BA000AB1B4091DA125091DB126091DC127091D4
:104BB000DD12841B950BA60BB70BBC01CD010E9427
:104BC0004860E62EC72EA82EF92E78942DB73EB752
:104BD0002A5030400FB6F8943EBF0FBE2DBF8DB6A1
:104BE0009EB60894811C911CCE010296800F911FE5
:104BF000ADB7BEB712969C938E93119788E790E05D
:104C0000F4019383828385E893E0958384836091A4
:104C10008E0470918F0480E090E00E9448609B01B8
:104C2000AC018E2D9C2DAA2DBF2DBC01CD010E9463
:104C3000E05FDC01CB01F40186839783A087B18715
:104C40000E949A65080F191FF8948091A81B9091F3
:104C5000A91BA091AA1BB091AB1B8093DA12909371
:104C6000DB12A093DC12B093DD1278942DB73EB71F
:104C7000265F3F4F0FB6F8943EBF0FBE2DBF809109
:104C8000900487FF3BC04091AC1B5091AD1B6091DD
:104C9000AE1B7091AF1B8DB79EB70A970FB6F894F5
:104CA0009EBF0FBE8DBFEDB7FEB73196CE01029607
:104CB000800F911FADB7BEB712969C938E9311973C
:104CC00088E790E09383828382E993E095838483ED
:104CD00046835783608771870E949A65080F191F62
:104CE000EDB7FEB73A960FB6F894FEBF0FBEEDBF14
:104CF000C8010E945423009709F0CDC2809190040E
:104D00009091910490FF7EC080918E0490918F04C9
:104D1000009709F477C0F8948091AC1B9091AD1B7B
:104D2000A091AE1BB091AF1B4091DE125091DF12EB
:104D30006091E0127091E112841B950BA60BB70BEA
:104D4000BC01CD010E944860E62EC72EA82EF92E88
:104D500078942DB73EB72A5030400FB6F8943EBF36
:104D60000FBE2DBF8DB69EB60894811C911CCE013E
:104D70000296800F911FADB7BEB712969C938E938B
:104D8000119788E790E0F401938382838BE993E0A5
:104D90009583848360918E0470918F0480E090E00D
:104DA0000E9448609B01AC018E2D9C2DAA2DBF2D29
:104DB000BC01CD010E94E05FDC01CB01F4018683E0
:104DC0009783A087B1870E949A65080F191FF894EE
:104DD0008091AC1B9091AD1BA091AE1BB091AF1B0D
:104DE0008093DE129093DF12A093E012B093E11251
:104DF00078942DB73EB7265F3F4F0FB6F8943EBF6D
:104E00000FBE2DBF809190049091910491FF3BC003
:104E10004091531B5091541B6091551B7091561B30
:104E20008DB79EB70A970FB6F8949EBF0FBE8DBF81
:104E3000EDB7FEB73196CE010296800F911FADB748
:104E4000BEB712969C938E93119788E790E0938358
:104E5000828388EA93E095838483468357836087BF
:104E600071870E949A65080F191FEDB7FEB73A9631
:104E70000FB6F894FEBF0FBEEDBFC8010E945423C9
:104E8000009709F008C2809190049091910492FFDC
:104E90003CC02DB73EB72A5030400FB6F8943EBF05
:104EA0000FBE2DBFEDB7FEB73196CE010296800F33
:104EB000911FADB7BEB712969C938E93119788E75A
:104EC00090E09383828381EB93E095838483809148
:104ED0004F1390915013A0915113B09152138683A8
:104EE0009783A087B1870E949A65080F191FEDB7B5
:104EF000FEB73A960FB6F894FEBF0FBEEDBFC801DD
:104F00000E945423009709F0C6C1809190049091AB
:104F1000910493FF3CC02DB73EB72A5030400FB6E6
:104F2000F8943EBF0FBE2DBFEDB7FEB73196CE0150
:104F30000296800F911FADB7BEB712969C938E93C9
:104F4000119788E790E0938382838CEB93E09583BD
:104F500084838091F01F9091F11FA091F21FB09176
:104F6000F31F86839783A087B1870E949A65080FF5
:104F7000191FEDB7FEB73A960FB6F894FEBF0FBEF5
:104F8000EDBFC8010E945423009709F084C18091AD
:104F900090049091910494FF4CC081E00E949D097F
:104FA000AB01BC012DB73EB72A5030400FB6F89484
:104FB0003EBF0FBE2DBFEDB6FEB60894E11CF11C3E
:104FC000CE010296800F911FADB7BEB712969C938B
:104FD0008E93119788E790E0F7019383828389ECA1
:104FE00093E095838483CB01BA012091AD04309185
:104FF000AE044091AF045091B0040E94FA60DC010D
:10500000CB01F70186839783A087B1870E949A65B9
:10501000080F191F2DB73EB7265F3F4F0FB6F89404
:105020003EBF0FBE2DBFC8010E945423009709F058
:1050300032C1809190049091910495FF4BC082E021
:105040000E949D09AB01BC018DB79EB70A970FB6B0
:10505000F8949EBF0FBE8DBFEDB6FEB60894E11C5E
:10506000F11CCE010296800F911FADB7BEB712960C
:105070009C938E93119788E790E0F7019383828346
:1050800086ED93E095838483CB01BA012091A90436
:105090003091AA044091AB045091AC040E94FA6094
:1050A000DC01CB01F70186839783A087B1870E943B
:1050B0009A65080F191F2DB73EB7265F3F4F0FB6F1
:1050C000F8943EBF0FBE2DBFC8010E945423009725
:1050D00009F0E1C0779A809122069091230693FD12
:1050E000749A809122069091230682FD08C08091D7
:1050F0008C0480FD04C081FF31C01D9B2FC000D0F7
:1051000000D083EE93E0ADB7BEB712969C938E931A
:105110001197CE01029614969C938E9313970E943A
:1051200033652091A8040F900F900F900F902223C9
:10513000A9F000D000D0EDB7FEB7319684EA99E02F
:10514000ADB7BEB712969C938E93119722831382AC
:105150000E9445650F900F900F900F9080914D0623
:105160008983FE01E00FF11F128280912206909147
:10517000230680FF12C000D000D08AEE93E0EDB786
:10518000FEB792838183C8010296948383830E9431
:1051900033650F900F900F900F9062E0C62ED12CC8
:1051A000C00ED11ECE010196B6010E94B831809189
:1051B0008C0482FF49C082E994E0BE016F5F7F4F9B
:1051C000A60120EB3BE10E940D36809122069091D2
:1051D000230692FF39C040EBE42E4BE1F42E00E0B1
:1051E00010E05BEFA52E53E0B52ED7018D917D0128
:1051F00000D000D0EDB7FEB73196ADB7BEB712966E
:10520000BC92AE921197828313820E9433650F5F26
:105210001F4F0F900F900F900F900031110529F73D
:105220008AE090E00E94656500D000D080E094E0C4
:10523000EDB7FEB792838183D482C3820E94336527
:105240000F900F900F900F9080912206909123065F
:1052500082FD73980E94D33B82E496E00E94D52998
:1052600080911F0690912006009711F00E94C43C87
:1052700080914D068F5F80934D068091220690911C
:10528000230682FF7DCA739A7BCAD20111961C92B3
:105290001E9283E002C001C081E0C658DF4F0FB606
:1052A000F894DEBF0FBECDBFDF91CF911F910F915C
:1052B000FF90EF90DF90CF90BF90AF909F908F9036
:1052C0007F906F905F904F9008950895FC01DB01EF
:1052D0008C91808311968C91119781830895FC01A4
:1052E000DB0190818C91981741F421E030E09181AD
:1052F00011968C911197981711F020E030E0C901B8
:105300000895BC0185E090E20E9466290895DC01C1
:105310001996ED91FC911A970280F381E02D309758
:1053200009F0099508950F931F93CF93DF9300D051
:10533000CDB7DEB78C0188E10E942732BC01CE01D7
:1053400001960E946629D8011996ED91FC911A9751
:105350000190F081E02DC801BE016F5F7F4F09957C
:105360000F900F90DF91CF911F910F910895EF92C1
:10537000FF920F931F93CF93DF93EC018B017A0180
:1053800047EC54E00E94E329FA86E986C8016BECF9
:1053900074E00E94412ADF91CF911F910F91FF90FD
:1053A000EF9008950E94FC290895CF93DF93EC01BC
:1053B00088E165E070E20E941D32CE010E94FF2963
:1053C000DF91CF910895EF92FF920F931F93CF93A8
:1053D000DF93EC018B017A010E941D2AF886EF828F
:1053E000C8016FEC74E00E94412ADF91CF911F91B8
:1053F0000F91FF90EF9008950E94262A08950E9431
:105400003C420895DC011796ED91FC9118970190AC
:10541000F081E02D09950895DC011796ED91FC913E
:1054200018970280F381E02D309709F009950895CF
:105430008EEC99E00E94902C0895FC0173836283A6
:105440008EEC99E0BF010E94032D0895BC018EEC03
:1054500099E00E94CE2C0895CF93DF93EC018EEC5F
:1054600099E00E94942C08C0FC01228133812C1702
:105470003D0721F00E943A2D0097B1F7DF91CF91BF
:1054800008950F931F93CF93DF938B010E942C2AD3
:10549000EC01009731F01D830C83C8010E947F440A
:1054A0008E83DF91CF911F910F9108951F93CF931A
:1054B000DF93EC01162F888580FF1DC0EC81FD81F4
:1054C0003097C9F0D093D109C093D00982E0888782
:1054D000CE0106960995992787FD9095029782300F
:1054E000910510F0133829F4CE01BE010E947F2AE5
:1054F00002C081E08887DF91CF911F910895CF92FC
:10550000DF92EF92FF920F931F93CF93DF93EC0103
:105510007B01C090D009D090D1090091D20910919F
:10552000D309F80103C00190F081E02DEC17FD07CD
:1055300019F03097C1F746C0209709F443C0888519
:10554000882309F118860BC0C017D10729F0C801BC
:1055500067E8AE010E94562AF80100811181011509
:10556000110591F7EC81FD81309769F0CE15DF05CB
:1055700051F0D093D109C093D009CE01069663E8CB
:1055800040E050E00995E091D209F091D309CE179F
:10559000DF0791F4888199819093D3098093D20990
:1055A0000DC0808191818C179D0729F48881998194
:1055B0009183808303C0FC01309799F7D092D10981
:1055C000C092D009DF91CF911F910F91FF90EF9082
:1055D000DF90CF9008951F93CF93DF931092D4095B
:1055E000C091D209D091D30911E00EC089858823DA
:1055F00041F018871986CE0162E840E050E00E9431
:10560000562A0990D881C02D209781F7DF91CF913C
:105610001F9108958091D509982F9F5F9093D50988
:1056200008956091D0097091D1090E947F2A089550
:105630008AE88093D5091092D6091092D709109262
:10564000D3091092D2091092D1091092D00908956D
:105650008091D409882311F00E94EB2A7091D70918
:10566000772309F455C02091D60930E0F901EE0FF7
:10567000FF1FEE0FFF1FE20FF31FE852F64F60818E
:105680006093780A4181528150937A0A4093790A53
:105690008381948190937C0A80937B0A2F5F3F4F94
:1056A0002F7130702093D60971507093D7090097ED
:1056B00041F58091D2099091D30918C08091D40905
:1056C000882311F00E94EB2A4091790A50917A0ABE
:1056D00080917D0A90917E0A6091780A0E94562AF4
:1056E000E0917D0AF0917E0A8081918190937E0AFB
:1056F00080937D0A80917D0A90917E0A0097F1F651
:1057000007C0613819F421E0FC0120870E94562A65
:105710008091D4092091D70990E0820F911D0895BE
:105720008091D4092091D70990E0820F911D0895AE
:105730009C017091D7097032D9F08091D609870FFA
:105740008F7180937F0A90E0FC01EE0FFF1FEE0F38
:10575000FF1FE80FF91FE852F64F60835283418321
:10576000348323837F5F7093D70980E090E00895AE
:1057700081E090E00895CF93DF93C091D009D0915C
:10578000D1090E94562AD093D109C093D009DF9144
:10579000CF910895FC01AB019091D2098091D3097A
:1057A000A92FB82F03C00D90BC91A02DAE17BF0735
:1057B00091F01097C1F7309771F090838183F09347
:1057C000D309E093D20981E0808717821682CF0146
:1057D00061E80E94BB2B0895FC01009741F0808591
:1057E0008150823020F481E081878093D40908952C
:1057F00021E030E0FC018085882311F420E030E0D6
:10580000C9010895CF93DF93EC014A815B818C81BC
:105810009D8160E070E00E94BD642A813B818881A7
:105820009981289FA001299F500D389F500D112468
:105830008E819F8160E070E00E94BD64DF91CF9116
:105840000895DC0112962D913C91139780E090E031
:105850001DC01496ED91FC911597E80FF91F40813A
:10586000442399F421E020832D913C911197829F4C
:10587000A001839F500D929F500D112416968D917B
:105880009C911797840F951F08950196821793078F
:1058900001F780E090E00895FC0146815781A281E4
:1058A000B38120E030E019C04617570781F4A48186
:1058B000B581A20FB31F8C91181614F481508C93EC
:1058C0000480F581E02DE20FF31F8081089580812F
:1058D0009181480F591F2F5F3F4F2A173B0721F730
:1058E0008FEF0895FC014681578164177507A8F072
:1058F000A081B18182819381A89F9001A99F300DE1
:10590000B89F300D1124240F351F81E090E06217FD
:10591000730728F080E090E0089580E090E008951B
:10592000FC01118210820895FC018081918108950B
:10593000FB0120813181FC01318320830895FC012A
:1059400080819181009711F40895C901FC012081A3
:10595000318121153105C9F70895DC01ED91FC91E4
:105960001197309729F40BC0DF010190F081E02DF1
:10597000808191810097C1F711961C921E92CF01F0
:105980000895DC01ED91FC911197309729F0808109
:10599000918111969C938E93CF010895CF93DF93BD
:1059A000EC01E881F9813097B9F0A0E0B0E002C0E5
:1059B000DF01FC0180819181E617F70759F4109708
:1059C00019F49983888303C011969C938E93118256
:1059D000108202C0009761F7DF91CF9108950F9375
:1059E0001F93CF93DF938C01EB010E94CE2CF80123
:1059F0008081918199838883D183C083DF91CF9106
:105A00001F910F9108950F931F93CF93DF938C01F4
:105A1000EB010E94CE2C19821882C8010E949F2C93
:105A2000009711F4F80101C0FC01D183C083DF911C
:105A3000CF911F910F910895DC01ED91FC91119789
:105A400080E090E004C001960190F081E02D309755
:105A5000D1F70895FB01BA01309719F40E94EF2C99
:105A6000089580819181DA0111969C938E935183E0
:105A700040830895009721F0FC0180819181089571
:105A800080E090E008958091800A9091810A0097CB
:105A900029F41092830A1092820A08950E944439D0
:105AA000BC01E091800AF091810A4281538180819A
:105AB0009181480F591F461B570B0CC0828193815F
:105AC00020813181820F931F861B970B84179507C6
:105AD00008F4AC010480F581E02D309779F7460F8A
:105AE000571F5093830A4093820A08958DED94E0E6
:105AF0000E94EC2B0895EF92FF920F931F93CF9388
:105B0000DF937C01FC0180819181009729F08A3527
:105B1000910509F06DC00BC01092810A1092800AA5
:105B20008AE590E0F7019183808381E065C0673862
:105B300059F5A091800AB091810A04C014960D9085
:105B4000BC91A02D109741F316968D919C911797BB
:105B50008417950799F3A093800AB093810A0DC02A
:105B6000868197818417950739F4848195811596EC
:105B70009C938E931497FD01DF011496ED91FC9197
:105B80001597309769F7CCCF623851F6C091800AEB
:105B9000D091810A00E010E028C0CE010E94644844
:105BA0000097F1F08E819F8168E8AE010E94982BEA
:105BB0000097A1F41F821E828C819D810115110521
:105BC00021F0F8019583848304C09093810A809327
:105BD000800A1D821C820E94432DD8CF0E94762D00
:105BE0009C818D818E01C92FD82F2097B1F698CF37
:105BF000F7011182108283E0DF91CF911F910F9105
:105C0000FF90EF900895CF93DF93EC010E94762DE3
:105C10008E819F813091800A2091810A009759F0EE
:105C2000E32FF22F06C0EC17FD0789F00480F58101
:105C3000E02D3097C1F78091D0099091D1099F83D1
:105C40008E833C832D83D093810AC093800A0E9467
:105C5000432DDF91CF910895CF93DF93EC010E9404
:105C60004448CE010E94032EDF91CF910895CF9337
:105C7000DF93EC010E945048CE010E94032EDF9179
:105C8000CF910895CF93DF93EC010E945A48CE0143
:105C90000E94032EDF91CF910895FC0180819181B4
:105CA000860F971F918380830E94432D089521E0E2
:105CB00030E0FC0186819781009711F020E030E010
:105CC000C9010895FC012281338180819181280FCF
:105CD000391FC9010895FC0180819181089581E0F7
:105CE00090E02091800A3091810A2115310511F44C
:105CF00080E090E008958091800A9091810A009759
:105D000029F08091820A9091830A089580E090E0C2
:105D10000895CF93DF93EC01E091800AF091810A1E
:105D20008E179F0741F48C819D819093810A809307
:105D3000800A14C0FC01309731F0848195818C1762
:105D40009D07C1F707C01D821C821F821E82DF9142
:105D5000CF9108958C819D81958384830E94432DEA
:105D6000F2CFCF93DF93D0910520C09106200E94FF
:105D70007039AB01BC018DB79EB7825590400FB60C
:105D8000F8949EBF0FBE8DBFEDB7FEB731968AEA7D
:105D900099E0ADB7BEB712969C938E931197D283BC
:105DA0001382C483158246835783608771878091ED
:105DB000F8219091F921A091FA21B091FB218287DD
:105DC0009387A487B5878091FC219091FD21A091B4
:105DD000FE21B091FF2186879787A08BB18B8091A0
:105DE000002290910122A0910222B0910322828B85
:105DF000938BA48BB58B8091042290910522A09166
:105E00000622B0910722868B978BA08FB18F80914D
:105E1000082290910922A0910A22B0910B22828F30
:105E2000938FA48FB58F80910C2290910D22A09119
:105E30000E22B0910F22868F978FA0A3B1A38091DD
:105E4000102290911122A0911222B091132282A3CC
:105E500093A3A4A3B5A38091142290911522A0919D
:105E60001622B091172286A397A3A0A7B1A780916D
:105E7000182290911922A0911A22B0911B2282A778
:105E800093A7A4A7B5A780911C2290911D22A09151
:105E90001E22B0911F2286A797A7A0ABB1AB80911D
:105EA000202290912122A0912222B091232282AB24
:105EB00093ABA4ABB5AB8091242290912522A09105
:105EC0002622B091272286AB97ABA0AFB1AF8091CD
:105ED000282290912922A0912A22B0912B2282AFD0
:105EE00093AFA4AFB5AFEDB7FEB7FF9680912C226C
:105EF00090912D22A0912E22B0912F228083918308
:105F0000A283B383EDB7FEB7ED5BFF4F80913022E4
:105F100090913122A0913222B091332280839183DB
:105F2000A283B383EDB7FEB7E95BFF4F80913422C4
:105F300090913522A0913622B091372280839183AF
:105F4000A283B383EDB7FEB7E55BFF4F80913822A4
:105F500090913922A0913A22B0913B228083918383
:105F6000A283B383EDB7FEB7E15BFF4F80913C2284
:105F700090913D22A0913E22B0913F228083918357
:105F8000A283B3830E944565D0910520C09106206D
:105F90008DB79EB78E5A9F4F0FB6F8949EBF0FBE17
:105FA0008DBF0E947039AB01BC01ADB7BEB7D297AF
:105FB0000FB6F894BEBF0FBEADBFEDB7FEB73196BA
:105FC00086E89AE012969C938E931197D28313825F
:105FD000C4831582468357836087718780914022EE
:105FE00090914122A0914222B091432282879387CF
:105FF000A487B5878091442290914522A0914622A2
:10600000B091472286879787A08BB18B80914822D9
:1060100090914922A0914A22B0914B22828B938B7E
:10602000A48BB58B80914C2290914D22A0914E2251
:10603000B0914F22868B978BA08FB18F8091502289
:1060400090915122A0915222B0915322828F938F2E
:10605000A48FB58F8091542290915522A091562201
:10606000B0915722868F978FA0A3B1A38091582219
:1060700090915922A0915A22B0915B2282A393A3BE
:10608000A4A3B5A380915C2290915D22A0915E2291
:10609000B0915F2286A397A3A0A7B1A780916822A1
:1060A00090916922A0916A22B0916B2282A793A756
:1060B000A4A7B5A780916C2290916D22A0916E2229
:1060C000B0916F2286A797A7A0ABB1AB0E944565A0
:1060D0008DB79EB7C2960FB6F8949EBF0FBE8DBF08
:1060E000DF91CF91089580E38093880A0895CF933C
:1060F000DF936091880A70E0C0E3D0E0C61BD70B45
:106100006557754FAE010E94B464CE01DF91CF9107
:106110000895CF92DF92EF92FF920F931F93CF9348
:10612000DF937C01C090860AD090870A6091880A2C
:1061300070E08601005D1F4F061B170B013811052B
:10614000D8F4C0E3D0E0C61BD70B6557754FAE013E
:106150000E94B464C7018C0F9D1F6091890A7091E1
:106160008A0A2091840A3091850A620F731FA60162
:106170000E94B464C80102C080E090E0DF91CF913A
:106180001F910F91FF90EF90DF90CF900895909125
:10619000880A980F9093880A08954091860A509132
:1061A000870A9C014817590798F08091840A9091BA
:1061B000850A820F931F9093850A8093840A421B5D
:1061C000530B5093870A4093860A81E090E008952C
:1061D00080E090E008959093870A8093860A08955E
:1061E0008091840A9091850A8554954F08958091F5
:1061F000880A90E08557954F089581E090E02091BE
:10620000890A30918A0A4AE02B3B340711F480E076
:1062100090E008950E94FD30009769F08BEB9AE0C2
:106220006091890A70918A0A4091860A5091870A82
:106230000E94B46408954091840A5091850A4115E2
:106240005105C1F08091860A9091870AC096ABEB08
:10625000BAE020E330E007C0FD01E40FF51F6081E4
:106260006D932F5F3F4F28173907B4F31092850ABB
:106270001092840A08958091890A90918A0A08955B
:106280008091860A9091870A08959091880A80E308
:10629000891B089520E38091880A281B8091860A33
:1062A0009091870A820F911D08951F93CF93DF93DA
:1062B000EC011091880A812F90E08C179D076CF0FB
:1062C0000E944A318C0F9D1F8138910530F41C1BB0
:1062D0001093880A81E090E002C080E090E0DF91B6
:1062E000CF911F910895CF93DF93EFE0F0E21192E9
:1062F000119280E2EF33F807D1F7C0E0D0E0CE0191
:10630000880F991F895F9F4D65EC74E00E94662994
:106310002196C430D10599F7DF91CF91089510925D
:10632000850A1092840A1092870A1092860A80E3E6
:106330008093880A8BEB9AE090938A0A8093890A6B
:106340000E94733108950F931F93CF93DF93EC0155
:106350008B010E948F31D0938A0AC093890A1093CF
:10636000870A0093860ADF91CF911F910F910895BC
:10637000EF92FF920F931F93CF93DF9300D0CDB78F
:10638000DEB78C0169837A830E948F316981E62EA2
:106390007A81F72E81E8E816F10418F030E8E32E50
:1063A000F12C8091890A90918A0AB801A7010E9474
:1063B000B464F092870AE092860AC7010F900F90AA
:1063C000DF91CF911F910F91FF90EF900895FC0105
:1063D000AFE0B0E280E30D9001928150E1F7FB0164
:1063E000A7E0B0E288E00D9001928150E1F70895B6
:1063F000AFE0B0E2FC0180E301900D928150E1F743
:10640000A7E0B0E2FB0188E001900D928150E1F736
:106410000895E82FF0E0EE0FFF1FE15FFF4D71835D
:10642000608381E090E00895E82FF0E0EE0FFF1F19
:10643000E15FFF4D80819181089590E0880F991F61
:106440008952904E0E94662981E090E0089590E084
:10645000880F991F8952904E08958115910511F06A
:106460000197F1F70895E0914220F0914320908147
:106470008091412089230895E0913F20F0914020B0
:10648000808190914120892B8083E0914420F0917C
:106490004520808190914120892B80830895E0914F
:1064A0003F20F09140209081809141208095892368
:1064B0008083E0914420F09145209081809141209B
:1064C00080958923808308951F93CF93DF93E09174
:1064D0003F20F09140209081809141208095892338
:1064E0008083E0914420F09145208081909141206B
:1064F000892B80838FEB93E00E942D321FB7F89495
:10650000E0914420F0914520908180914120809538
:106510008923808383E890E00E942D32E09142201D
:10652000F0914320D081C09141201FBF78948BE32C
:1065300093E00E942D32E0914220F091432080812F
:1065400090914120892319F08D2F8C2301C081E087
:10655000DF91CF911F91089550934520409344209F
:106560007093402060933F2090934320809342207B
:1065700081E090E002C0880F991F2A95E2F780938E
:1065800041200E9464320895CF93DF93C82FDFB774
:10659000F894E0914420F091452080819091412031
:1065A000892B808383E090E00E942D32CC2351F030
:1065B000E0914420F0914520908180914120809588
:1065C0008923808387E190E00E942D32E091422070
:1065D000F0914320808190914120892309F4C0E00B
:1065E00089E590E00E942D32E0914420F091452011
:1065F000908180914120809589238083DFBF8BE348
:1066000090E00E942D328C2FDF91CF910895CF938F
:10661000DF93C82FD8E08C2F81700E94C432C695BA
:106620008111C068D150B9F78C2FDF91CF910895B7
:106630008FEF0E9407330895DF92EF92FF920F933E
:106640001F93CF93DF93182FEB010E9464328823AE
:1066500081F580EF0E940733EE2400E498E0D92E04
:1066600081E00E94C432F82E81E00E94C432882367
:1066700019F0FF2069F020C0FF2051F4011728F025
:10668000888180FF05C0101719F0E02EFF24F394D5
:106690008F2D0E94C432888186958883FF2011F057
:1066A000806888830150DA94D9F621960023B1F6E8
:1066B00005C0EE24EA9402C08EEFE82E8E2DDF9105
:1066C000CF911F910F91FF90EF90DF9008950F935E
:1066D0001F93CF93DF93182FEB010E946432209712
:1066E00051F085E50E94073308E089910E94073345
:1066F0000150D9F703C08CEC0E940733812F0E9410
:106700000733DF91CF911F910F9108950F931F933E
:10671000CF93DF93E82FDB01EA01B9014C9150E000
:1067200011969C91119780E0482B592BE03181F410
:10673000CA018E7F33E0880F991F3A95E1F71696CC
:106740002C9116974CE050E0421B5109480F591FFD
:1067500057FF06C081E08883509541955F4F01C087
:106760001882E83299F414968C91149790E09C0169
:10677000207630702036310549F086FF02C04E7F0A
:1067800005C085FF02C04C7F01C0487FCA0124E0DC
:10679000969587952A95E1F7FB0180834F70F80164
:1067A000408380E0DF91CF911F910F9108950F9367
:1067B0001F93CF93DF93EC018B018881B8010E9476
:1067C0001C33888381508D3F30F4F80180818832FA
:1067D00011F0803191F7DF91CF911F910F910895C2
:1067E000CF93DF93EC010E94643284EBBE010E94E0
:1067F000673381E00E94C432C82F0E94643281E076
:10680000CC2309F480E0DF91CF9108951F93CF93BB
:10681000DF93182FEB010E9464320E9433328823E9
:1068200049F084E4BE010E946733113029F00E94D0
:106830003C3202C082E001C080E0DF91CF911F9125
:1068400008956F927F928F929F92BF92CF92DF9224
:10685000EF92FF920F931F93CF93DF93CDB7DEB7E5
:1068600029970FB6F894DEBF0FBECDBF7C014B0158
:106870003A0169010E9464328EEBB7010E946733CE
:106880008E010F5F1F4FE9E0BE2E0E941833F80102
:1068900081938F01BA94C9F7CE01019669E070E047
:1068A0000E94324E882361F4F7018081BE016F5F40
:1068B0007F4FA401930186010E94863380E001C0CE
:1068C00083E029960FB6F894DEBF0FBECDBFDF91EF
:1068D000CF911F910F91FF90EF90DF90CF90BF90DD
:1068E0009F908F907F906F9008958F929F92AF921C
:1068F000BF92CF92DF92EF92FF920F931F93CF93AD
:10690000DF93CDB7DEB729970FB6F894DEBF0FBE81
:10691000CDBFD82E5B014A0179018EEB60E070E0BB
:106920000E9467338E010F5F1F4FF9E0CF2E0E9448
:106930001833F80181938F01CA94C9F7CE010196EB
:1069400069E070E00E94324E882359F48D2DBE011B
:106950006F5F7F4FA501940187010E94863380E01D
:1069600001C083E029960FB6F894DEBF0FBECDBFFD
:10697000DF91CF911F910F91FF90EF90DF90CF901B
:10698000BF90AF909F908F900895EF92FF921F93CA
:10699000CF93DF93CDB7DEB728970FB6F894DEBF5D
:1069A0000FBECDBF182F262FDE011196E7EEF4E0C3
:1069B00088E001900D928150E1F7E42EFF24E7FC7E
:1069C000F09441E752E0E49EC001E59E900DF49EF4
:1069D000900D112464E670E00E949061CB0134E6D2
:1069E000239F90011124820F931FFE01319640E0F6
:1069F000219130E0E216F30611F4019603C04F5FD7
:106A00004830B1F7112319F0909581959F4F289642
:106A10000FB6F894DEBF0FBECDBFDF91CF911F91AF
:106A2000FF90EF9008950F931F93CF93DF93CDB70F
:106A3000DEB72B970FB6F894DEBF0FBECDBF182F71
:106A4000092F885F612F792F0E940634882309F06F
:106A500048C066E471E48FE090E00E947E35812FAB
:106A6000902FBE016D5F7F4FAE014E5F5F4F9E0165
:106A70002F5F3F4F0E942134882399F5DE01149641
:106A8000E7EEF4E088E001900D928150E1F7E981B2
:106A90004E2F50E021E732E0429FC001439F900D0E
:106AA000529F900D112464E670E00E949061CB012A
:106AB0003A8124E6329F90011124820F931FDE0158
:106AC000149620E03D91E31711F4019603C02F5F67
:106AD0002830C1F72B81222331F0909581959F4F6B
:106AE00002C084E391E22B960FB6F894DEBF0FBE8E
:106AF000CDBFDF91CF911F910F910895DC01CB01A4
:106B000081159105A105B10529F081509040A04063
:106B1000B040D9F708951092B90080E28093B80090
:106B2000089594EA9093BC009091BC0097FFFCCF2D
:106B30009091B900987F983011F0903199F480933A
:106B4000BB0084E88093BC008091BC0087FFFCCF31
:106B50009091B900987F983139F081E0903429F410
:106B600080E0089581E0089580E0089544EA34E8E3
:106B700024E94093BC009091BC0097FFFCCF90911A
:106B8000B900987F983011F0903199F78093BB004D
:106B90003093BC009091BC0097FFFCCF9091B9005E
:106BA000987F903211F0983539F42093BC00909181
:106BB000BC0094FDFCCFDDCF08950E94913508956F
:106BC00084E98093BC008091BC0084FDFCCF0895D3
:106BD0008093BB0084E88093BC008091BC0087FF59
:106BE000FCCF9091B900987F81E0983209F480E061
:106BF000089584EC8093BC008091BC0087FFFCCF9B
:106C00008091BB00089584E88093BC008091BC0013
:106C100087FFFCCF8091BB000895FC0180E191913A
:106C200090933F018150D9F780913C018F7D8093F3
:106C30003C0180913C01877F80933C01FB0180E116
:106C4000919190933E018150D9F780913C018068E9
:106C500080933C0180913D0180FFFCCF405150402A
:106C600080913C01806280933C0180913C01877F50
:106C700080933C0112C0FB0180E1919190933E0111
:106C80008150D9F780913C01806880933C018091CC
:106C90003D0180FFFCCF40515040141615065CF3B7
:106CA000F90180E190913E0191938150D9F781E003
:106CB00090E00895E6E4F1E08081208190813081C8
:106CC000829586958695837022952F70822B832BD3
:106CD00092959F70892B0895DF92EF92FF920F9308
:106CE0001F93CF93DF9300D0CDB7DEB780E06CE089
:106CF00046E00E94083A89E18093C4001092C500E2
:106D000082E08093C00080E00E94AA3A0E94343959
:106D100084B784B784B784B784B7E6ECF8E222E49A
:106D200032E4318320833A968DB79EB70A97E817ED
:106D3000F907B8F300D000D085EF9AE0ADB7BEB741
:106D400012969C938E9311978FEE94E014969C93D9
:106D50008E9313970E9445650F900F900F900F90A0
:106D60000E94634A0E94182B8DED94E060E070E071
:106D70000E94CA2B0E94F648E0913A05F0913B052B
:106D800009950E945A3690E00E94A04ACE010196D1
:106D90000E946638882359F000D080E19BE0EDB76F
:106DA000FEB7928381830E9445650F900F90CE01BC
:106DB00001960E9481290E9470388C010E947538CA
:106DC000BC01C801AE014F5F5F4F0E94A43D0E940D
:106DD000D3370E94893D0E947A380E94253F00D017
:106DE00080E39BE0ADB7BEB712969C938E9311974C
:106DF0000E94456500D0EDB7FEB731960DE31BE06C
:106E0000ADB7BEB712961C930E9311978A818283F9
:106E100013820E944565EDB7FEB73196ADB7BEB798
:106E200012961C930E9311978981828313820E947C
:106E300045650F900F9081E49BE0EDB7FEB792831C
:106E400081830E9445650F900F900E94A64AE091B1
:106E5000BD05F091BE050995E091A405F091A50549
:106E60000995E0916605F091670509950091A205E5
:106E70001091A305E090BB05F090BC050E94863DF3
:106E8000D82E0E942D3F2DB73EB72A5030400FB666
:106E9000F8943EBF0FBE2DBFEDB7FEB7319623E489
:106EA0003BE0ADB7BEB712963C932E931197138378
:106EB0000283F582E482D6821782808711860E943F
:106EC0004565E091C705F091C8052DB73EB7265F2F
:106ED0003F4F0FB6F8943EBF0FBE2DBF3097D1F095
:106EE0000995BC0100D000D08EE59BE0ADB7BEB7E0
:106EF00012969C938E93119780E890E00E947C619B
:106F0000EDB7FEB7748363830E9445650F900F90C1
:106F10000F900F9000D081E79BE0ADB7BEB71296FF
:106F20009C938E9311970E9445650F900F908FEF61
:106F300095E060E070E00E94CA2B88E094E00E9437
:106F4000284800D083E79BE0EDB7FEB792838183AA
:106F50000E9445650F900F900F900F90DF91CF9199
:106F60001F910F91FF90EF90DF90089500D000D017
:106F700000D0EDB7FEB731962BE73BE0ADB7BEB71B
:106F800012963C932E931197938382837583648327
:106F90000E9445658DB79EB706960FB6F8949EBFC2
:106FA0000FBE8DBF08950F931F93CF93DF93CDB77F
:106FB000DEB7A0970FB6F894DEBF0FBECDBF82E25A
:106FC00090E00E948566082F282F2B50203108F072
:106FD000982F9095891709F46DC000D081EA9BE045
:106FE000ADB7BEB712969C938E9311970E944565DC
:106FF0008E010F5F1F4F0F900F90D80180E090E03F
:10700000FC01E756F44FE491ED9301968830910529
:10701000B9F7F894CE0101966EE370E048E050E0D5
:107020000E948B66D80180E090E0FC01E557F44FA8
:10703000E491ED9301968E309105B9F7CE0101965A
:1070400060E370E04EE050E00E948B6680E090E0EC
:10705000FC01EF57F44FE491D801ED938D010196B7
:107060008A309105A9F7CE01019666E270E04AE008
:1070700050E00E948B6680E290E06DEC7BEA0E941B
:10708000A3668EE190E060E070E00E94A3668DE16F
:1070900090E060E00E94956684E290E060E070E03D
:1070A0000E94A3660AE182E290E06AE175EE0E9426
:1070B000A3667894802FA0960FB6F894DEBF0FBE1B
:1070C000CDBFDF91CF911F910F910895F8946EE39A
:1070D00070E042E050E00E946D66789480E0089590
:1070E00080E290E00E94856608958EE190E00E9423
:1070F000856608958DE190E00E947D660895409137
:10710000542050915520609156207091572090E066
:10711000A0E0B0E0480F591F6A1F7B1F4093542026
:1071200050935520609356207093572040915020E3
:10713000509151206091522070915320480F591F57
:107140006A1F7B1F40935020509351206093522020
:10715000709353202091F4212223A1F040914C20E0
:1071600050914D2060914E2070914F20480F591F33
:107170006A1F7B1F40934C2050934D2060934E20FC
:1071800070934F2008951F920F920FB60F920BB677
:107190000F9211242F933F934F935F936F937F939D
:1071A0008F939F93AF93BF93EF93FF9380913F0B88
:1071B0009091400B01969093400B80933F0B8091F0
:1071C0003E0B8F5F80933E0B8038A9F410923E0BEC
:1071D0008091542090915520A0915620B091572035
:1071E0000196A11DB11D8093542090935520A0932A
:1071F0005620B09357208091F4218823E1F08091AC
:107200003D0B8F5F80933D0B8038A9F410923D0BAE
:1072100080914C2090914D20A0914E20B0914F2014
:107220000196A11DB11D80934C2090934D20A093F9
:107230004E20B0934F200E946F2E009711F00E94B5
:10724000762DFF91EF91BF91AF919F918F917F919B
:107250006F915F914F913F912F910F900BBE0F90C7
:107260000FBE0F901F901895F8941092B60016BCA0
:1072700083EF87BD82E084BD94E095BD95B395BB57
:1072800080936E007894089580913F0B9091400B0D
:1072900020913F0B3091400B82179307A9F7089577
:1072A00007C022E330E0000021503040E1F70197B1
:1072B0000097B9F708950F931F93CF93DF938C0135
:1072C0000E944439EC010E9444398C1B9D0B8017AD
:1072D0009107C8F3DF91CF911F910F910895089501
:1072E0000F931F9300915420109155202091562008
:1072F000309157208091542090915520A091562094
:10730000B0915720081719072A073B0759F7B8010A
:10731000C9011F910F9108951F920F920FB60F92FE
:107320001124109205050F900FBE0F901F90189515
:107330001F920F920FB60F920BB60F9211242F933C
:107340003F934F935F936F937F938F939F93AF93ED
:10735000BF93EF93FF93E091FB04F091FC048081D5
:10736000E0910605F0910705309709F00995FF9126
:10737000EF91BF91AF919F918F917F916F915F91AD
:107380004F913F912F910F900BBE0F900FBE0F901A
:107390001F9018951F920F920FB60F921124109202
:1073A00012050F900FBE0F901F9018951F920F920D
:1073B0000FB60F920BB60F9211242F933F934F935A
:1073C0005F936F937F938F939F93AF93BF93EF934D
:1073D000FF93E0910805F09109058081E091130584
:1073E000F0911405309709F00995FF91EF91BF9145
:1073F000AF919F918F917F916F915F914F913F914D
:107400002F910F900BBE0F900FBE0F901F901895ED
:1074100090E02DE030E0829FF001839FF00D929F7D
:10742000F00D1124E550FB4FA281B3811C92A48181
:10743000B5816C93A681B78188ED8C93A085B185C9
:107440004C93128614861386089590E02DE030E068
:10745000829FF001839FF00D929FF00D1124E55063
:10746000FB4F81E08287A081B1816C933A96808145
:107470008823E9F70895CF93C82F8A3031F480919B
:10748000810B6DE00E94253A02C08D3029F0809179
:10749000810B6C2F0E94253A80E090E0CF910895F7
:1074A0001F93CF93DF93182FEB010CC08A3021F488
:1074B000812F6DE00E94253A69916D3019F0812F7E
:1074C0000E94253A8881882389F7DF91CF911F9107
:1074D00008950F931F93CF93DF93CDB7DEB79E012F
:1074E000265F3F4F01E41BE0C80160E470E048857F
:1074F00059850E94D7658F81B8010E94503ADF916B
:10750000CF911F910F9108951F93CF93DF93182F61
:10751000EB0104C0812F0E94253A2196FE0164915F
:107520006623C1F7DF91CF911F91089590E02DE080
:1075300030E0829FF001839FF00D929FF00D1124A7
:10754000E550FB4F748763870895682F80E00E94A1
:10755000253A08958093810B85E195E09093C128A9
:107560008093C028089584B7877F84BF88E10FB6D1
:10757000F89480936000109260000FBE08952FE091
:1075800088E190E00FB6F894A895809360000FBE54
:10759000209360000895A895089588E10FB6F894A7
:1075A00080936000109260000FBE0895F89428E068
:1075B00088E190E00FB6F894A895809360000FBE24
:1075C00020936000FFCF80915F2080915F2090E04A
:1075D00008958091390181FD10C081E491E06FE14F
:1075E00040E00E94C440813059F021E030E0813118
:1075F00011F020E030E0C901089580E090E00895A6
:1076000081E090E0089581E491E06FE140E00E9424
:10761000C4400895E9E3F1E0808180818D7F80831B
:107620008DE090E00197F1F782E491E06FE140E0B6
:1076300023E00E94CE4083E090E00197F1F70895A7
:107640009091390191FD0AC0282F803108F02FE078
:1076500085E491E06FE040E00E94CE400895809183
:10766000390181FD13C081E491E06FE140E00E94A7
:10767000C440982F8151823038F09F3129F09130E9
:1076800019F081E0923019F480E0089581E00895C6
:107690000E942F3B8823E1F30895CF93DF93C82FF7
:1076A000883049F0863039F0893029F0863119F078
:1076B000893109F045C08091390181FD44C00E94A3
:1076C000483B0E94033BD82FC817B9F1C83019F4C2
:1076D0000E940A3B2BC0C93141F48631A9F482E4EF
:1076E00091E06FE140E029E009C0C63169F48931D9
:1076F00059F482E491E06FE140E026E00E94CE4040
:10770000E3E0F0E03197F1F782E491E06FE140E0EF
:107710002C2F0E94CE40D83029F489E691E00197C1
:10772000F1F704C0E3E0F0E03197F1F70E94033B8A
:107730008C1719F083E490E008C080E490E005C065
:1077400082E490E002C084E490E0DF91CF9108955C
:10775000809194009091950090938D2280938C223B
:1077600021E0209379228091390181FF15C0209377
:10777000F3218091940090919500909389228093B9
:10778000882220937722809139018D7F809339015F
:107790008091F3218823E1F786E10E944D3B81E04F
:1077A0008093F42108958091F421882351F48091ED
:1077B000830B882321F081E08093050C02C00E9496
:1077C000A83B81E090E008950E94483B1092F4218C
:1077D0000E940A3B80913901826080933901809137
:1077E00077228823E9F1809194009091950020916F
:1077F00088223091892282179307A0F48091542225
:1078000090915522A0915622B09157228C57914EBB
:10781000AF4FBF4F8093542290935522A09356228E
:10782000B09357228091940090919500821B930B06
:10783000A0E0B0E040915422509155226091562230
:1078400070915722840F951FA61FB71F8093542253
:1078500090935522A0935622B093572210927722EC
:10786000809179228823E9F180919400909195008C
:1078700020918C2230918D2282179307A0F4809161
:107880005C2290915D22A0915E22B0915F228C5784
:10789000914EAF4FBF4F80935C2290935D22A09397
:1078A0005E22B0935F228091940090919500821B9C
:1078B000930BA0E0B0E040915C2250915D2260917A
:1078C0005E2270915F22840F951FA61FB71F8093C1
:1078D0005C2290935D22A0935E22B0935F2210926F
:1078E000792208958091050C882321F00E94A83BFD
:1078F0001092050C8091060C882321F00E94E43B35
:107900001092060C1092830B08950F931F93CF9340
:10791000DF93F82FE92FAB0181E08093830B009177
:1079200038221091392220913A2230913B220F5F68
:107930001F4F2F4F3F4F009338221093392220932F
:107940003A2230933B22862F8E5F87FF0CC08091B6
:10795000F1219091F22101969093F2218093F121EF
:10796000CFEFDFEF09C024E83BE0C9016F2F7E2F86
:107970000E94B464C0E0D0E00E94723CCE01DF916E
:10798000CF911F910F9108958091F421882399F050
:107990008091830B882321F40E942F3B882331F4AC
:1079A00081E08093060C81E090E008950E94E43B22
:1079B00080E090E0089580E090E008951F93CF93D9
:1079C000DF930F92CDB7DEB78FB789838091830B9A
:1079D000882331F5F8948091F421882351F0809127
:1079E000390181FD1BC00E942F3B8823B9F080E044
:1079F00003C00E94D33B81E0909147019E3010F07C
:107A000010E001C01FEF882311F00E94C43C16FF54
:107A100005C089818FBF81E090E004C089818FBF5C
:107A200080E090E00F90DF91CF911F9108958093B7
:107A3000820B08950E94033B8250813130F4E82F7D
:107A4000F0E0E25BFA4F8081089581E008950895A7
:107A50008FEF80934E018CE691E060EF44E022E0EE
:107A60000E94CE408CE290E06EE041E025E00E9472
:107A7000CE4080E880936F018091460180936D0134
:107A800084E491E060E245E021E00E94CE40089568
:107A9000CF93DF93CDEFD3E0CE010197F1F70E94B2
:107AA000BA40109268201092EA2010926C21109235
:107AB000672010926620E9E3F1E080818E7F808369
:107AC00080818D7F80838DE090E00197F1F7808148
:107AD0008160808382E491E06FE140E023E00E94D6
:107AE000CE402197F1F780915D0180915E010E9467
:107AF000283D80E395E060E070E00E94CA2B0E9480
:107B0000A83B81E090E0DF91CF9108958091070C30
:107B10000895CF93DF930F92CDB7DEB789830E948C
:107B2000483B29812093070C88E491E06FE140E015
:107B30000E94CE400F90DF91CF9108950E94893D21
:107B400086E00E944D3B0895FA0180936201909374
:107B5000630160936001709361013097C1F080818F
:107B600080936B01818180936A0182818093690196
:107B700083818093680184818093670185818093EC
:107B800066018681809365018781809364010895F1
:107B900080E395E00E94EC2B81E080935F20809150
:107BA00060209091612001969093612080936020E5
:107BB00081E090E00895CF93DF9350916720252FC7
:107BC00030E0F901EE0FFF1F3695322F222737954F
:107BD0002795E20FF31FE859FF4D4081442309F434
:107BE000F4C02091390121FDF0C02091F42122231D
:107BF00009F4EBC047FF23C0852F90E0FC01EE0F96
:107C0000FF1F9695982F882797958795E80FF91F5E
:107C1000E859FF4D10828091282290912922A0914D
:107C20002A22B0912B220196A11DB11D80932822FA
:107C300090932922A0932A22B0932B22C6C04330CE
:107C400018F5852F90E0FC01EE0FFF1F9695982FF9
:107C5000882797958795E80FF91FE859FF4D1082FF
:107C60008091242290912522A0912622B091272252
:107C70000196A11DB11D8093242290932522A093EB
:107C80002622B0932722A1C0C42FD0E022976C17E0
:107C90007D0718F5852F90E0FC01EE0FFF1F9695EC
:107CA000982F882797958795E80FF91FE859FF4D7A
:107CB00010828091202290912122A0912222B091C5
:107CC00023220196A11DB11D809320229093212291
:107CD000A0932222B093232278C0252F30E0B9014F
:107CE000660F771F3695322F222737952795620F1B
:107CF000731F67597F4D50E00E94B4642091672044
:107D0000822F90E0FC01EE0FFF1F9695982F882799
:107D100097958795E80FF91FE851FF4D8081809373
:107D20005820822F90E0FC01EE0FFF1F9695982FB0
:107D3000882797958795E80FF91FE859FF4D10821E
:107D40002F5F20936720233010F0109267208091DE
:107D5000672090E0FC01EE0FFF1F9695982F882773
:107D600097958795E80FF91FE859FF4D8081882383
:107D700011F00E94C83D60914701609359208091A5
:107D80005E20882311F0681710F460935E2084E071
:107D900070E00E9409326091582083E070E00E94F8
:107DA000093280913C2290913D22A0913E22B091D7
:107DB0003F220196A11DB11D80933C2290933D224C
:107DC000A0933E22B0933F2202C0C0E0D0E0CE019B
:107DD000DF91CF910895CF93DF93EC018881998152
:107DE000009729F024E08B3F920739F505C08BEF0F
:107DF00094E09983888325C0623819F510925F203A
:107E00000E948F310E94F03060E870E00E94DB3DFC
:107E10001816190644F40E94EB30E091C105F09168
:107E2000C2050995E4CF80915C2090915D20019678
:107E300090935D2080935C20DACF1982188283E0D2
:107E400001C081E0DF91CF91089591E09093830B81
:107E50000E94203B0E94723C08958091390181FD6F
:107E600007C085E491E06FE040E00E94C4400895BF
:107E700080E108950F931F93CF93DF93C82F21E0E4
:107E80002093830BD091F4218091390181FF16C09A
:107E900080919400909195009093892280938822FC
:107EA000209377222093F321809139018D7F809355
:107EB00039018091F3218823E1F7D0E00E94483B0B
:107EC0008091F421882309F441C08091792288238C
:107ED000E9F1809194009091950020918C2230914D
:107EE0008D2282179307A0F480915C2290915D22ED
:107EF000A0915E22B0915F228C57914EAF4FBF4F41
:107F000080935C2290935D22A0935E22B0935F22C7
:107F10008091940090919500821B930BA0E0B0E0BB
:107F200040915C2250915D2260915E2270915F22AF
:107F3000840F951FA61FB71F80935C2290935D222C
:107F4000A0935E22B0935F221092792289E10E9471
:107F50004D3B86E00E941432009751F00E942D3F65
:107F6000082F86E00E94143281500E94203B02C0FC
:107F700000E010E0809194009091950090938B2206
:107F800080938A2281E080937822F894809139014D
:107F9000826080933901809139018D7F809339010E
:107FA0006C2F6E5F84E89BE00E94FF407894809184
:107FB000EE219091EF2101969093EF218093EE2195
:107FC0000E94483B82E491E060EE45E00E94C4409C
:107FD000C82F86E00E941432009719F0802F0E946B
:107FE000203BDD2319F00E94A83B02C00E94E43B25
:107FF000809178228823E9F18091940090919500F6
:1080000020918A2230918B2282179307A0F48091CD
:10801000582290915922A0915A22B0915B228C57FC
:10802000914EAF4FBF4F8093582290935922A09307
:108030005A22B0935B228091940090919500821B0C
:10804000930BA0E0B0E040915822509159226091EA
:108050005A2270915B22840F951FA61FB71F809331
:10806000582290935922A0935A22B0935B221092E7
:1080700078228091F421882361F08091940090917E
:10808000950090938D2280938C2281E080937922B9
:1080900007C082E491E06FE140E023E00E94CE401F
:1080A0000E94723CC130E1F0C330A9F480913022CB
:1080B00090913122A0913222B09133220196A11DDC
:1080C000B11D8093302290933122A0933222B0933D
:1080D0003322C2E00AC0C53029F0C73031F404C0F1
:1080E000C0E003C0C3E001C0C1E08C2F90E0DF918D
:1080F000CF911F910F910895CF93DF93EB010E94D1
:10810000853C009729F4CE010E943A3F009751F038
:108110002091F1213091F2212F5F3F4F3093F221D6
:108120002093F121DF91CF910895CF93DF93809138
:10813000F421882321F40E94D33BC1E001C0C0E0B8
:108140000E94033B863111F0813119F4D09147012F
:1081500009C086E491E06FE140E00E94C440D82F5E
:10816000DD0FD80FCC2311F00E94C43C8D2FDF917E
:10817000CF9108951092090C1092080CEFE6F0E0F0
:108180008081806280830895FC018081862390E055
:1081900002C0959587954A95E2F70895F894FC01F9
:1081A0009081862F8095892330E002C0220F331FF3
:1081B0004A95E2F72623282B208378940895CF93BD
:1081C000DF93EC012196E0917B01DC01EC932E2FF3
:1081D000A0E8B1E03D9139932150E1F7E150F0E0A2
:1081E000E058FE4F2181FC01E058FF4F20838F575C
:1081F0009F4F21E0FC012083DF91CF910895FC0186
:1082000060938001A1E8B1E0615881918D936A1774
:10821000E1F708951F920F920FB60F920BB60F92CF
:1082200011242F933F934F935F936F937F938F937B
:108230009F93AF93BF93EF93FF93809147018093F8
:1082400059202091662030E0C901880F991F36958A
:10825000322F222737952795820F931F88599F4DDC
:108260000E94DF40809166208F5F8093662083307C
:1082700010F0109266200E94C83DFF91EF91BF91CF
:10828000AF919F918F917F916F915F914F913F91AE
:108290002F910F900BBE0F900FBE0F901F9018954F
:1082A0001F920F920FB60F9211240F900FBE0F90D6
:1082B0001F9018951F920F920FB60F9211240F90D6
:1082C0000FBE0F901F9018951F920F920FB60F922E
:1082D00011240F900FBE0F901F9018951F920F92B0
:1082E0000FB60F9211241092F3210F900FBE0F9032
:1082F0001F9018951F920F920FB60F921124109293
:10830000F3210F900FBE0F901F9018951F920F92A0
:108310000FB60F9211248F9381E080935F208F918D
:108320000F900FBE0F901F9018951F920F920FB6CF
:108330000F9211241092F3210F900FBE0F901F90F7
:1083400018951F920F920FB60F9211248F939F933F
:108350008091080C9091090C01969093090C8093E0
:10836000080C9F918F910F900FBE0F901F90189542
:108370000F931F93CF93DF938091FC219091FD2168
:10838000A091FE21B091FF210196A11DB11D809306
:10839000FC219093FD21A093FE21B093FF210E9428
:1083A00050448C018AE09CE00E94942C08C0EA8131
:1083B000FB81309709F00995CE010E943A2DEC011E
:1083C0000097A9F70115110519F0C8010E94022AAA
:1083D000DF91CF911F910F9108950E94A64A0E94AC
:1083E0008F310E94694282EA95E09093F721809351
:1083F000F6210E944D4482E090E060E074E040E0AD
:108400005EE12FEF31E00E940E440895CF92DF929B
:10841000EF92FF920F931F93CF93DF936C018B0129
:108420007A018AE09CE00E94942C09C0EC81FD81D5
:10843000309711F0C8010995CE010E943A2DEC0148
:108440000097A1F7C601B801A7010E940C2ADF918D
:10845000CF911F910F91FF90EF90DF90CF900895F3
:10846000BC018AE09CE00E94032D0895BC018AE0D3
:108470009CE00E94CE2C0895CF93DF93EC01809175
:10848000F8219091F921A091FA21B091FB21019658
:10849000A11DB11D8093F8219093F921A093FA2199
:1084A000B093FB21CE010E946344009769F00E94C3
:1084B0000A31E091A605F091A70586E092E4BE019D
:1084C000099581E090E002C080E090E0DF91CF91DB
:1084D00008958CE09CE00E94902C08950F93CF9318
:1084E000DF93EC017B836A8318865F834E838CE085
:1084F0009CE0BE010E94032DE0910E0CF0910F0C48
:10850000309749F04C815D818A819B81688520E0AC
:1085100030E001E00995DF91CF910F910895BC0102
:108520008CE09CE00E94CE2C08950F93DC011896FD
:108530001C921897E0910E0CF0910F0C309759F0A7
:1085400012968D919C91139760E040E050E020E0FE
:1085500030E000E009950F9108950F93DC01AB0125
:1085600014962D913C91159781E018968C9318974D
:1085700015967C936E931497E0910E0CF0910F0C6E
:10858000309739F012968D919C91139761E000E03D
:1085900009950F9108950F93DC01E0910E0CF09175
:1085A0000F0C309769F014962D913C911597129607
:1085B0008D919C91139718966C91A90101E00995F2
:1085C0000F910895E091100CF091110C309709F083
:1085D000099508959093110C8093100C0895909331
:1085E0000F0C80930E0C08958CE09CE00E94942C5C
:1085F0000895EF92FF920F931F93CF93DF938C0117
:10860000EB017A018CE09CE00E94942C15C0DC0107
:1086100012962D913C9113972C173D0759F41696FD
:10862000ED91FC911797309749F0B801AE01970191
:10863000099504C00E943A2D009749F7DF91CF9128
:108640001F910F91FF90EF9008950895AF92BF9200
:10865000CF92DF92EF92FF920F931F93CF93DF930E
:1086600000D0CDB7DEB75B010E94F030FC01E080A6
:10867000F180FA82E982FCE0EF16F10418F400E0E0
:1086800010E02DC000D000D08AE695E0EDB7FEB72F
:1086900092838183F482E3820E9433650F900F906E
:1086A0000F900F901FC00E94F030F801EE0FFF1FD7
:1086B000EE0FFF1FE80FF91FC280D3800E94F03039
:1086C0000F5F1F4FF801EE0FFF1FEE0FFF1FE80FA8
:1086D000F91F40815181C501B6010E94F9420E1572
:1086E0001F0509F70F900F90DF91CF911F910F9108
:1086F000FF90EF90DF90CF90BF90AF900895CF9311
:10870000DF93CDE2DCE06091430C7091440CCE012C
:1087100042EA53E420E030E00E9403490E94A34A69
:108720006091430C7091440C0E947C61BC01CE01AD
:10873000409746EC53E420E030E00E940349DF918B
:10874000CF9108958091430C9091440C2091410C5D
:108750003091420C880F991F2817390708F4C90176
:108760009093440C8093430C0E947F4308950F9391
:10877000013051F480913D0C90913E0C9093440C4B
:108780008093430C0E947F430F910895CF93DF9312
:108790000E948F310E94F030EC01198218820E94F1
:1087A000F44220C012962D913C911397FC01EE0FDC
:1087B000FF1FEE0FFF1FEC0FFD1F33832283149664
:1087C0002D913C9115970196FC01EE0FFF1FEE0FC6
:1087D000FF1FEC0FFD1F3183208399838883CD0118
:1087E0000E943A2DDC0188819981109729F0189612
:1087F0002C9118972223B1F6880F991F880F991F83
:1088000002960E94EB3088819981009721F082E1E5
:108810009CE00E94D529DF91CF910895EF92FF92BD
:108820000F931F93CF93DF93FC018B017A01E90132
:1088300082E19CE0BF0147E855E00E94B729109310
:108840003E0C00933D0CF092400CE0923F0CD09314
:10885000420CC093410C87EB93E40E94EF42DF91FE
:10886000CF911F910F91FF90EF900895CF93DF93D9
:10887000CDE2DCE0CE010E948A49CE0140970E9401
:108880008A49CE014B970E94D229DF91CF9108955A
:108890008091430C9091440C08950E94182A0895E9
:1088A000CF93DF93E0918B05F0918C050995EC0156
:1088B000009729F06A817B8181E00E940932CE0114
:1088C000DF91CF9108950F931F93CF93DF93EC0126
:1088D000E0918D05F0918E0509958C016A817B816F
:1088E00081E00E94093281E090E00115110511F448
:1088F00080E090E0DF91CF911F910F910895E0917A
:108900008F05F0919005099508959C0180E090E015
:1089100005C0F90131974081840F911D2E5F3F4FB3
:10892000F901329740814423A1F70895FC01308179
:1089300020E0818190E0822B932B02C0880F991F49
:108940006A95E2F7892F9927FA01EF56FA4F2081AD
:1089500030E08223932328E030E0241B350B02C053
:10896000969587952A95E2F708956F927F928F9258
:108970009F92AF92BF92CF92DF92EF92FF920F93AE
:108980001F93CF93DF935C013B018A01690128307B
:10899000310544F4CB01BA01A9010E949644F501C6
:1089A00080834EC0790173E0F594E7947A95E1F7FE
:1089B0004115510521F04501C0E0D0E005C0F301AB
:1089C000D50180E090E021C0C3018C0F9D1FB8014C
:1089D00048E050E00E949644F40181934F012196B3
:1089E000CE15DF058CF3C701F7FE02C080E090E0F2
:1089F000A601477050704115510511F1E501C80FEE
:108A0000D91F860D971DB80118C021912D9301968D
:108A10008E159F05D4F3C701F7FE02C080E090E0F9
:108A2000A601477050704115510551F0E501C80F7E
:108A3000D91F860D971D60E070E00E9496448883E0
:108A4000DF91CF911F910F91FF90EF90DF90CF902A
:108A5000BF90AF909F908F907F906F9008958F926E
:108A60009F92AF92BF92CF92DF92EF92FF920F93BD
:108A70001F93CF93DF9300D000D0CDB7DEB70E9415
:108A8000F0308C0182E090E00E94CD30009709F434
:108A90005FC0F801918180E02081820F911D0E94CA
:108AA0002C2A7C01009709F455C00E94F0304C013B
:108AB000F7018681482F46954695469550E090E00F
:108AC0008770907021E030E0009711F420E030E0F2
:108AD000CA01820F931F0E94CD300097C9F1F701A0
:108AE00004811581CC24DD242EC0F801A180BB2493
:108AF000B601A3E075956795AA95E1F7680D791D14
:108B0000A60147705070883168F0CE010396950138
:108B10000E94B544F8018081BE016D5F7F4F0E94C5
:108B20001D320DC01A821982CE01019695010E9454
:108B3000B54469817A81F80180810E940932CA0CAA
:108B4000DB1C0E5F1F4FF8018081882371F602C085
:108B5000EE24FF24C7010F900F900F900F90DF912C
:108B6000CF911F910F91FF90EF90DF90CF90BF902A
:108B7000AF909F908F900895FC0150E080E190E0CD
:108B8000861B970B821B930B02C0440F551F8A95BF
:108B9000E2F78081852B80838181842B81830895F6
:108BA0006F927F928F929F92AF92BF92CF92DF92FD
:108BB000EF92FF920F931F93CF93DF933C016B01D2
:108BC0005A0179012830310524F4C301FA014081AA
:108BD00059C08901B3E015950795BA95E1F761157C
:108BE000710521F04A01C0E0D0E005C0FA01D301CF
:108BF00080E090E023C0F40141914F01C3018C0F4C
:108C00009D1FB60128E030E00E94BC452196C017A8
:108C1000D1078CF3980117FF02C020E030E0D701A4
:108C2000A770B070109781F1F501E20FF31F40813A
:108C300050E0C6018A1B9B0B089619C021912D9309
:108C4000019680179107D4F3980117FF02C020E026
:108C500030E0D701A770B0701097B1F0F501E20FC6
:108C6000F31F408150E088E090E08A1B9B0B02C01C
:108C7000559547958A95E2F7C301820F931F60E0EF
:108C800070E09D010E94BC45DF91CF911F910F9133
:108C9000FF90EF90DF90CF90BF90AF909F908F901C
:108CA0007F906F9008956F927F928F929F92AF9274
:108CB000BF92CF92DF92EF92FF920F931F93CF93C9
:108CC000DF9300D0CDB7DEB77C01DC0116968C9126
:108CD0001697282F26952695269530E090E08770E8
:108CE000907001E010E0009711F400E010E0020F36
:108CF000131FC80102960E945531009709F451C014
:108D00000E94F730FC01D70112968C911297808354
:108D100013968C9181830E94F73032E0632E712C80
:108D2000680E791EC30160E070E0A8010E94BD6476
:108D3000F701E480F580CC24DD242CC0D701119606
:108D4000AC901197BB24860193E0159507959A95F1
:108D5000E1F7060D171D27E0822E912C8C209D2017
:108D6000883130F00E942732AC01C801B40109C03B
:108D70000E9414329A838983C801B401AE014F5F07
:108D80005F4F95010E94D045CA0CDB1CE2E0F0E089
:108D9000EE0EFF1ED7018C91882381F681E090E0D2
:108DA00002C080E090E00F900F90DF91CF911F9173
:108DB0000F91FF90EF90DF90CF90BF90AF909F907A
:108DC0008F907F906F900895E091BF05F091C0055E
:108DD00009950895E0916805F09169050995089550
:108DE000E091C305F091C40509950895E091C5058A
:108DF000F091C6050995089580E090E008950895E2
:108E0000E0914A05F0914B050995089580E090E0C6
:108E100008950F931F93CF93DF93CDB7DEB7E097FD
:108E20000FB6F894DEBF0FBECDBF0E9440318C015B
:108E30000E94F030602FAE014F5F5F4F0E943350B1
:108E4000882309F446C088A99801281B3109C90163
:108E50000E94CD300097E9F12E81222379F18A8595
:108E60009B853BEA8D3C930721F03FEF8F3F9307B3
:108E700081F5223069F088E090E00197E1E0F0E0D0
:108E8000EC0FFD1FE80FF91F23852F3F21F007C0CE
:108E900082E090E0F2CF181619067CF30FC089E14A
:108EA000BE01645F7F4F0E941D3289E10E9427321C
:108EB00065E070E20E946F29009759F088E1BE01D9
:108EC0006A5E7F4F0E941D32E091A805F091A905CE
:108ED0000995E0960FB6F894DEBF0FBECDBFDF91C7
:108EE000CF911F910F910895AF92BF92CF92DF92D1
:108EF000EF92FF920F931F93CF93DF93CDB7DEB71F
:108F0000E0970FB6F894DEBF0FBECDBF5C016B01DA
:108F1000FE01319680E3DF011D928A95E9F781E039
:108F200089838CE00E9414328C831D821F82809181
:108F3000470C89878F5F8093470C03E008878DEC8F
:108F40009BEA9B878A8789E10E94273265EC74E05F
:108F50000E946F29009731F082E08E838FEF8C871B
:108F60008D8709C089E10E942732BC01CE010C9691
:108F70000E9466290E838DEC9BEA9D8B8C8BCE0123
:108F8000469665E070E20E9466290E94F0309FA735
:108F90008EA70E94403188ABCE0101960E94444FBB
:108FA000082F90E00E945531009749F10E94F73058
:108FB000BC01CE010196402F0E94624F00914005F6
:108FC000109141050E94F7307C010E944A31BC019A
:108FD000C701F8010995A114B10489F0009721F0A7
:108FE0008130910561F404C0C60160E070E003C007
:108FF000C60164E070E041E050E0F5010995E096BB
:109000000FB6F894DEBF0FBECDBFDF91CF911F9199
:109010000F91FF90EF90DF90CF90BF90AF900895A9
:109020000E94A34A8093470CE0914A05F0914B05BA
:1090300009950895009731F0E0914A05F0914B05AC
:1090400009950895E0914C05F0914D050995089515
:10905000CF93DF93EC0104C060E070E00E94CA2B64
:10906000899199910097C1F7DF91CF910895CF939E
:10907000DF93EC0102C00E94112B89919991009716
:10908000D1F7DF91CF910895CF93DF93EC017B83EC
:109090006A830E94443999838883DF91CF91089530
:1090A000FC018081918122813381820F931F918302
:1090B00080830895CF93DF93EC010E944439998314
:1090C0008883DF91CF910895CF93DF93EC010E94C5
:1090D000443928813981AC01421B530B9A012F5F1F
:1090E0003F4F81E090E04A815B814217530710F0C7
:1090F00080E090E0DF91CF910895CF93DF93FC0162
:10910000C281D38180819181C80FD91F0E944439C7
:109110009E01281B390BC901DF91CF910895EF9271
:10912000FF920F931F93CF93DF937C018A01FC0181
:1091300080819181009729F08B34910509F049C015
:109140001AC089E49CE00E94942CEC0109C06C8157
:109150007D81CE0102960E942C2E0990D881C02DCF
:109160002097A9F781E08093480C8BE490E0F70109
:109170009183808333C0683889F589E49CE00E943C
:10918000942CEC0123C0CE01029608171907D9F4DC
:1091900089E49CE0BE010E94CE2C0091D009109180
:1091A000D1098A859B859093D1098093D009EC855C
:1091B000FD85309719F08E859F8509951093D1090B
:1091C0000093D009D2CF0990D881C02D2097D9F62D
:1091D000CCCFF7011182108283E001C081E0DF91E2
:1091E000CF911F910F91FF90EF9008951092480C2E
:1091F00089E49CE00E94902C88ED95E060E070E0AE
:109200000E94CA2B08950F931F93CF93DF93EC0115
:109210000091D0091091D1091B870A875D874C877F
:109220003F872E878091480C882379F088ED95E060
:109230009093D1098093D009CE0102960E942C2EE2
:109240001093D1090093D00902C07D836C8389E417
:109250009CE0BE010E94CE2C89E49CE0BE010E94ED
:10926000032DDF91CF911F910F9108950F931F93BD
:10927000CF93DF93EC018091480C882391F000910B
:10928000D0091091D10988ED95E09093D109809390
:10929000D009CE0102960E94372E1093D109009377
:1092A000D00989E49CE0BE010E94CE2C89E49CE0B8
:1092B000BE010E94032DDF91CF911F910F91089560
:1092C0000F931F93CF93DF93EC018091480C882379
:1092D00091F00091D0091091D10988ED95E090931B
:1092E000D1098093D009CE0102960E94422E10939C
:1092F000D1090093D00989E49CE0BE010E94CE2CE4
:1093000089E49CE0BE010E94032DDF91CF911F9163
:109310000F910895CF93DF93EC018091480C88233F
:1093200029F0CE0102960E94892E04C01F821E825F
:109330001986188689E49CE0BE010E94CE2CDF913C
:10934000CF910895CF93DF93EC018091480C88234F
:1093500029F0CE0102960E94572E12C089E49CE0AB
:109360000E94942C06C08C179D0741F0FC0180815F
:1093700091810097C1F781E090E002C080E090E029
:10938000DF91CF910895CF93DF93EEE7F2E2C0E44F
:10939000D2E2A2E7B2E211921192199219921992B5
:1093A00019921D9282E2E639F807A9F7DF91CF9171
:1093B00008950F931F93CF93DF93FC01EE58FD4D5B
:1093C00020818C01000F111F000F111F222311F1AA
:1093D0002091940030919500E801C05CDD4DFC01C6
:1093E000EE0FFF1FE258FD4D80819181A901481BBE
:1093F000590BCA01A0E0B0E0488159816A817B81A4
:10940000840F951FA61FB71F88839983AA83BB83E8
:1094100031832083F801E05CFD4D608171818281A0
:109420009381DF91CF911F910F91089560E070E0DB
:1094300080E090E00895FC01EE0FFF1FEE0FFF1F8C
:10944000E05CFD4D40835183628373830895EF9206
:10945000FF920F931F93CF93DF93B2E7EB2EB2E20D
:10946000FB2EE0E4F2E2CEE7D2E220E030E0D701EA
:109470008D917D018823C9F0009194001091950091
:1094800088819981A801481B590B60E070E08081B8
:109490009181A281B381840F951FA61FB71F80837E
:1094A0009183A283B383198308832F5F3F4F349640
:1094B00022962C303105D9F6DF91CF911F910F9173
:1094C000FF90EF9008950E94C64E08950F931F934A
:1094D000FC0180914B0C90914C0C338322831583BB
:1094E000048371836083F0934C0CE0934B0C0097E2
:1094F00019F4CB010E94E04E80E090E01F910F91A3
:10950000089580914B0C90914C0C0097C1F01092F3
:109510004C0C10924B0CDC0114966D917C911597BC
:109520001296ED91FC9113970995E0914B0CF091F7
:109530004C0C309721F0808191810E94E04E08957B
:109540000E94566208950E945162089582EE95E04D
:109550000E94022C8AEE95E00E94022C0895CF937F
:10956000DF930E94FD300097A9F08AEE95E00E94FB
:10957000212CEC01009729F10E94403199838883C6
:109580000E943B319B838A83CE0104960E947730F0
:109590008CAB17C082EE95E00E94212CEC01009765
:1095A00071F002960E94893099838883BE016E54BF
:1095B0007F4FCE018E579F4F0E94E73102C0C0E01F
:1095C000D0E0CE01DF91CF910895BC016E547F4F62
:1095D0008E579F4F0E94E7310895CF93DF93EC01A0
:1095E00082EE95E0BE010E94722C009719F082EE87
:1095F00095E009C08AEE95E0BE010E94722C0097AA
:1096000029F08AEE95E0BE010E944C2CDF91CF91AB
:109610000895CF93DF93EC0182EE95E0BE010E94A6
:10962000722C009779F068817981CE0102960E94B0
:10963000B831BE016E547F4FCE018E579F4F0E94AE
:10964000F8311CC08AEE95E0BE010E94722C009792
:10965000A9F00E948F31688179818A819B810E9463
:10966000B8318CA990E00E9455310E94F7304CA986
:10967000BE016C5F7F4F50E00E94B464DF91CF91D8
:109680000895CF93DF93EC0182EE95E0BE010E9436
:10969000722C009719F0CE0102960CC08AEE95E06C
:1096A000BE010E94722C009719F08A819B8102C032
:1096B00080E090E0DF91CF910895FC01808191815D
:1096C000089570E06F5B7F4F660F771F680F791FFB
:1096D000CB010895E62FF0E0EF5BFF4FEE0FFF1F89
:1096E000E80FF91F808191810895089586EA92E13B
:1096F0000E94572E009721F086EA92E10E94422EA6
:109700000895E0919112F0919212309711F009951D
:10971000089580E00895EF92FF920F931F93CF93E7
:10972000DF937C018A01FC0180819181009731F0F7
:10973000F3E08C309F0709F0FFC02BC080E0E82FDA
:10974000F0E0EE0FFF1FEE0FFF1FEC56FD4E1182F3
:1097500010828F5F843098F3809393128091D009A8
:109760009091D109E4E9F2E1918B808B0E940A2B60
:109770008093962286EA92E160E470E00E942C2EAB
:109780000E94A8518CE093E0F7019183808381E0EF
:10979000D7C0623009F4B2C0633030F4662309F4F4
:1097A00082C0613079F795C0673819F0683851F791
:1097B0003AC01092AE12C4E9D2E113C08A819B81F3
:1097C0008017910741F4888199810E94DE521982A5
:1097D00018821B821A8224968091AE128F5F80932A
:1097E000AE128091AE12843048F3E6EAF7E2848D3F
:1097F000958D8017910719F4158E148E118EB096E1
:1098000028E2E632F20798F3ECE3F8E281859285EC
:109810008017910711F4158214823D9688E2EE3B81
:10982000F807A0F3AFCFE2E1463A5E0709F0AACF0E
:10983000CA010E94572E009709F4A4CF1092AE12CD
:109840002DC0F0E035E0EE0FFF1F3A95E1F7EA5545
:10985000F84D818D8823E9F086EA92E10E94422E3C
:109860008091AE1290E025E0880F991F2A95E1F7CC
:109870008A55984D9093A5278093A42782E00E9453
:1098800012538091972290919822009711F00E9494
:10989000814B8091AE128F5F8093AE12E091AE1239
:1098A000E43078F26FCF4115510509F46BCF509336
:1098B000A5274093A42783E00E941253809197220A
:1098C00090919822009711F00E94814B0E94764B54
:1098D00059CF4115510509F455CF5093A127409315
:1098E000A02785E00E9412538091972290919822A0
:1098F000009709F447CF0E94814B44CF8091972273
:1099000090919822009709F43DCF8091A82286304B
:1099100031F48091C02281FF02C00E94764B81E029
:109920000E9412538091972290919822009709F4F7
:1099300029CF0E94AE4D26CFF7011182108283E01D
:10994000DF91CF911F910F91FF90EF900895909329
:1099500092128093911208959C014091D0095091E8
:10996000D10960E0E4E9F2E114C0808191818217BD
:10997000930769F4828193818417950741F460937A
:10998000AF1211821082C9010E94DE5208953496EE
:109990006F5F643050F36093AF12089540E0E4E9E4
:1099A000F2E116C0542F5F5F20813181211531050E
:1099B00069F44093B012918380832091D009309153
:1099C000D109338322830E94F85208953496452F9B
:1099D000443040F34093B0120895FC018091D009C7
:1099E0009091D109958F848F778F668F0895FC01B0
:1099F0008091D0099091D10992878187748763877C
:109A00000895CF93DF93EA010E946A52009749F0CC
:109A10002091D0093091D109FC0132872187D48768
:109A2000C387DF91CF9108950F931F93CF93DF9357
:109A300000D000D0CDB7DEB78C01AB018FEF8983AA
:109A40008A838B838C83CE010196B8010E94014DDD
:109A5000009719F0FC01158304830F900F900F906D
:109A60000F90DF91CF911F910F9108958FEF95E0A7
:109A700062E040E050E00E94BB2B109298221092CE
:109A800097220895AC018FEF95E061E00E94982B3A
:109A90000895AC018FEF95E060E00E94982B089547
:109AA0000F931F93CF93DF938A010E94DE51EC0145
:109AB000009759F08091D0099091D1099D8F8C8F9A
:109AC0001F8F0E8FCE010E94494DCE01DF91CF91A5
:109AD0001F910F910895CF93DF93A091A427B09188
:109AE000A527109719F0ED016C9605C0C091A0272D
:109AF000D091A127299680919F2786FF22C010929E
:109B0000B11240E0E4E9F2E116C08081918114963F
:109B10002D913C9115978217930759F48281938177
:109B2000009739F04093B112998388831B821A827F
:109B300006C034964F5F443040F34093B1120E9408
:109B4000764B88819981009731F04A815B816091E1
:109B500096220E94BB2BDF91CF9108950F931F9304
:109B6000CF93DF938091A822863009F074C0809152
:109B700097229091982225E08030920709F06BC0DF
:109B8000C4E9D2E0D0939822C093972202E00093D8
:109B9000A12214E91093A2221092C4221092C3228F
:109BA0000E94A051809590959093C4228093C322E7
:109BB0001092AA221092A9220E948F51809590950E
:109BC0009093AA228093A9220E94814BD09398223D
:109BD000C09397220093A1221093A2229091A227D2
:109BE0008091A327E92FF82FDF01A459BD4F8CE600
:109BF00092E00D9001920197E1F787EB92E26CE61B
:109C000072E00E944C5180919B228093B7228091F8
:109C10009C228093B82280919D228093B9228091CA
:109C20009E228093BA221092C4221092C3220E94D4
:109C3000A051809590959093C4228093C322109256
:109C4000AA221092A9220E948F51809590959093FC
:109C5000AA228093A9220E94814BDF91CF911F916C
:109C60000F910895FC0120E030E080E0A8E111C0F0
:109C7000419198E0542F5827B52FB17050FD8A2795
:109C80008695B13009F480684695915099F72F5F19
:109C90003F4F2617370761F708951F920F920FB6AF
:109CA0000F920BB60F9211242F933F934F935F9314
:109CB0006F937F938F939F93AF93BF93EF93FF9394
:109CC00080919400909195009093832280938222BA
:109CD00081E08093742280917100807D8093710077
:109CE0000E94814A809174228823E9F18091940036
:109CF00090919500209182223091832282179307C0
:109D0000A0F48091482290914922A0914A22B091DA
:109D10004B228C57914EAF4FBF4F80934822909368
:109D20004922A0934A22B0934B22809194009091B3
:109D30009500821B930BA0E0B0E040914822509127
:109D4000492260914A2270914B22840F951FA61FD1
:109D5000B71F8093482290934922A0934A22B09340
:109D60004B2210927422FF91EF91BF91AF919F917E
:109D70008F917F916F915F914F913F912F910F90B4
:109D80000BBE0F900FBE0F901F9018959FB7F894C1
:109D9000E1E7F0E08081807D808388B38F6288BBBB
:109DA00010929000E1E9F0E010821092920010927F
:109DB0009500109294008081856080839FBF0895F4
:109DC0002FB7F894909399008093980088B38F628E
:109DD00088BBE1E7F0E08081826080832FBF089537
:109DE000CF93DF93FC01DB0185E0EB0119928A95AB
:109DF000E9F7858190E083709070009711F082E020
:109E00008C93878190E083709070009721F082E0BE
:109E100012968C931297858190E0837090700097D2
:109E200099F0878190E083709070009769F02389A2
:109E30003489818592852817390731F481E084833C
:109E400012961C92129701C01482C581C370C25031
:109E5000C23028F4D0E0C75FD94F888101C080E0CC
:109E600011968C931197E781E370E250E23028F469
:109E7000F0E0E75FF94F808101C080E013968C939A
:109E80001397DF91CF910895CF93DF9300D000D047
:109E90000F92CDB7DEB7BE016F5F7F4F0E94F04ECD
:109EA00089819A81890F8D5F9B81890F9C81890FA0
:109EB0009D81890F0F900F900F900F900F90DF9161
:109EC000CF910895DF92EF92FF920F931F93CF935C
:109ED000DF9300D000D000D0CDB7DEB78C017B017E
:109EE000BE016F5F7F4F4E830E94F04E79816A8181
:109EF000AB81BC81872F90E00396860F911D8A0F5E
:109F0000911D8B0F911D2D81820F911D4E8150E06F
:109F1000481759070CF498C0F801218130E02170EE
:109F2000307083E0220F331F8A95E1F7828190E041
:109F30008170907034E0880F991F3A95E1F7822B79
:109F400090819770892B438150E04170507095E06B
:109F5000440F551F9A95E1F7842B448150E04170DE
:109F6000507026E0440F551F2A95E1F7842BF70126
:109F70008083F801258130E023703070220F331F79
:109F8000220F331F868190E08370907054E0880F19
:109F9000991F5A95E1F7822B97819295990F990F06
:109FA000907C982BF7019183F8018085F7018283DB
:109FB000723051F4F8018185F7018383F8018285BD
:109FC000F701848355E001C053E040E080E090E079
:109FD0009801260F311D09C0F901E80FF91FD3843C
:109FE000F701E70FF11DD0824F5F742F750F0197B6
:109FF000461791F7972FA23089F49701270F311D4B
:10A00000F8018389F9018083872F8F5F9701280FDB
:10A01000311DF8018489F90180839E5F40E020E0D2
:10A0200030E00B0F111D09C0F801E20FF31F558935
:10A03000F701E80FF11D50834F5F842F890F2150E6
:10A0400030404B1789F701C080E026960FB6F89490
:10A05000DEBF0FBECDBFDF91CF911F910F91FF905B
:10A06000EF90DF900895BF92CF92DF92EF92FF9230
:10A070000F931F93CF93DF937C01B62EEA0182E00A
:10A08000861708F0AEC0F7018081D82ED294D694FE
:10A09000D69463E0D622F1E0DF22F7019181292FE7
:10A0A000269526952370C92EC294C694C69473E053
:10A0B000C722382F37703883382F36953695369526
:10A0C00031703983382F329531703A838295869575
:10A0D00081708B83DC822D83892F829583708E83A0
:10A0E000CF8282818887222369F13381948180E045
:10A0F000830F911D9A878987223079F4CA010B96C4
:10A1000065EC74E00E946629F70186818B87858162
:10A110008C878701095F1F4F20C087010B5F1F4F8E
:10A120002330D9F4F7013D96DA0180E092911B9635
:10A130009C931B978F5F11968830C1F78701035F4F
:10A140001F4F0BC087010D5F1F4FCA010B9665ECB7
:10A1500074E00E9466291A861986CC2089F1DD20D8
:10A1600059F4F8012081918180E0820F911D9C8B30
:10A170008B8B0E5F1F4F04C089859A859C8B8B8BC0
:10A18000F2E0CF1671F4CE01459665EC74E00E94C2
:10A190006629F80181818D8B80818E8B0E5F1F4F28
:10A1A00017C0F3E0CF16A1F4085F1F4FD801FE01DE
:10A1B00080E09E91958B8F5F31968830D1F708C0F3
:10A1C000CE01459665EC74E00E9466291C8A1B8AC4
:10A1D000802F8E199B2D981B9FA71EA70DA7B81621
:10A1E00008F480E0DF91CF911F910F91FF90EF90E5
:10A1F000DF90CF90BF9008959C0141505040460F92
:10A20000571FFB010EC0B081A0E08181BD01680F26
:10A21000711D260F371F2617370710F42F5F3F4F8A
:10A220003296E417F50778F3E417F50749F49081BF
:10A2300080E0280F391F2817390710F42F5F3F4F90
:10A24000C9010895CF93DF93C091A222D0E0649713
:10A250003091A12220E0C20FD31F9E01280F311D93
:10A26000C9016BEA72E248E050E00E94FC5063EBE7
:10A2700072E2AE010E94FC50009721F098278927D6
:10A28000982702C08FEF9FEFDF91CF9108959093B1
:10A29000B9128093B8120895FC014381460F409390
:10A2A0009E22872F99272281280F20939D22A1810A
:10A2B000A0939C22508150939B2230E028173907AD
:10A2C00048F48A2F8F5F80939C22882319F45F5F64
:10A2D00050939B22842F90E070708617970798F414
:10A2E00080919D228F5F80939D22882361F48091CD
:10A2F0009C228F5F80939C22882329F480919B224B
:10A300008F5F80939B2208959C01AB0180E090E0D9
:10A31000B9010E94FC50982789279827089580E06A
:10A3200090E06FE972E244E150E00E94FC50009737
:10A3300021F098278927982708958FEF9FEF089598
:10A3400086E00E942251089581E10E9422510895E1
:10A3500080E0E82FF0E0EE0FFF1FEA5DF74D11827D
:10A3600010828F5F8430A8F380E0E82FF0E035E0C2
:10A37000EE0FFF1F3A95E1F7EA55F84D118E8F5F0A
:10A38000843098F380E094E09093BC128093BB12E9
:10A3900040E08DE090E0242F30E0289FF001299FDD
:10A3A000F00D389FF00D1124E45CF74D15821482F6
:10A3B0004F5F4A3080F34093BA120895CF93DF93F2
:10A3C000EC012091BB123091BC122F5F3F4F8DE703
:10A3D0002030380710F020E030E1522F432FA0E06A
:10A3E00012C0EA2FF0E0B5E0EE0FFF1FBA95E1F7DB
:10A3F000EA55F84D818D882329F084819581841751
:10A40000950719F3AF5FA43061F73093BC12209326
:10A41000BB121092BA1280E0E0E0F0E01EC0A82F5C
:10A42000B0E055E0AA0FBB1F5A95E1F7AA55B84D09
:10A4300059969C915997992321F48093BA12FD0162
:10A4400010C0973049F4309731F05A962C915A97B2
:10A45000928D921708F4FD018F5F843000F3809392
:10A46000BA12309799F182E0818F8091BD12848772
:10A470008091BE1285878091BF1286878091C0121D
:10A48000878788ED94E0938B828B958B848B81E01A
:10A4900090E0918B808B138E81E0828F83E0808FA0
:10A4A000168A80E1878B8091BB129091BC1298270D
:10A4B0008927982795838483778366838881998108
:10A4C000AA81BB8180839183A283B383CF01DF9173
:10A4D000CF9108950F931F93CF93DF93EC018B01DE
:10A4E0002091BB123091BC126DE070E02F5F3F4FA6
:10A4F0008DE72030380710F020E030E1522F432F55
:10A50000A0E011C08A2F90E0869FF001879FF00D98
:10A51000969FF00D1124E45CF74D84819581AF5F27
:10A520008417950719F3AA3069F73093BC1220936A
:10A53000BB1240E02DE030E018C0542F5F5F842F45
:10A5400090E0829FF001839FF00D929FF00D112407
:10A55000E45CF74D84819581009731F44093BA1201
:10A560009F01309749F424C0452F4A3030F340937F
:10A57000BA1220E030E01CC08091BB129091BC1256
:10A5800098278927982795838483178306832097A4
:10A5900029F4108211821282138208C08881998165
:10A5A000AA81BB8180839183A283B38380E4808767
:10A5B000C901DF91CF911F910F91089540E013C021
:10A5C000E42FF0E0542F5F5FEE0FFF1FEA5DF74DC1
:10A5D000208131812817390729F44093BA1211825A
:10A5E00010820895452F443058F34093BA120895CD
:10A5F00040E013C0E42FF0E0542F5F5FEE0FFF1F29
:10A60000EA5DF74D208131812115310529F4409310
:10A61000BA12918380830895452F443058F34093B4
:10A62000BA120895AF92BF92CF92DF92EF92FF924B
:10A630000F931F93CF93DF93C091A427D091A527A9
:10A64000843009F4F1C127EC32E23093A327209340
:10A65000A22730939A2220939922833071F4898D16
:10A6600090E08F7090708330910509F074C08889F4
:10A670009989009709F031C78DC0823009F08EC0EA
:10A680008091C0128F5F8093C012882399F48091CB
:10A69000BF128F5F8093BF12882361F48091BE1236
:10A6A0008F5F8093BE12882329F48091BD128F5F43
:10A6B0008093BD12109298221092972210923B28FC
:10A6C00010923A28898D873011F0853041F48A8DB7
:10A6D0008F5F8A8F843109F000C7198EFEC68823E8
:10A6E00009F4FBC6288939892115310509F44EC0C2
:10A6F0009A8D292F21502A8F992309F0EEC69B8D20
:10A70000983031F0282F2150223048F4953039F418
:10A71000198E80E880939F270E946B4D94C59530D9
:10A7200048F423E030E0092E02C0220F331F0A94C0
:10A73000E2F701C020E32A8F9F5F9B8F90E08F702C
:10A74000907083309105E1F0843091054CF48130B4
:10A75000910509F469C38230910509F0BEC60DC0A8
:10A760008630910509F47EC58830910509F47AC5D3
:10A770008430910509F0B1C675C51092C02257C347
:10A7800084E080939F270E946B4D92C58F70833029
:10A7900009F0A3C688E080939F274AC5853019F544
:10A7A000E091A027F091A12784819581009709F479
:10A7B00094C61092A5271092A4272C5030403093B5
:10A7C000A3272093A22730939A22209399221092B4
:10A7D0003B2810923A28109298221092972288E0F3
:10A7E00080939F271FC180919F22853409F075C6F1
:10A7F0001091A12200E08091A222080F111D8091EA
:10A800009722909198228017910708F466C61093BA
:10A810009822009397228091A52290E08F739070E8
:10A82000009709F05AC68091A622882309F055C6E0
:10A830004091362850913728A0900B06B0900C0616
:10A840004A155B0559F48091382890913928209158
:10A850000D0630910E0682179307A1F08091AF226A
:10A860009091B0228417950709F037C62091B12244
:10A870003091B222809138289091392828173907D1
:10A8800009F02BC60E948F512FEF8F3F920709F0DE
:10A8900024C68091A822863009F42EC18131D1F1DD
:10A8A000813009F01AC68091B322883009F015C6AC
:10A8B0001092B3228091B5229091B6222FEF873F5C
:10A8C000920710F0099601C008969093B6228093E3
:10A8D000B522EFE9F2E28091AB229091AC22A091F7
:10A8E000AD22B091AE228093AF229093B022A0937C
:10A8F000B122B093B2228091362890913728A0914E
:10A900003828B091392884879587A687B78780E44F
:10A910008087C0C50C511040109398220093972255
:10A920008BEB92E29093A3278093A2278091B92288
:10A930009091BA22009739F00E94A4512FEF8F3FD7
:10A94000920709F0CAC54091B5225091B62241152F
:10A95000510509F4C2C58CE398E29093A127809336
:10A96000A0276091B3227091B422A0910D06B091FE
:10A970000E06C0910F06D09110060091110610919D
:10A980001206E090AB22F090AC22C090AD22D090A5
:10A99000AE222EC084819581009721F14817590776
:10A9A00009F586819781009719F068177907D1F426
:10A9B000208131812A153B0529F4828193818A17F0
:10A9C0009B07F9F02C173D0729F4828193818017AA
:10A9D0009107B9F0E216F30629F482819381C81633
:10A9E000D90679F0CF010D969093A1278093A027E7
:10A9F000E091A027F091A12788E2EE3BF80750F202
:10AA00006CC51092A5271092A42782E080939F27FF
:10AA10008BEB92E290939A228093992210923B289A
:10AA200010923A280E946B4D80913A2890913B28D1
:10AA3000009709F452C59C01245E3F4F3093982241
:10AA4000209397223093A1222093A222E091A02765
:10AA5000F091A12720852093A72221E12093A8220D
:10AA600008969827892798279093B8228093B72231
:10AA70001092BA221092B922848195819093B422C7
:10AA80008093B322868197819093B6228093B522DA
:10AA90008091362890913728A0913828B091392894
:10AAA0008093AB229093AC22A093AD22B093AE22C0
:10AAB00080819181A281B3818093AF229093B02253
:10AAC000A093B122B093B22287EC92E29093A32795
:10AAD0008093A2270E94A451809590959093BA22CA
:10AAE0008093B922009709F0D5C48FEF9FEF909320
:10AAF000BA228093B922CEC40E94A0512FEF8F3F7B
:10AB0000920709F0EAC42091B5223091B6222115AE
:10AB1000310509F4E2C44091B3225091B4224115A9
:10AB2000510509F4DAC4E091AB22F091AC22A09176
:10AB3000AD22B091AE22C6EAD7E2698D6623A9F0B4
:10AB40008C819D812817390781F48E819F81481758
:10AB5000590759F488819981E817F90731F48A81F6
:10AB60009B81A817B90709F47AC1A09688E2C6307C
:10AB7000D80719F310F38091C0228F738230B9F493
:10AB80003093C2122093C11240E00DC0E42FF0E0D8
:10AB9000EE0FFF1FEA5DF74D808191814F5F28170F
:10ABA000390709F47DC0443088F34093BA1280918C
:10ABB000C02282FD92C484E18093C02288E290E0AA
:10ABC000909398228093972280E58093BF22809172
:10ABD000BA229091BE229093BA223091B9229091DC
:10ABE000BD229093B9223093BD222091B82290913A
:10ABF000BC229093B8222093BC229091B7229093CC
:10AC0000BA124091BB224093B7229093BB228F5F30
:10AC10008093BE22882379F4832F8F5F8093BD2297
:10AC2000882349F4822F8F5F8093BC22882319F4F4
:10AC30009F5F9093BB228091B3229091B422909316
:10AC4000C2128093C1122091B5223091B622309366
:10AC5000B4222093B3229093B6228093B5228091A0
:10AC6000AB229091AC22A091AD22B091AE22809304
:10AC7000AF229093B022A093B122B093B2228091E0
:10AC8000362890913728A0913828B09139288093A0
:10AC9000AB229093AC22A093AD22B093AE22DFC33F
:10ACA0001092BA1280E0C0E0D0E022C0E82FF0E0BD
:10ACB00075E0EE0FFF1F7A95E1F7EA55F84D918D9B
:10ACC000992321F48093BA12EF0116C0973079F4DA
:10ACD000209721F0228D9A8D921748F4C82FD0E04A
:10ACE00065E0CC0FDD1F6A95E1F7CA55D84D8F5F3F
:10ACF0008430E0F28093BA12209709F4EEC3D09327
:10AD0000A527C093A42783E08A8F888F1E8A84E0BA
:10AD10008F8B1B8E8091B5229091B6229D838C8360
:10AD20008091B3229091B4229F838E838091AB2235
:10AD30009091AC22A091AD22B091AE2288839983EC
:10AD4000AA83BB8381E0898F8091BD128C8780911B
:10AD5000BE128D878091BF128E878091C0128F871F
:10AD600081E090E0998B888B8091BA228B878091CB
:10AD7000B9228A878091B82289878091B7228887F3
:10AD800081E090E00E94A95B8091BF22282F30E0F3
:10AD9000207F3070213531050CF446C082958F70CC
:10ADA00090E00597880F991F880F991F3091C31263
:10ADB00020E031C0E156FD4D30A5332329F4209326
:10ADC000BA121092C31230C0313011F42F5F23C079
:10ADD0003230E9F441A54430D1F42093BA123093D3
:10ADE000C31292A580E023A530E0282B392B3093A5
:10ADF000C2122093C112C90124E0893D920710F0CC
:10AE000088ED94E09B8B8A8B9D8B8C8B0DC041A52C
:10AE1000442331F0240FE22FF0E0E817F90754F251
:10AE20002093BA123093C31280E18093C0228091A4
:10AE3000C02282608093C02282E08093C72284E097
:10AE40008093C8228093C92288ED8093CA228CE225
:10AE500090E0909398228093972280E6ADC2D093A1
:10AE6000A527C093A42710929F274091C02250E0AD
:10AE700042FF03C0198E80E248C28091BF228295B2
:10AE80008F70880F880F8093BA129801281B3109A0
:10AE9000245130403093982220939722862F90E0BF
:10AEA0008F7090708230910539F4CA018F73907061
:10AEB0008231910551F429C08130910531F4CA01E4
:10AEC0008F7390708230910501F12115310529F4BD
:10AED000CA01837090700097C1F09091B722888565
:10AEE000981709F05FC29091B8228985981709F0E8
:10AEF00059C29091B9228A85981709F053C290914E
:10AF0000BA228B85981709F04DC244FF4AC0688960
:10AF100079896115710509F444C0CE010C960E942F
:10AF20004C513091BB2280919B223817D1F5209152
:10AF3000BC2280919C222817A1F59091BD2280917E
:10AF40009D22981771F58091BE2240919E22841710
:10AF500041F53C872D879E878F878B8D8823D1F481
:10AF60002E89888D9A8D891B922F96959695969508
:10AF7000891B280F2E8B87FD81959F89392F369548
:10AF80003695931B980F9F8B822F86958695869575
:10AF9000890F888F81E080939F27888D8A8F198AF7
:10AFA000188A498D50E0CA018F70907084309105E5
:10AFB00009F4B0C18530910564F482309105C9F17E
:10AFC000833091050CF0B6C08130910509F085C23F
:10AFD00011C08630910509F4DDC1863091050CF46D
:10AFE000B9C18730910509F4DDC18830910509F0B8
:10AFF00074C285C180919F2780FF14C083E0898F30
:10B0000080E480939F27198A188A809197229091D3
:10B010009822009709F408C122E420939F270E94F8
:10B02000A95B02C18091C0228F73823009F055C2A2
:10B03000FBCE80919F2780FF72C08091C0228F73CA
:10B04000823109F06CC08091BF22282F30E0207F30
:10B050003070213531050CF446C082958F7090E038
:10B060000597880F991F880F991F3091C31220E010
:10B0700031C0E156FD4D30A5332329F42093BA1297
:10B080001092C31230C0313011F42F5F23C0323020
:10B09000E9F441A54430D1F42093BA123093C3129D
:10B0A00092A580E023A530E0282B392B3093C212E3
:10B0B0002093C112C90124E0893D920710F088ED68
:10B0C00094E09B8B8A8B9D8B8C8B0DC041A5442378
:10B0D00031F0240FE22FF0E0E817F90754F2209343
:10B0E000BA123093C31283E0898F8091B722888788
:10B0F0008091B82289878091B9228A878091BA226B
:10B100008B8781E090E00E94A95B82E480939F2777
:10B11000198A188A109298221092972285C080E28C
:10B1200080939F270E946B4DE091A427F091A52763
:10B13000118E3DCD8091C02280FF25C044FD23C0EB
:10B1400088899989009709F0C8C1809197229091C8
:10B15000982201960E94A95B20919F27822F8061EF
:10B1600080939F278091972290919822009719F0C1
:10B17000226120939F270E946B4D81E090E0998B84
:10B18000888B88E06DC085FF1CC09091C52280E04F
:10B190002091C62230E0282B392B8091A227909154
:10B1A000A327820F931F9093A3278093A2278091B8
:10B1B000972290919822821B930B909398228093D0
:10B1C00097228091972290919822009749F044FD10
:10B1D00007C020919F27226020939F270E94A95B90
:10B1E0009091C12280E02091C222820F911D909304
:10B1F000C2128093C1122C893D892817390710F09B
:10B20000009721F43093C2122093C1128091C11291
:10B210009091C2129B8B8A8B80919F2790E08370C4
:10B220009070009709F459C110923B2810923A2867
:10B230000E946B4D20919F2725FF07C010923B284D
:10B2400010923A28198E84E1AEC024FF0DC01092EE
:10B250003B2810923A2881E090E0998B888B84E01B
:10B26000898F1B8E81E19FC080913A2890913B2865
:10B270000097E9F020FF02C0198A188A28893989C5
:10B280002115310581F42A893B892817390720F4D3
:10B2900030933B2820933A2880913A2890913B287C
:10B2A000998B888B04C030933B2820933A281B8EBF
:10B2B0008091992290919A229093A3278093A2271C
:10B2C00080913A2890913B28009759F08889998974
:10B2D000009739F08896909398228093972288E17E
:10B2E0000BC080919F2781FFF8C088E290E0909387
:10B2F00098228093972280E18093C0225CC0809145
:10B300009F2780FFEAC0198E80E180939F270E94CB
:10B310006B4DE3C08091972290919822009711F095
:10B320000E94A95B9091C02280919F2790FF0BC043
:10B3300080FF06C087E0898F1A8E198A188A19C083
:10B3400086E0898F16C080FF1EC085E0898F198A2C
:10B35000188AC3C08091972290919822009711F08B
:10B360000E94A95B8091C02280FF0DC087E0898F79
:10B370001A8E81E090E00E94A95B80E180939F2774
:10B380000E946B4D0FC08091972290919822009758
:10B3900049F4A3C080919F2780FF9FC087E0898FD9
:10B3A0001A8E9BC080E18093C02288E290E0909347
:10B3B00098228093972280E58093BF22888580938E
:10B3C000BB2289858093BC228A858093BD228B8590
:10B3D0008093BE228C858093B7228D858093B8227E
:10B3E0008E858093B9228F858093BA2286E08093E0
:10B3F000A8228C819D819093B4228093B3228E8168
:10B400009F819093B6228093B522809136289091A7
:10B410003728A0913828B09139288093AB22909397
:10B42000AC22A093AD22B093AE2288819981AA81EB
:10B43000BB818093AF229093B022A093B122B093AE
:10B44000B222898D84FF05C01092C2221092C122BF
:10B4500006C084E08093C12288ED8093C22280E4FC
:10B460008093A72280919722909198229093A12275
:10B470008093A2221092C6221092C5221092C4225A
:10B480001092C3220E94A051809590959093C4225F
:10B490008093C32285E480939F221092A022109271
:10B4A000A6221092A5228091B8129091B91201960D
:10B4B0009093B9128093B8129093A3228093A42200
:10B4C0001092AA221092A9220E948F5180959095E5
:10B4D0009093AA228093A92204C0109298221092DD
:10B4E000972210929F27DF91CF911F910F91FF908C
:10B4F000EF90DF90CF90BF90AF9008959827892765
:10B50000982708950F931F93DC01CB011A2F0B2F5F
:10B5100020E030E0982789279827A0E0B0E0DC0100
:10B5200099278827082B192B2A2B3B2BB801C901F7
:10B530001F910F910895FC012091992230919A2238
:10B540008FE997E2821B930BAB01861797070CF4E8
:10B55000AC01141615065CF440933A2850933B282E
:10B56000E217F30721F0C901BF010E94B4640895F6
:10B57000CF92DF92EF92FF920F93CF93DF93CDB7ED
:10B58000DEB760970FB6F894DEBF0FBECDBF0023C5
:10B5900009F45AC029873A874B875C876D877E8775
:10B5A0008F87988B80E2801B49855A856B857C85C7
:10B5B0001816B4F019821A821B821C82992787FD03
:10B5C0009095909581959F4F04C0440F551F661F1D
:10B5D000771F8A95D2F74D835E836F8378872CC05F
:10B5E0006A017B01002E04C0CC0CDD1CEE1CFF1C8C
:10B5F0000A94D2F7C982DA82EB82FC826A017B016B
:10B6000004C0F694E794D794C7948A95D2F7D701EB
:10B61000C6014D855E856F85788904C0440F551F2E
:10B62000661F771F0A95D2F7842B952BA62BB72B75
:10B630008D839E83AF83B88729813A814B815C815A
:10B640006D817E818F81988560960FB6F894DEBFFC
:10B650000FBECDBFDF91CF910F91FF90EF90DF90A4
:10B66000CF900895A0E1B0E0E8E3FBE50C94CD6154
:10B6700029873A874B875C876D877E878F87988B72
:10B68000A982BA82CB82DC82ED82FE820F83188788
:10B690004D855E856F8578898D819E81AF81B88566
:10B6A000481759076A077B07C8F084179507A6074C
:10B6B000B70790F049855A856B857C8589819A8189
:10B6C000AB81BC81481759076A077B0738F084179C
:10B6D0009507A607B70720F482E003C080E001C009
:10B6E00081E06096EAE00C94E96180E88093610073
:10B6F000109261000E946C360E94282B0E94CB3A67
:10B700008091462090914720009729F001979093CF
:10B71000472080934620C0904820D0904920E09058
:10B720004A20F0904B200E947039DC01CB01C816F2
:10B73000D906EA06FB0601F30E947039DC01CB0151
:10B740008093482090934920A0934A20B0934B20A7
:10B75000D3CFBC018091A4279091A52708960E9481
:10B760004C51E091A427F091A52780919B228087DE
:10B7700080919C22818780919D22828780919E2248
:10B78000838708952F923F924F925F926F927F929C
:10B790008F929F92AF92BF92CF92DF92EF92FF92E1
:10B7A0000F931F93CF93DF93CDB7DEB765970FB697
:10B7B000F894DEBF0FBECDBF4C017F876E87FC01C2
:10B7C00017821682838181FD04C076C34C855D8516
:10B7D00004C01E010894211C311CF4019381EE85E4
:10B7E000FF8593FD859193FF8191FF87EE878823E5
:10B7F00009F45EC3853241F493FD859193FF8191F5
:10B80000FF87EE87853259F490E0B4014C8B5D8B55
:10B810000E9407654C895D895D874C87D7CFFF24DF
:10B82000DD2410E01032B0F48B3269F08C3228F451
:10B83000803251F0833271F40BC08D3239F0803395
:10B8400049F411602CC01260146029C0186027C030
:10B85000106125C017FD2EC0282F20532A3098F4E0
:10B8600016FF08C08F2D880FF82EFF0CFF0CF80E66
:10B87000F20E15C08D2D880FD82EDD0CDD0CD80EE4
:10B88000D20E10620CC08E3221F416FD11C310646A
:10B8900006C08C3611F4106802C0883659F4EE8563
:10B8A000FF8593FD859193FF8191FF87EE87882324
:10B8B00009F0B8CF982F9554933018F41061805E3A
:10B8C00006C0982F9556933008F0A2C11F7E16FD32
:10B8D00002C0E6E0FE2E1F73853611F4106406C028
:10B8E000863611F4106802C0F110FA9417FF07C0F1
:10B8F000FBE3FF1548F0EF2CE39427E00DC027E0B1
:10B900002F1530F02F2D07C027E07CE3E72E04C071
:10B9100027E067E0F62EEE24CA0104969D878C8707
:10B92000FA016081718182819381A1010E2D0E94B3
:10B93000C4635C01C9802C2D30E0398B288BC0FE9C
:10B9400003C0388933FF06C011FD06C012FF06C0D0
:10B9500000E205C00DE203C00BE201C000E08889EF
:10B9600099898C709070009709F43CC0002311F005
:10B9700084E001C083E08D1558F4D81A13FD09C086
:10B9800080E290E0B4010E940765DA94C9F701C033
:10B99000DD24002329F0802F90E0B4010E94076588
:10B9A000888983FD05C032EDE32E3BE0F32E11C004
:10B9B0002EECE22E2BE0F22E0CC00115110509F041
:10B9C000805290E0B4010E9407650894E11CF11CCC
:10B9D00004C0012F10E000711070F70184918823DA
:10B9E00061F763C217FF0EC0EA0CF889F4FF04C0C8
:10B9F0008A81813309F4EA941E144CF528E02E154F
:10BA000048F12CC016FD2AC08F2D90E08A159B05A9
:10BA100044F03CEFA3163FEFB3061CF0106801C0E2
:10BA2000FA94FF2049F0E2E0F0E0EC0FFD1FEF0D8B
:10BA3000F11D80818033A1F317FF10C0EF2CE39438
:10BA40008F2D90E0A816B90644F4FA1807C0EE242A
:10BA5000E39404C098E0E92E01C0FF2417FF07C05B
:10BA60001A141B043CF495012F5F3F4F05C025E0DD
:10BA700030E002C021E030E0002311F02F5F3F4FA3
:10BA8000FF2029F08F2D90E00196280F391F8D2D72
:10BA900090E02817390714F4D21A01C0DD24612E72
:10BAA0007724C30189709070009749F406C080E242
:10BAB00090E0B4010E940765DA94DD20C1F700230D
:10BAC00029F0802F90E0B4010E94076563FC09C053
:10BAD00006C080E390E0B4010E940765DA94DD209F
:10BAE000C1F717FF48C08501B7FE02C000E010E0B3
:10BAF0004424552495012E1931093B8B2A8B35019D
:10BB0000601A710A620C731C6F2D70E0EE24FF2422
:10BB1000E61AF70A3FEF0F3F130729F48EE290E091
:10BB2000B4010E940765A016B10654F02A893B892A
:10BB3000201731072CF4F301E40DF51D818101C0BC
:10BB400080E3015010400894411C511C0E151F0544
:10BB50002CF090E0B4010E940765DCCF0A151B05AC
:10BB600041F49A81963320F4953319F4388934FFDF
:10BB700081E390E049C08A81813311F09FEEC922B0
:10BB800090E0B4010E940765FF2089F08EE290E00A
:10BB9000B4010E94076512E0F101E10FF11D1F5F82
:10BBA000808190E0B4010E940765FA94A9F764FED1
:10BBB00003C085E490E002C085E690E0B4010E94F5
:10BBC0000765B7FC05C0A114B10441F4C4FE06C06A
:10BBD000B094A194B108B3948DE201C08BE290E0DF
:10BBE000B4010E94076580E305C08F5FE6EFFFEFB9
:10BBF000AE0EBF1EFAE0AF16B104BCF790E0B40180
:10BC00000E940765C501C096B4010E9407654DC139
:10BC1000833631F0833789F0833509F059C022C06B
:10BC20009A012E5F3F4F3D872C87FA0180818983DF
:10BC300081E0E82EF12C510113C09A012E5F3F4F95
:10BC40003D872C87FA01A080B18016FF03C06F2DBD
:10BC500070E002C06FEF7FEFC5010E94CD647C01F0
:10BC60001F7714C09A012E5F3F4F3D872C87FA0142
:10BC7000A080B18016FF03C06F2D70E002C06FEF8F
:10BC80007FEFC5010E94A4647C01106813FD1CC0F5
:10BC900006C080E290E0B4010E940765DA948D2D21
:10BCA00090E0E816F906A8F30FC0F50117FD85919D
:10BCB00017FF81915F0190E0B4010E940765D110E8
:10BCC000DA940894E108F108E114F10471F7EDC089
:10BCD000843611F0893671F59A0117FF0AC02C5F7E
:10BCE0003F4F3D872C87FA0180819181A281B381EA
:10BCF0000BC02E5F3F4F3D872C87FA0180819181D9
:10BD0000AA2797FDA095BA2F012F0F76B7FF08C07D
:10BD1000B095A095909581959F4FAF4FBF4F00680C
:10BD2000BC01CD01A1012AE030E00E940F66E82E9F
:10BD3000E21841C0853721F41F7E2AE030E020C0A0
:10BD4000197F8F36A9F0803720F4883509F0B0C00C
:10BD50000BC0803721F0883709F0AAC001C01061FC
:10BD600014FF09C0146007C014FF08C0166006C0A5
:10BD700028E030E005C020E130E002C020E132E000
:10BD8000CA0117FF09C004969D878C87FA0160815C
:10BD900071818281938108C002969D878C87FA0108
:10BDA0006081718180E090E0A1010E940F66E82E21
:10BDB000E218012F0F7706FF09C00E7FEF1430F451
:10BDC00004FF06C002FD04C00F7E02C01E2D01C08C
:10BDD0001F2D802F90E004FF0CC0FE01EE0DF11D21
:10BDE0002081203311F4097E09C002FF06C01E5FC6
:10BDF00005C086789070009709F01F5FA02EBB24C5
:10BE000003FD12C000FF0DC0FE2C1D1550F4FD0CEB
:10BE1000F11A1D2D06C080E290E0B4010E94076572
:10BE20001F5F1D15C0F304C01D1510F4D11A01C009
:10BE3000DD24A4FE0FC080E390E0B4010E940765FA
:10BE4000A2FE1FC0A1FE03C088E590E010C088E7F5
:10BE500090E00DC0C50186789070009791F0A1FC2C
:10BE600002C080E201C08BE207FD8DE290E0B401E8
:10BE70000E94076506C080E390E0B4010E94076558
:10BE8000FA94EF14C0F3EA94F101EE0DF11D8081F4
:10BE900090E0B4010E940765EE20A9F706C080E299
:10BEA00090E0B4010E940765DA94DD20C1F78ECCE2
:10BEB000F4018681978102C08FEF9FEF65960FB6E0
:10BEC000F894DEBF0FBECDBFDF91CF911F910F91D0
:10BED000FF90EF90DF90CF90BF90AF909F908F90AA
:10BEE0007F906F905F904F903F902F9008955058A3
:10BEF000BB27AA270ED044C135D130F03AD120F06B
:10BF000031F49F3F11F41EF42AC10EF4E095E7FBD3
:10BF100020C1E92F46D180F3BA176207730784075F
:10BF2000950718F071F49EF55EC10EF4E0950B2EA6
:10BF3000BA2FA02D0B01B90190010C01CA01A0017B
:10BF40001124FF27591B99F0593F50F4503E68F1D6
:10BF50001A16F040A22F232F342F4427585FF3CF17
:10BF6000469537952795A795F0405395C9F77EF4E8
:10BF70001F16BA0B620B730B840BBAF09150A1F031
:10BF8000FF0FBB1F661F771F881FC2F70EC0BA0FB7
:10BF9000621F731F841F48F4879577956795B7953F
:10BFA000F7959E3F08F0B3CF9395880F08F0992737
:10BFB000EE0F979587950895A8D008F481E008952D
:10BFC0000CD0DEC0D6D040F0CDD030F021F45F3FB1
:10BFD00019F0BFC0511108C1C2C0E3D098F3992332
:10BFE000C9F35523B1F3951B550BBB27AA2762173D
:10BFF0007307840738F09F5F5F4F220F331F441F82
:10C00000AA1FA9F333D00E2E3AF0E0E830D09150B9
:10C010005040E695001CCAF729D0FE2F27D0660FA6
:10C02000771F881FBB1F261737074807AB07B0E8E5
:10C0300009F0BB0B802DBF01FF2793585F4F2AF0FB
:10C040009E3F510568F085C0CFC05F3FECF3983E3E
:10C05000DCF3869577956795B795F7959F5FC9F758
:10C06000880F911D9695879597F90895E1E0660FE1
:10C07000771F881FBB1F621773078407BA0720F05A
:10C08000621B730B840BBA0BEE1F88F7E0950895C3
:10C09000E89409C097FB3EF4909580957095619562
:10C0A0007F4F8F4F9F4F9923A9F0F92F96E9BB2718
:10C0B0009395F695879577956795B795F111F8CF94
:10C0C000FAF4BB0F11F460FF1BC06F5F7F4F8F4FFF
:10C0D0009F4F16C0882311F096E911C0772321F0F5
:10C0E0009EE8872F762F05C0662371F096E8862F8D
:10C0F00070E060E02AF09A95660F771F881FDAF7E4
:10C10000880F9695879597F90895990F0008550F10
:10C11000AA0BE0E8FEEF16161706E807F907C0F0CD
:10C1200012161306E407F50798F0621B730B840BD5
:10C13000950B39F40A2661F0232B242B252B21F4AF
:10C1400008950A2609F4A140A6958FEF811D811D4F
:10C15000089597F99F6780E870E060E008959FEF89
:10C1600080EC089500240A9416161706180609068E
:10C17000089500240A94121613061406050608955D
:10C18000092E0394000C11F4882352F0BB0F40F4E5
:10C19000BF2B11F460FF04C06F5F7F4F8F4F9F4F25
:10C1A000089557FD9058440F551F59F05F3F71F0A7
:10C1B0004795880F97FB991F61F09F3F79F087950E
:10C1C0000895121613061406551FF2CF4695F1DF97
:10C1D00008C0161617061806991FF1CF8695710527
:10C1E000610508940895E894BB2766277727CB015B
:10C1F00097F908950BD0C4CFB5DF28F0BADF18F057
:10C20000952309F0A6CFABCF1124EECFCADFA0F360
:10C21000959FD1F3950F50E0551F629FF001729FDB
:10C22000BB27F00DB11D639FAA27F00DB11DAA1FFA
:10C23000649F6627B00DA11D661F829F2227B00D47
:10C24000A11D621F739FB00DA11D621F839FA00DD2
:10C25000611D221F749F3327A00D611D231F849F22
:10C26000600D211D822F762F6A2F11249F57504079
:10C270008AF0E1F088234AF0EE0FFF1FBB1F661F14
:10C28000771F881F91505040A9F79E3F510570F0CD
:10C2900060CFAACF5F3FECF3983EDCF386957795AD
:10C2A0006795B795F795E7959F5FC1F7FE2B880FC8
:10C2B000911D9695879597F90895629FD001739F78
:10C2C000F001829FE00DF11D649FE00DF11D929F32
:10C2D000F00D839FF00D749FF00D659FF00D992771
:10C2E000729FB00DE11DF91F639FB00DE11DF91F95
:10C2F000BD01CF0111240895AA1BBB1B51E107C04A
:10C30000AA1FBB1FA617B70710F0A61BB70B881FE5
:10C31000991F5A95A9F780959095BC01CD01089574
:10C3200097FB092E07260AD077FD04D0E5DF06D05B
:10C3300000201AF4709561957F4F0895F6F7909557
:10C3400081959F4F0895A1E21A2EAA1BBB1BFD01E8
:10C350000DC0AA1FBB1FEE1FFF1FA217B307E407E4
:10C36000F50720F0A21BB30BE40BF50B661F771F3C
:10C37000881F991F1A9469F760957095809590951C
:10C380009B01AC01BD01CF0108952F923F924F92C6
:10C390005F926F927F928F929F92AF92BF92CF9255
:10C3A000DF92EF92FF920F931F93CF93DF93CDB75E
:10C3B000DEB7CA1BDB0B0FB6F894DEBF0FBECDBFD6
:10C3C00009942A88398848885F846E847D848C84A7
:10C3D0009B84AA84B984C884DF80EE80FD800C81B0
:10C3E0001B81AA81B981CE0FD11D0FB6F894DEBF93
:10C3F0000FBECDBFED0108958F929F92AF92BF9275
:10C40000CF92DF92EF92FF92CF93DF93EC0188817E
:10C410009981AA81BB810097A105B10521F484E22D
:10C4200099EDABE5B7E0BC01CD012DE133EF41E083
:10C4300050E00E94426849015A0127EA31E440E095
:10C4400050E00E945D616B017C01C501B4012CEEDE
:10C4500034EF4FEF5FEF0E945D61DC01CB01C80E4E
:10C46000D91EEA1EFB1EF7FE08C08FEF9FEFAFEF4D
:10C47000BFE7C80ED91EEA1EFB1EC882D982EA8217
:10C48000FB82C6019F77DF91CF91FF90EF90DF9005
:10C49000CF90BF90AF909F908F9008950E94FC61C5
:10C4A000089583E196E00E94FC610895A0E0B0E069
:10C4B0008093130690931406A0931506B093160666
:10C4C00008953F924F925F926F927F928F929F92C8
:10C4D000AF92BF92CF92DF92EF92FF920F931F9392
:10C4E000CF93DF9300D000D0CDB7DEB72B017A0118
:10C4F0006115710529F0DB018C9311969C931197BE
:10C50000E114F10439F09701225030402332310513
:10C5100008F0FCC06C0186010894C11CD11CF80114
:10C5200030803601832D90E00E949C64009799F73B
:10C53000FDE23F1661F4D80111963C90119792E00C
:10C54000692E712C600E711ECC24C3940BC0BBE20B
:10C550003B1639F4F801318082E0682E712C600EB0
:10C56000711ECC24E114F10421F0F0E1EF16F10486
:10C57000F9F480E3381691F4D3018C91883711F0E7
:10C58000883561F4F301318082E090E0680E791E15
:10C5900092E0C92AB0E1EB2EF12C0AC0E114F104BB
:10C5A00039F4A0E33A16D1F0AAE0EA2EF12C30C01B
:10C5B000BAE0EB16F10461F1E0E1EE16F10429F0C6
:10C5C000F8E0EF16F104B1F409C0FFEF8F2EFFEF92
:10C5D0009F2EFFEFAF2EFFE0BF2E22C078E0E72EA8
:10C5E000F12CEFEF8E2EEFEF9E2EEFEFAE2EEFE160
:10C5F000BE2E16C09701442737FD4095542F6FEF8C
:10C600007FEF8FEF9FEF0E94A36149015A0108C09D
:10C6100069E9862E69E9962E69E9A62E69E1B62EAA
:10C6200040E000E010E020E030E0C701AA2797FDDD
:10C63000A095BA2F89839A83AB83BC8350EDD52E06
:10C64000D30C99E09D1570F4832D81548A3118F430
:10C6500099ECD92E06C0832D81568A3168F589EA76
:10C66000D82ED30C8D2D90E08E159F052CF54F3FC5
:10C67000F9F080169106A206B306B8F0C901B80118
:10C6800029813A814B815C810E945D618B019C0113
:10C690008D2D90E0A0E0B0E0080F191F2A1F3B1F6E
:10C6A000081719072A073B0710F44FEF01C041E0B4
:10C6B000D3013D903D01C2CF4114510489F0442380
:10C6C00039F0089461087108F2017182608208C033
:10C6D000C1FE06C0C3010297D20111969C938E93AE
:10C6E000C0FE07C030952095109501951F4F2F4F24
:10C6F0003F4F47FF0FC082E290E09093C5288093A0
:10C70000C4280FEF1FEF2FEF3FEF04C000E010E051
:10C7100020E030E0B801C9010F900F900F900F900A
:10C72000DF91CF911F910F91FF90EF90DF90CF900D
:10C73000BF90AF909F908F907F906F905F904F9041
:10C740003F900895662777270C94A866FC018827F8
:10C750009927E89421912032E9F3293010F02E3006
:10C76000C8F32B3241F02D3239F4689404C00E9492
:10C77000FF64820F911D219120532A30C0F31EF4D3
:10C78000909581959F4F0895283008F027E0332732
:10C79000DA01990F311D87FD9160009661057105E1
:10C7A00039F432602E5F3D9330E32A95E1F7089526
:10C7B0009F3F30F080387105610509F03C5F3C5FB8
:10C7C0003D93913008F08068911DDF93CF931F93C4
:10C7D0000F93FF92EF92192F987F9695E92F9695D8
:10C7E0009695E90FFF27E05DF34F99273327EE2455
:10C7F000FF24A701E70105900894079428F4360F59
:10C80000E71EF81E491F511D660F771F881F991FCD
:10C810000694A1F70590079428F4E70EF81E491F27
:10C82000561FC11D770F881F991F661F0694A1F719
:10C830000590079428F4F80E491F561FC71FD11DF5
:10C84000880F991F661F771F0694A1F7059007941C
:10C8500020F4490F561FC71FD81F990F661F771F57
:10C86000881F0694A9F784911095177041F0D6950A
:10C87000C79557954795F794E7941A95C1F7E6ED54
:10C88000FBE068941590159135916591959105900F
:10C890007FE27395E118F10A430B560BC90BD009DF
:10C8A000C0F7E10CF11E431F561FC91FD01D7EF4B7
:10C8B000703311F48A95E6CFE894015030F0080FF8
:10C8C0000AF40027021708F4202F2395022F7A3349
:10C8D00028F079E37D932A95E9F710C07D932A9596
:10C8E00089F6069497956795379517951794E118EB
:10C8F000F10A430B560BC90BD00998F023957E9192
:10C9000073957A3308F070E37C932013B8F77E9127
:10C9100070617D9330F0839571E37D9370E32A9588
:10C92000E1F71124EF90FF900F911F91CF91DF91CC
:10C93000992787FD90950895911189C3803219F048
:10C9400089508550D0F70895FC01059061507040E2
:10C950000110D8F7809590958E0F9F1F089544EC95
:10C9600052E10E94D8640895FB01DC0102C00190ED
:10C970000D9241505040D8F70895DC0101C06D93ED
:10C9800041505040E0F70895FB01DC018D9101908A
:10C9900080190110D9F3990B0895FC016150704082
:10C9A00001900110D8F7809590958E0F9F1F0895E4
:10C9B000FA01A191B081009719F41097E1F0CD012F
:10C9C000DC01CD010D90002011F4C00113C0FB016A
:10C9D0002191222319F02015D9F7F3CFFB012191E2
:10C9E000201519F41E92119606C02223C1F70D904E
:10C9F0000020A1F7D001FA01A193B08308957AE055
:10CA0000979F902D879F802D910D112408950F934E
:10CA10001F93CF93DF938C01EB018B8181FF1BC0B0
:10CA200082FF0DC02E813F818C819D81281739079F
:10CA300064F4E881F9810193F983E88306C0E8850D
:10CA4000F985802F0995009731F48E819F81019699
:10CA50009F838E8302C00FEF1FEFC801DF91CF913C
:10CA60001F910F910895CF93DF93CDB7DEB7FE01ED
:10CA70003596619171918091C0289091C128AF0144
:10CA80000E94C25BDF91CF910895CF93DF93CDB722
:10CA9000DEB7FE013596619171918091C028909129
:10CAA000C128DC0113962C911397286013962C93C0
:10CAB000AF010E94C25BE091C028F091C1282381A0
:10CAC000277F2383DF91CF9108956091C0287091D3
:10CAD000C1280E94076508950F931F93CF93DF939A
:10CAE0008C01E091C028F091C128838181FF1AC098
:10CAF000C0E0D0E005C00995009711F0CFEFDFEF5F
:10CB0000F80181918F016091C0287091C128DB01EB
:10CB10001896ED91FC911997882369F78AE0099599
:10CB2000009711F0CFEFDFEFCE01DF91CF911F9192
:10CB30000F9108950F931F93CF93DF93CDB7DEB777
:10CB40002E970FB6F894DEBF0FBECDBF0D891E899C
:10CB50008F89988D26E02C831A83098397FF02C062
:10CB600080E090E801979E838D83AE01455E5F4F24
:10CB7000CE010196698D7A8D0E94C25B4D815E81E6
:10CB800057FD0AC02F813885421753070CF49A01CC
:10CB9000020F131FF80110822E960FB6F894DEBF15
:10CBA0000FBECDBFDF91CF911F910F9108950F93CD
:10CBB0001F93CF93DF93CDB7DEB72E970FB6F894C0
:10CBC000DEBF0FBECDBF8C0186E08C831A83098344
:10CBD00077FF02C060E070E8615070407E836D8333
:10CBE000CE010196BA01A9010E94C25B4D815E810E
:10CBF00057FD0AC02F813885421753070CF49A015C
:10CC0000020F131FF80110822E960FB6F894DEBFA4
:10CC10000FBECDBFDF91CF911F910F910895FA0103
:10CC2000AA27283051F1203181F1E8946F936E7F6B
:10CC30006E5F7F4F8F4F9F4FAF4FB1E03ED0B4E05C
:10CC40003CD0670F781F891F9A1FA11D680F791F9D
:10CC50008A1F911DA11D6A0F711D811D911DA11DAE
:10CC600020D009F468943F912AE0269F11243019BE
:10CC7000305D3193DEF6CF010895462F4770405D59
:10CC80004193B3E00FD0C9F7F6CF462F4F70405D08
:10CC90004A3318F0495D31FD4052419302D0A9F763
:10CCA000EACFB4E0A6959795879577956795BA955D
:10CCB000C9F700976105710508959B01AC010A2E23
:10CCC00006945795479537952795BA95C9F7620FFA
:10CCD000731F841F951FA01D0895DC01CB01FC016B
:10CCE000F999FECF06C0F2BDE1BDF89A319600B4C5
:10CCF0000D9241505040B8F70895F999FECF92BD7A
:10CD000081BDF89A992780B50895A8E1B0E042E086
:10CD100050E00C946F66DC01CB0103C02D910E94A2
:10CD2000966641505040D0F70895262FF999FECFCE
:10CD30001FBA92BD81BD20BD0FB6F894FA9AF99A38
:10CD40000FBE019608950E949566272F0C94966653
:10CD50006F927F928F929F92AF92BF92CF92DF920B
:10CD6000EF92FF920F931F93CF93DF935B016115B7
:10CD7000710521F0DB018C9311969C937C01E701F6
:10CD80000894E11CF11C08816701802F90E00E944B
:10CD90009C640097A1F70D3241F4098142E0C42E52
:10CDA000D12CCC0EDD1E11E009C00B3231F409810B
:10CDB00032E0C32ED12CCC0EDD1E10E0E60121970F
:10CDC000CE0160ED7CE043E050E00E942A680097CD
:10CDD000D1F4E6012296CE0163ED7CE045E050E01F
:10CDE0000E942A68009711F4E6012796A114B10465
:10CDF00019F0F501D183C08330E020E090E81123E1
:10CE000009F40DC107C1CE0168ED7CE043E050E0BC
:10CE10000E942A68009759F4A114B10409F4FCC0D7
:10CE2000C6010296D50111969C938E93F5C040E001
:10CE300050E060E070E08824992400530A3090F5B7
:10CE40001260212F30E0C9018870907012FF06C077
:10CE5000009769F50894811C911C29C0009719F06E
:10CE6000089481089108DB01CA01D2E0880F991F5C
:10CE7000AA1FBB1FDA95D1F7480F591F6A1F7B1FE6
:10CE8000440F551F661F771F400F511D611D711DF7
:10CE90004839B9E95B07B9E96B07B9E17B0738F0B5
:10CEA000146005C00E3F39F413FD43C01860F6014D
:10CEB00001916F01C2CF053311F00531D1F5D601D3
:10CEC000EC91ED3211F4106108C0EB3229F0C6018B
:10CED000019621E030E008C0D6011196EC9111973F
:10CEE000C601029622E030E0E053EA3020F06C0107
:10CEF000C21AD30A1EC0DC0120E030E0FCE020387A
:10CF00003F075CF4C901880F991F880F991F280FEC
:10CF1000391F220F331F2E0F311DED91E0536D018C
:10CF2000EA3060F314FF03C0309521953F4F820E25
:10CF3000931EC12FD0E011FF08C0A114B10429F045
:10CF4000C6010197D5018D939C93CB01BA010E9434
:10CF500048606B017C01CE01837090708330910535
:10CF600021F4F7FAF094F7F8F094C701B60120E045
:10CF700030E040E050E00E94DC5F882309F445C0C7
:10CF800097FE07C09094819491089394C7E0DDE0E8
:10CF900002C0CFEEDCE098EE692E9FEF792E6C0E8A
:10CFA0007D1E20E2A22EB12C0FC0FE01059115912D
:10CFB00025913491C701B601A90198010E94FA6038
:10CFC0006B017C018A189B088A149B0474F72497D0
:10CFD000B594A794C615D705B9F7C601D7012A2F6E
:10CFE000220F2B2F221F2F3F51F0BC01CD0120E03B
:10CFF00030E040E050E00E94DC5F882331F482E2C0
:10D0000090E09093C5288093C4283C2D2D2D9E2D13
:10D010008F2D06C08FEF04C030E020E090EC8FE74A
:10D02000B901AC01872F922FA52FB42FBC01CD01E0
:10D03000DF91CF911F910F91FF90EF90DF90CF90F4
:10D04000BF90AF909F908F907F906F900895992799
:10D0500088270895FB01DC014150504088F08D91F4
:10D0600081341CF08B350CF4805E659161341CF0CA
:10D070006B350CF4605E861B611171F3990B08959A
:10D08000881BFCCF97FB092E05260ED057FD04D038
:10D090005AD90AD0001C38F4509540953095219506
:10D0A0003F4F4F4F5F4F0895F6F7909580957095DD
:0ED0B00061957F4F8F4F9F4F0895F894FFCFEB
:10D0BE00263A202573205B414444523D252D642E93
:10D0CE00252D64205345513D252D6420525353493F
:10D0DE003D252D75204C51493D252D75204452502E
:10D0EE003D252D642E253032645D0A00536368653C
:10D0FE0064756C6564206576656E74206174203D80
:10D10E00256C642066756E633D25780D0A005363A9
:10D11E00686564756C6564206576656E74206E6FE7
:10D12E00773D256C64206E6578743D256C640D0A20
:10D13E0000284578745077722900007374617475F5
:10D14E00733D3078253032780A2000312E3020465B
:10D15E0069726D77617265205665722E20332E309E
:10D16E0020323031322D30392D30320065657072FB
:10D17E006F6D006F6E006F6666004F6E006131005E
:10D18E00726573657400613200765F696E00617559
:10D19E00746F00666C75736800414444523D252DD2
:10D1AE00642E252D64205345513D252D6420525368
:10D1BE0053493D252D75204C51493D252D750A00AD
:10D1CE007472696D0043683D252D64205478507744
:10D1DE00723D252D640A004572726F7220545820DC
:10D1EE004C656E6774683D25640A0049443D002510
:10D1FE00303278002050533D25640020543D252DBB
:10D20E00362E3266002054313D252D362E326600E4
:10D21E0020545F4D43553D252D352E316600205649
:10D22E005F4D43553D252D342E3266002050303D46
:10D23E00252D6C58002050305F543D252D372E3350
:10D24E0066002050313D252D6C58002050315F5422
:10D25E003D252D372E3366002055503D252D6C581B
:10D26E00002052483D252D342E31660020565F4950
:10D27E004E3D252D352E32660020565F41313D251F
:10D28E002D352E32660020565F41323D252D352E2E
:10D29E00326600263A2025730A00545820706B74AB
:10D2AE00206C656E203D2025640A00253032580022
:10D2BE006C656E3D25640A0082046C0456043E04BF
:10D2CE0022040000536C6565702070726F63657385
:10D2DE00730000001404970E0000000062726F616C
:10D2EE0064636173742070726F6365737300000002
:10D2FE002C04862300000000737464696E20707223
:10D30E006F636573730000004804AF0D00000000EA
:10D31E00666F6F2070726F63657373000000600438
:10D32E006C0800000000636D642070726F6365739B
:10D33E00730000007604C9220000000002003C00C9
:10D34E00130A6162636465666768696A6B6C6D6E09
:10D35E006F7020090D00A2041A22FFCC3B22FFCCD5
:10D36E003BED478A3C01001000C20600000D004054
:10D37E00004E068E06000093298729181000000023
:10D38E00004576656E742074696D6572000000D17B
:10D39E00047B2D00000000020306070A0B0E0F434C
:10D3AE006F6E74696B6920322E3500C600C500C4DD
:10D3BE0000C100C200000000CE00CD00CC00C900AC
:10D3CE00CA0000000000000002000000003B3A000E
:10D3DE000000005246323330206472697665720066
:10D3EE0000002305EB3E00000000483D853C3A3F1F
:10D3FE007C40DB3DDE3CE93AE33AD33BC43C0001E2
:10D40E0001010101010101010101010101010052AE
:10D41E00696D65005F05ED41B84161646174612E0F
:10D42E006E756D20776179206F75742074686572E2
:10D43E00653A2025640A00264325432F4553468529
:10D44E00440080C0E0F0F8FCFEFF6E756C6C6D6100
:10D45E0063009A05FF46E446EA46F046F646FC4669
:10D46E00736963736C6F776D616300B005104874F8
:10D47E0047094700471A4806474374696D6572208D
:10D48E0070726F63657373000000C9058F480000EA
:10D49E000000BA0008004D0C550C35000200251294
:10D4AE0027125443502F495020737461636B000050
:10D4BE0000F2058B4B00000000020800000000FF88
:08D4CE00FFFFFF010000000058
:00000001FF
